S01C00005354345F537065637472756D5F576F726B696E672E737265633B
S31508008000000002207DC00308CDC00308CDC00308C8
S31508008010CDC00308CDC00308CDC00308000000008A
S31508008020000000000000000000000000CDC00308AA
S31508008030CDC0030800000000CDC0030845B70308FB
S31508008040CDC00308CDC00308CDC00308CDC00308C2
S31508008050CDC00308CDC00308CDC00308CDC00308B2
S31508008060CDC00308CDC00308CDC00308CDC00308A2
S3150800807049B70308CDC0030855B70308CDC00308A0
S3150800808061B703086DB70308CDC00308CDC0030860
S31508008090CDC00308CDC00308CDC00308CDC0030872
S315080080A0CDC00308CDC00308CDC00308CDC0030862
S315080080B079B7030885B70308CDC00308CDC0030800
S315080080C0CDC00308CDC00308CDC00308CDC0030842
S315080080D0CDC0030891B703089DB70308A9B70308DD
S315080080E0CDC00308CDC00308CDC00308CDC0030822
S315080080F0CDC00308CDC00308CDC00308B5B7030833
S31508008100CDC00308C1B70308CDC00308CDB703081F
S31508008110CDC00308CDC00308CDC00308CDC00308F1
S31508008120CDC00308CDC00308D9B70308E5B70308CF
S31508008130CDC003080000000000000000CDC0030801
S31508008140CDC00308CDC00308CDC00308F1B70308A6
S31508008150CDC00308FDB7030809B80308CDC0030856
S31508008160CDC00308CDC00308CDC00308CDC00308A1
S31508008170CDC00308CDC00308CDC003080000000029
S3150800818000000000CDC00308000000000000000049
S31508008190CDC003080000000000000000CDC00308A1
S315080081A0000000000000000000000000CDC0030829
S315080081B0CDC00308CDC00308CDC00308CDC0030851
S30D080081C0CDC003084433221167
S315080081D010B5054C237833B9044B13B10448AFF3F3
S315080081E000800123237010BD880F002000000000C6
S315080081F0D4E3040808B5034B1BB103490348AFF39E
S31508008200008008BD000000008C0F0020D4E304089D
S3150800821010F8012B11F8013B012A28BF9A42F7D022
S31508008220D01A7047034613F8012B002AFBD1181AF7
S315080082300138704700000000000000000000000040
S3150800824001F0FF01102A2BDB10F0070F08D010F8F9
S31508008250013B013A8B422DD010F0070F42B3F6D1FD
S31508008260F0B441EA012141EA014122F007047FF016
S3150800827000070023F0E80256083C85EA010586EA6D
S31508008280010685FA47F5A3FA87F586FA47F6A5FAA9
S3150800829087F68EB9EED1F0BC01F0FF0102F00702B5
S315080082A032B110F8013B013A83EA010313B1F8D160
S315080082B00020704701387047002D06BF3546033841
S315080082C0073815F0010F07D1013015F4807F02BF7A
S315080082D0013015F4C03F0130F0BC0138704700BFCB
S315080082E081F0004102E000BF83F0004330B54FEA59
S315080082F041044FEA430594EA050F08BF90EA020FC6
S315080083001FBF54EA000C55EA020C7FEA645C7FEA58
S31508008310655C00F0E2804FEA5454D4EB5555B8BF7B
S315080083206D420CDD2C4480EA020281EA030382EAEC
S31508008330000083EA010180EA020281EA0303362D7E
S3150800834088BF30BD11F0004F4FEA01314FF4801C51
S315080083504CEA113102D0404261EB410113F0004F63
S315080083604FEA03334CEA133302D0524263EB43031A
S3150800837094EA050F00F0A780A4F10104D5F1200EB8
S315080083800DDB02FA0EFC22FA05F2801841F1000113
S3150800839003FA0EF2801843FA05F359410EE0A5F1E7
S315080083A020050EF1200E012A03FA0EFC28BF4CF018
S315080083B0020C43FA05F3C01851EBE37101F00045CE
S315080083C007D54FF0000EDCF1000C7EEB00006EEBDB
S315080083D00101B1F5801F1BD3B1F5001F0CD3490865
S315080083E05FEA30004FEA3C0C04F101044FEA4452BC
S315080083F012F5800F80F09A80BCF1004F08BF5FEA43
S31508008400500C50F1000041EB045141EA050130BD22
S315080084105FEA4C0C404141EB0101013C28BFB1F534
S31508008420801FE9D291F0000F04BF01460020B1FA7F
S3150800843081F308BF2033A3F10B03B3F120020CDA52
S315080084400C3208DD02F1140CC2F10C0201FA0CF030
S3150800845021FA02F10CE002F11402D8BFC2F1200C95
S3150800846001FA02F120FA0CFCDCBF41EA0C0190404B
S31508008470E41AA2BF01EB0451294330BD6FEA040494
S315080084801F3C1CDA0C340EDC04F11404C4F120027F
S3150800849020FA04F001FA02F340EA030021FA04F391
S315080084A045EA030130BDC4F10C04C4F1200220FAE8
S315080084B002F001FA04F340EA0300294630BD21FA26
S315080084C004F0294630BD94F0000F83F4801306BFEC
S315080084D081F480110134013D4EE77FEA645C18BFE0
S315080084E07FEA655C29D094EA050F08BF90EA020F77
S315080084F005D054EA000C04BF1946104630BD91EA6F
S31508008500030F1EBF0021002030BD5FEA545C05D171
S315080085104000494128BF41F0004130BD14F58004B0
S315080085203CBF01F5801130BD01F0004545F0FE4124
S3150800853041F470014FF0000030BD7FEA645C1ABF59
S31508008540194610467FEA655C1CBF0B46024650EA90
S31508008550013406BF52EA033591EA030F41F40021BC
S3150800856030BD00BF90F0000F04BF0021704730B542
S315080085704FF4806404F132044FF000054FF0000117
S3150800858050E700BF90F0000F04BF0021704730B5D8
S315080085904FF4806404F1320410F0004548BF4042AD
S315080085A04FF000013EE700BF42004FEAE2014FEA02
S315080085B031014FEA02701FBF12F07F4393F07F4FDD
S315080085C081F06051704732F07F4208BF704793F0E0
S315080085D07F4F04BF41F40021704730B54FF46074F3
S315080085E001F0004521F000411CE700BF50EA0102F6
S315080085F008BF704730B54FF000050AE050EA01029F
S3150800860008BF704730B511F0004502D5404261EB0E
S3150800861041014FF4806404F132045FEA915C3FF44F
S31508008620D8AE4FF003025FEADC0C18BF03325FEAEC
S31508008630DC0C18BF033202EBDC02C2F1200300FA9D
S3150800864003FC20FA02F001FA03FE40EA0E0021FAC2
S3150800865002F11444BDE600BF70B54FF0FF0C4CF4B0
S31508008660E06C1CEA11541DBF1CEA135594EA0C0F62
S3150800867095EA0C0F00F0DEF82C4481EA030621EA9D
S315080086804C5123EA4C5350EA013518BF52EA0335D8
S3150800869041F4801143F4801338D0A0FB02CE4FF08A
S315080086A00005E1FB02E506F00042E0FB03E54FF0BA
S315080086B00006E1FB03569CF0000F18BF4EF0010EB2
S315080086C0A4F1FF04B6F5007F64F5407404D25FEAAE
S315080086D04E0E6D4146EB060642EAC62141EA555161
S315080086E04FEAC52040EA5E504FEACE2EB4F1FD0CA3
S315080086F088BFBCF5E06F1ED8BEF1004F08BF5FEA21
S31508008700500E50F1000041EB045170BD06F00046D2
S3150800871046EA010140EA020081EA0301B4EB5C047F
S31508008720C2BFD4EB0C0541EA045170BD41F4801177
S315080087304FF0000E013C00F3AB8014F1360FDEBF9C
S31508008740002001F0004170BDC4F10004203C35DA78
S315080087500C341BDC04F11404C4F1200500FA05F3FB
S3150800876020FA04F001FA05F240EA020001F000429C
S3150800877021F0004110EBD37021FA04F642EB060112
S315080087805EEA430E08BF20EAD37070BDC4F10C043C
S31508008790C4F1200500FA04F320FA05F001FA04F200
S315080087A040EA020001F0004110EBD37041F10001EC
S315080087B05EEA430E08BF20EAD37070BDC4F12005F7
S315080087C000FA05F24EEA020E20FA04F301FA05F25F
S315080087D043EA020321FA04F001F0004121FA04F207
S315080087E020EA020000EBD3705EEA430E08BF20EAD7
S315080087F0D37070BD94F0000F0FD101F00046400011
S3150800880041EB010111F4801F08BF013CF7D041EA92
S31508008810060195F0000F18BF704703F00046520096
S3150800882043EB030313F4801F08BF013DF7D043EA67
S315080088300603704794EA0C0F0CEA135518BF95EA1D
S315080088400C0F0CD050EA410618BF52EA4306D1D1A4
S3150800885081EA030101F000414FF0000070BD50EAC3
S31508008860410606BF1046194652EA430619D094EA4D
S315080088700C0F02D150EA013613D195EA0C0F05D137
S3150800888052EA03361CBF104619460AD181EA03018B
S3150800889001F0004141F0FE4141F470014FF0000043
S315080088A070BD41F0FE4141F4780170BD70B54FF0DE
S315080088B0FF0C4CF4E06C1CEA11541DBF1CEA13555E
S315080088C094EA0C0F95EA0C0F00F0A7F8A4EB050440
S315080088D081EA030E52EA03354FEA013100F0888037
S315080088E04FEA03334FF0805545EA131343EA126300
S315080088F04FEA022245EA111545EA10654FEA0026B5
S315080089000EF000419D4208BF964244F1FD0404F56D
S31508008910407402D25B084FEA3202B61A65EB0305C9
S315080089205B084FEA32024FF480104FF4002CB6EB86
S31508008930020E75EB030E22BFB61A754640EA0C0006
S315080089405B084FEA3202B6EB020E75EB030E22BF46
S31508008950B61A754640EA5C005B084FEA3202B6EB87
S31508008960020E75EB030E22BFB61A754640EA9C0046
S315080089705B084FEA3202B6EB020E75EB030E22BF16
S31508008980B61A754640EADC0055EA060E18D04FEAD4
S31508008990051545EA16754FEA06164FEAC30343EA74
S315080089A052734FEAC2025FEA1C1CC0D111F4801F41
S315080089B00BD141EA00014FF000004FF0004CB6E73A
S315080089C011F4801F04BF01430020B4F1FD0C88BFD9
S315080089D0BCF5E06F3FF6AFAEB5EB030C04BFB6EBE4
S315080089E0020C5FEA500C50F1000041EB045170BDD7
S315080089F00EF0004E4EEA113114EB5C04C2BFD4EB04
S31508008A000C0541EA045170BD41F480114FF0000E87
S31508008A10013C90E645EA060E8DE60CEA135594EA03
S31508008A200C0F08BF95EA0C0F3FF43BAF94EA0C0F06
S31508008A300AD150EA01347FF434AF95EA0C0F7FF47B
S31508008A4025AF104619462CE795EA0C0F06D152EACF
S31508008A5003353FF4FDAE1046194622E750EA4106B3
S31508008A6018BF52EA43067FF4C5AE50EA41047FF4C4
S31508008A700DAF52EA43057FF4EBAE12E74FF0FF3C29
S31508008A8006E000BF4FF0010C02E000BF4FF0010CFA
S31508008A904DF804CD4FEA410C7FEA6C5C4FEA430C73
S31508008AA018BF7FEA6C5C1BD001B050EA410C0CBFC2
S31508008AB052EA430C91EA030F02BF90EA020F002024
S31508008AC0704710F1000F91EA030F58BF994208BF8B
S31508008AD090422CBFD8176FEAE37040F00100704748
S31508008AE04FEA410C7FEA6C5C02D150EA013C07D19F
S31508008AF04FEA430C7FEA6C5CD6D152EA033CD3D0EA
S31508008B005DF8040B704700BF8446104662468C46E3
S31508008B101946634600E000BF01B5FFF7B7FF002816
S31508008B2048BF10F1000F01BD4DF808EDFFF7F4FF3F
S31508008B300CBF012000205DF808FB00BF4DF808EDCA
S31508008B40FFF7EAFF34BF012000205DF808FB00BFED
S31508008B504DF808EDFFF7E0FF94BF012000205DF80F
S31508008B6008FB00BF4DF808EDFFF7CEFF94BF0120C4
S31508008B7000205DF808FB00BF4DF808EDFFF7C4FFBD
S31508008B8034BF012000205DF808FB00BF4FEA410C06
S31508008B907FEA6C5C02D150EA013C0AD14FEA430CE9
S31508008BA07FEA6C5C02D152EA033C02D14FF0000026
S31508008BB070474FF0010070474FEA410212F5001264
S31508008BC015D211D56FF47873B3EB625212D94FEA06
S31508008BD0C12343F0004343EA505311F0004F23FAF0
S31508008BE002F018BF404270474FF00000704750EA45
S31508008BF0013005D111F0004008BF6FF00040704702
S31508008C004FF00000704700BF4A0011D212F500125B
S31508008C1011D20DD56FF47873B3EB62520ED44FEAC6
S31508008C20C12343F0004343EA505323FA02F0704746
S31508008C304FF00000704750EA013002D14FF0FF3084
S31508008C4070474FF0000070474FEA4102B2F1E04327
S31508008C5024BFB3F5001CDCF1FE5C0DD901F0004C15
S31508008C604FEAC0024CEA5070B2F1004F40EB830065
S31508008C7008BF20F00100704711F0804F21D113F191
S31508008C803872BCBF01F00040704741F480114FEACA
S31508008C905252C2F11802C2F1200C10FA0CF320FA53
S31508008CA002F018BF40F001004FEAC1234FEAD32370
S31508008CB003FA0CFC40EA0C0023FA02F34FEA4303DA
S31508008CC0CCE77FEA625307D150EA01331EBF4FF063
S31508008CD0FE4040F44000704701F0004040F0FE407E
S31508008CE040F40000704700BF53B94AB9002908BFCD
S31508008CF000281CBF4FF0FF314FF0FF3000F0A4B939
S31508008D00ADF1080C6DE904CE00F03CF8DDF804E09E
S31508008D10DDE9022304B0704738B500220023044673
S31508008D200D46FFF70BFF28B920462946BDE838400F
S31508008D3000F00AB8204605F1004100F005F8404267
S31508008D4061EB410138BD00BFD0B50C4B0022064689
S31508008D500F46FFF781FCFFF757FF0446FFF702FCB3
S31508008D60074B0022FFF778FC02460B463046394689
S31508008D70FFF7BAFAFFF748FF2146D0BD0000F03DDD
S31508008D800000F0412DE9F047089D04468C46002B6B
S31508008D9040F083808A42174647D9B2FA82F242B136
S31508008DA0C2F1200024FA00F09140974040EA010CF5
S31508008DB094404FEA1748230CBCFBF8F61FFA87FEC7
S31508008DC008FB16C143EA014306FB0EF1994209D98D
S31508008DD0FB1806F1FF3080F01981994240F216819E
S31508008DE0023E3B445B1AA4B2B3FBF8F008FB10330F
S31508008DF044EA034400FB0EFEA64509D93C1900F1D6
S31508008E00FF3380F00581A64540F2028102383C44D2
S31508008E1040EA0640A4EB0E0400261DB1D440002308
S31508008E20C5E900433146BDE8F08702B9FFDEB2FA6C
S31508008E3082F2002A50D1CB1B4FEA174E1FFA87F849
S31508008E400126B3FBFEFC210C0EFB1C3341EA034151
S31508008E5008FB0CF38B4207D979180CF1FF3002D2C4
S31508008E608B4200F2E9808446C91AA3B2B1FBFEF030
S31508008E700EFB101143EA014408FB00F8A04507D988
S31508008E803C1900F1FF3302D2A04500F2D9801846FA
S31508008E90A4EB080440EA0C40BFE78B4209D9002D31
S31508008EA000F0B1800026C5E9000130463146BDE82C
S31508008EB0F087B3FA83F6002E4AD18B4202D3824258
S31508008EC000F2B880841A61EB030101208C46002D5C
S31508008ED0A8D0C5E9004CA5E7C2F1200320FA03F69D
S31508008EE0974001FA02F04FEA174ED9403043030C77
S31508008EF0B1FBFEF61FFA87F80EFB161143EA01438B
S31508008F0006FB08F1994204FA02F409D9FB1806F19E
S31508008F10FF3C80F08D80994240F28A80023E3B44B5
S31508008F205B1A81B2B3FBFEF00EFB103341EA034134
S31508008F3000FB08F38B4207D9791800F1FF3C73D27E
S31508008F408B4271D902383944CB1A40EA064678E78B
S31508008F50C6F1200C03FA06F422FA0CF31C4320FA95
S31508008F600CF701FA06F34FEA144E21FA0CF11F43E7
S31508008F703B0CB1FBFEF91FFA84F80EFB191143EA04
S31508008F80014109FB08FA8A4502FA06F200FA06F3D5
S31508008F9008D9611809F1FF3048D28A4546D9A9F19E
S31508008FA002092144A1EB0A01BFB2B1FBFEF00EFB98
S31508008FB0101147EA014700FB08F8B84507D9E71931
S31508008FC000F1FF312ED2B8452CD90238274440EAA1
S31508008FD00940A7EB0807A0FB02894F45C646494644
S31508008FE01AD317D05DB1B3EB0E0267EB010707FA88
S31508008FF00CFCF2404CEA0202F740C5E900270026BD
S315080090003146BDE8F0872E4628460BE70646E9E6D0
S315080090101846FDE64345E5D2B8EB020E69EB0401B6
S315080090200138DFE70846D2E760468DE78146B9E7AB
S31508009030664675E730464AE7ACF1020C394413E751
S3150800904002383C4424E700BF704700BFF8B572B148
S3150800905006460C468F180025336814F8011B1B6852
S3150800906030469847A7420544F6D12846F8BD154626
S315080090702846F8BD2DE9F8430668DFF87C9077683E
S3150800908004460D4659B30846FFF7CCF84F458046C7
S3150800909027D160B12F184FF00008336815F8011B67
S315080090A020469847BD4226688044F6D177684F45E2
S315080090B00ED133680D212046984722680346126868
S315080090C020460A211C46904720444044BDE8F883C0
S315080090D0084920460222B8474044BDE8F883884636
S315080090E0E5E7024629462046B84726688046776857
S315080090F0DDE700BFBCE504084D9000084FF0FF30DF
S31508009100704700BF704700BF10B54FF0FF331446D5
S31508009110006992B238F002FB204610BD00B583B054
S315080091204FF0FF3301220DF10701006938F0A4FB67
S315080091309DF8070003B05DF804FB00BF10B504688E
S315080091400B4A646882B094428DF807100AD14FF032
S31508009150FF3301220DF10701006938F0DFFA01201B
S3150800916002B010BD01220DF10701A04702B010BDE3
S3150800917009910008F8B50026C0E90066044686602D
S3150800918079B108460D46FFF74DF80746013040F01D
S315080091904DFE30B1C4E900070670A760294641F0C4
S315080091A07DFC2046F8BD00BFF8B588424FF00005A3
S315080091B0C0E90055044685600DD00E685EB18F681B
S315080091C0781C40F033FE30B1C4E900070570A7608B
S315080091D0314641F063FC2046F8BD00BF30B4D1E902
S315080091E000258C6802600022C0E90154C1E900220A
S315080091F030BC8A60704700BF10B50446006840F06E
S315080092001DFE204610BD00BF884270B504461FD01B
S315080092100D680068ADB18E6810B163689E4209D9C1
S31508009220711C41F06FFB58B1A368C4E900060BB97D
S3150800923003702068A660294641F030FC204670BDC0
S31508009240206808B140F0FAFD0023C4E90133236021
S31508009250204670BD884238B5044612D000680D46CF
S3150800926028B162688B689A420DD240F0E7FDD5E9CD
S315080092700031AA6823600023C4E90112C5E9003356
S31508009280AB60204638BD096841F008FCAB68A360AE
S315080092900023AB60204638BD70B50446E1B10846E8
S315080092A00D46FEF7BFFF2368064613B16268904273
S315080092B00BD91846711C41F025FB034660B1A2681C
S315080092C0C4E900060AB902702368A660294618464A
S315080092D041F0E4FB204670BD206808B140F0AEFDC1
S315080092E00023C4E901332360204670BD30B5836886
S315080092F083B0044600688DF8041000225D1C8DF8C2
S31508009300052010B1626895420AD9991C41F0FAFA0B
S3150800931060B1A368C4E9000513B903702068A3689F
S31508009320184401A941F0BAFBA560012003B030BD7D
S31508009330826808B50B463AB161B10068FEF768FF66
S31508009340B0FA80F0400908BD31B11878B0FA80F05B
S31508009350400908BD0368F8E7012008BD82688A420B
S3150800936003D9006808B1084470470248002303700F
S31508009370704700BFA40F00208368934207D910B531
S315080093800468A01841F07DFB20B1001B10BD4FF00A
S31508009390FF3070474FF0FF3010BD00BF9A422DE9ED
S315080093A0F0411746984604460D4601D94746904669
S315080093B00026C4E90066A660012040F037FD08B122
S315080093C020600670AE68BE4202D82046BDE8F0812D
S315080093D046452B6828BF4646002213F806809A554C
S315080093E0296820463944FFF757FF2B6803F806809B
S315080093F02046BDE8F08100BF006808B140F0E7BC30
S31508009400704700BF30B5851840F2FE34A54285B0D6
S315080094101BDCFF280B4616D9B0F5007F18D3B0F52C
S31508009420407F34BFA421A6210E24CDE90032029440
S31508009430C2B20123074834F02DF9042032F098FE11
S31508009440012005B030BDA021EEE7002005B030BDF3
S31508009450A221E9E7E8C0012030B5851840F2FE34BC
S31508009460A54285B01BDCFF280B4616D9B0F5007F50
S3150800947018D3B0F5407F34BFA421A6210E24CDE928
S3150800948000320294C2B20123074834F003F90420DB
S3150800949032F06EFE012005B030BDA021EEE70020B7
S315080094A005B030BDA221E9E7E8C0012010B50B8858
S315080094B086B0841840F2FE315BBA8C42ADF814309F
S315080094C01BDCFF2817D9B0F5007F19D3B0F5407F0C
S315080094D034BFA421A62105AB0E2401920093C2B283
S315080094E001230294074834F0D5F8042032F040FEF0
S315080094F0012006B010BDA021EDE7002006B010BD82
S31508009500A221E8E7E8C0012010B50B6886B08418E8
S3150800951040F2FE311BBA8C4205931BDCFF2817D993
S31508009520B0F5007F19D3B0F5407F34BFA421A6213A
S3150800953005AB0E2401920093C2B201230294084897
S3150800954034F0A8F8042032F013FE012006B010BD4E
S31508009550A021EDE7002006B010BDA221E8E700BF74
S31508009560E8C0012030B5851840F2FE34A54285B022
S3150800957018DCFF280B4613D9B0F5007F15D3B0F5D4
S31508009580407F34BFA521A7210E24CDE900320294DD
S31508009590C2B20123064834F071F9012005B030BD86
S315080095A0A121F1E7002005B030BDA321ECE700BFFB
S315080095B0E8C0012030B540F2FE3384189C4287B0DB
S315080095C020DCFF280D461BD9B0F5007F1DD3B0F56A
S315080095D0407F34BFA521A72105AB0E240192009335
S315080095E0C2B2029401230A4834F048F99DF81420BF
S315080095F09DF81530012043EA02232B8007B030BDC1
S31508009600A121E9E7002007B030BDA321E4E700BFA8
S31508009610E8C0012030B5851840F2FE34A54285B071
S3150800962018DCFF280B4613D9B0F5007F15D3B0F523
S31508009630407F34BFA521A7210E24CDE9003202942C
S31508009640C2B20123064834F019F9012005B030BD2D
S31508009650A121F1E7002005B030BDA321ECE700BF4A
S31508009660E8C0012030B540F2FE3384189C4287B02A
S315080096701CDCFF280D4617D9B0F5007F19D3B0F5C5
S31508009680407F34BFA521A72105AB0E240192009384
S31508009690C2B202940123084834F0F0F8059B012071
S315080096A01BBA2B6007B030BDA121EDE7002007B03B
S315080096B030BDA321E8E700BFE8C001202DE9F0414D
S315080096C0044682B001464C2200F5FC7040F0BEFB11
S315080096D094F86D5294F8653294F86C1294F864E232
S315080096E094F8710294F8696294F8752294F868728D
S315080096F094F8748294F867C29FED657A2D0445EA5A
S3150800970001611B0494F8705243EA0E63000494F84E
S315080097106FE240EA056094F86E5281EA0E0141EA6A
S315080097200521360494F8775294F86AE261641204C3
S3150800973046EA076642EA086294F86B7294F87282FF
S3150800974083EA0C036A4094F866C2D4F85852019525
S315080097507E40D4F8505294F8737243EA0C2346EAD2
S315080097600E2605EB030C94F876E2019DE363784038
S31508009770D4F85472266442EA0E2237440D4440EA6D
S315080097800820C4E900C7C4E90250226194F88D2272
S3150800979094F88C0294F88F7294F878E294F87952D7
S315080097A084F83B70120442EA006245EA0E257A40C4
S315080097B094F87CE294F87D7294F87AC294F87B0265
S315080097C0258347EA0E27A783D4F87E72676240EAA4
S315080097D00C20D4F8827294F88EC294F890E294F829
S315080097E094526083C4F82E7094F89102D4F8867265
S315080097F0C4F83270D4F88A72C4F8367042EA0C2279
S3150800980040EA0E2094F8937294F892E26261803DE1
S3150800981084F83AC02562A08584F848E084F849703F
S3150800982094F89522803A07EE902AF8EEE77A67EEE2
S31508009830877AC4ED0A7A20B3B4F8242282420ED07D
S31508009840D4E97F52A4F8F401D4F8F801AE1B511AF2
S31508009850C31AC4F85462C4F85812C4F8503294F8BB
S31508009860773094F89720A3EB0E0EBA42BEFA8EFE16
S315080098704FEA5E1E0CBF0123002384F84AE084F8F1
S315080098804B30012384F85C3202B0BDE8F08100BF9A
S31508009890CDCCCC3DF0B504460D468FB000F25D2028
S315080098A004F25E213C2240F0DFFA94F85D3284F837
S315080098B09952492B01D00FB0F0BD94F85E32572B60
S315080098C0F9D194F85F32412BF5D194F86032502BD8
S315080098D0F1D194F86132492BEDD194F86232022B1A
S315080098E040F0AA8094F897323B2B40F0AC8094F86D
S315080098F09832212B40F0A7803B2D40F0A48004F23B
S31508009900622501AF04F2922C28686968AA68EB6898
S315080099103E460FC6103565453746F5D1286830608E
S31508009920DDE90132DDE9030103F07F35534002F03A
S315080099307F322A4403F080335340434002F07F329B
S3150800994000F07F30024403F0803353404B4002F06E
S315080099507F3201F07F315018DDE9052503F08033A9
S315080099604340534000F07F3002F07F32024403F058
S31508009970803353406B4002F07F3205F07F352A442E
S31508009980079903F080335340DDE908054B4002F0A0
S315080099907F3201F07F310A4403F08033534043405D
S315080099A002F07F3200F07F30024403F080335340E8
S315080099B06B4002F07F3205F07F352A440A9903F09E
S315080099C0803353404B4002F07F3201F07F318D18CF
S315080099D0DDE90B0203F080336B40434005F07F3529
S315080099E000F07F30284403F080334340534000F0B2
S315080099F07F3002F07F320D99024403F080335340E2
S31508009A004B4002F07F3201F07F310A4403F0803385
S31508009A105340C3F307221A44C3F307410A4402EB2F
S31508009A20136394F89622DBB29A420ED120460FB001
S31508009A30BDE8F040FFF742BE054906480FB0BDE84D
S31508009A40F040FFF717BB0449F7E70449F5E700BFFD
S31508009A50E0E50408301B002000E60408F0E50408E9
S31508009A6030B4C47B029D8583013414F0FF0408BF1B
S31508009A700124C473C0E9041230BC8361704700BF77
S31508009A8090F85C320BB91846704716490A7830B414
S31508009A900025012480F85C5280F818411AB1134653
S31508009AA0184630BC7047104A90F82E405578A542A3
S31508009AB018BF5470957890F82F40A54218BF947037
S31508009AC0D57890F8304090F83100A54218BFD47088
S31508009AD01479844218BF10710122184630BC0A70E6
S31508009AE0704700BFA50F0020A80F0020044B828DE9
S31508009AF0198891421ABF01201A800020704700BFBA
S31508009B00A60F002070B50446034694F84912D0F80B
S31508009B10450294F84422C4F8190184F81D1184F802
S31508009B201E21B4F8F45120686168A268A4F81F5190
S31508009B30C4F82921C4F82101C4F8251153F84C1F8B
S31508009B4094F864205868C4F83101C4F82D111B7ABA
S31508009B5084F83531234684F8362153F8551F5A6858
S31508009B609868C4F83F01C4F83711C4F83B219A89AC
S31508009B709B7B84F845312346A4F8432153F8681F94
S31508009B80A66F5A689868C4F84E01C4F84611C4F816
S31508009B904A219A899B7B84F85431A4F8522123469A
S31508009BA0E56FD4F88000B4F8841094F87720C4F8E8
S31508009BB05561C4F85951C4F85D01A4F8611184F8D7
S31508009BC0632153F8881FD4F89C505A689868C4F8DB
S31508009BD06C01C4F86411C4F868219A899B7BD4F88F
S31508009BE0A000A4F8702184F87231D4F89830C4F82B
S31508009BF07331B4F8A41094F89720C4F87751234623
S31508009C00C4F87B01A4F87F1184F8812153F8A81FB2
S31508009C105A689868C4F88A01C4F88211C4F886217B
S31508009C209A899B7B84F890312346A4F88E2153F8B1
S31508009C30B71F5A689868C4F89901C4F89111C4F80E
S31508009C4095219A899B7B84F89F312346A4F89D2108
S31508009C5053F8C60F9A685968C4F8A001C4F8A41145
S31508009C60C4F8A8219A899B7B84F8AE312346A4F8C8
S31508009C70AC2153F8D51F5A689868C4F8B701C4F8D8
S31508009C80AF11C4F8B3219A899B7B84F8BD3123466A
S31508009C90A4F8BB2153F8E41F5A689868C4F8C601AB
S31508009CA0C4F8BE11C4F8C2219A899B7B84F8CC31CA
S31508009CB02346A4F8CA2153F8F31F5A689868C4F8CB
S31508009CC0D501C4F8CD11C4F8D1219A899B7B84F8B3
S31508009CD0DB31B6B0D4F80801D4F80C11D4F8045125
S31508009CE0D4F81431A4F8D921D4F81021C4F8E00125
S31508009CF0C4F8E411C4F8E82104F58F71C4F8DC51FE
S31508009D00C4F8EC3101A8D22240F0A0F835AE01A87B
S31508009D10002150F8043B01F07F3503F07F324B40B9
S31508009D2003F080332A44B04282EA0301F1D19DF858
S31508009D30D4209DF8D530B4F84A02A4F8F1011344AA
S31508009D400B44C1F307221344C1F30742134494F8A2
S31508009D504C2284F8F32103EB116384F8F03136B012
S31508009D6070BD00BF012910D0022905D003291ED0D5
S31508009D70042913D000207047114B90F82F209978AA
S31508009D809142F7D09A70012070470D4B90F82E201B
S31508009D9058789042EED05A7008467047084B90F8AB
S31508009DA0312019799142E5D01A7101207047044B88
S31508009DB090F83020D9789142DCD0DA7001207047CB
S31508009DC0A80F00200020704700207047704700BF8A
S31508009DD0704700BF00207047704700BF00207047DB
S31508009DE02DE9F04104460D4600F062FCA36B217C88
S31508009DF0DBB9204600F0A4FC334F344E002D54D175
S31508009E00334BA16833481D8808F064FF3188A3687E
S31508009E103A782D1A05EBD57501EB650189B23180C3
S31508009E202C48BDE8F04108F0F1BE0139C9B2204618
S31508009E3000F086FC244F254E002D3DD1A268264908
S31508009E40264840F0BBFD224B244922481D8808F0CD
S31508009E5041FF3188214B3A780D442D1AA9B21D4885
S31508009E60318008F0D3FEA36A1B784FF00C08302522
S31508009E7018FB0353E358B3B1217C01312046C9B21C
S31508009E8000F05EFCA36A16491B78144818FB0355B4
S31508009E90625940F093FD3A783188104B0D48BDE879
S31508009EA0F04108F0B3BEBDE8F0813A7831880D4B31
S31508009EB0084808F0ABFEA3E73A783188094B05480D
S31508009EC008F0A4FEBAE700BFC40F0020C60F0020A2
S31508009ED0C80F002020C0012010E60408B00F00209B
S31508009EE0F44805080CE604081C3040F0D7BD00BF4E
S31508009EF070B50446084B44F8543B054600F1240661
S31508009F0020460C3CFFF778F9B442F9D1284600F010
S31508009F10ABFB284670BD00BF20E6040870B50546B1
S31508009F200A4B45F8543B044600F1240628460C3DE6
S31508009F30FFF762F9B542F9D1204600F095FB2046B5
S31508009F4060213EF0BDFD204670BD00BF20E6040836
S31508009F502DE9F04782B00225074600951E46DDE941
S31508009F600A9300F065FB3B46154A43F81C2B07F19C
S31508009F7030050022DFF84CA0FA612C465A601A8197
S31508009F8007F16008204651460C34FFF7F3F84445BC
S31508009F90F8D156B1314628460C35FFF735F945450F
S31508009FA006F10C06F6D10C9BBB62B9F1000F01D085
S31508009FB0C7F82C9001233846FB7102B0BDE8F0873C
S31508009FC020E604084041050810B5044600F01EFBCB
S31508009FD0E06A10BD704700BF10B50446D0F8D4003B
S31508009FE0084B236008B13EF069FD04F12C00FFF729
S31508009FF003F904F11C00FFF7FFF8204600F034FBD4
S3150800A000204610BDC8E604082DE9F04F044685B081
S3150800A0100D4600F04DFB217CDFF890815B4E204613
S3150800A02000F08EFB002D40F0A880A26858495948D8
S3150800A03040F0C4FC584B574958481D8808F04AFE5A
S3150800A0403188544B98F800200D442D1AA9B253486C
S3150800A050318008F0DBFD217C25790231C9B2204622
S3150800A060002D33D100F06CFB4D494C4808F032FE08
S3150800A070636932889B681044308023B3474FDFF802
S3150800A08030913846032108F089FF94F82830AB420E
S3150800A090384641D0D4F8D43098F800205B57318838
S3150800A0A004EB83030135DB6B039308F0AFFD039BD9
S3150800A0B03846194608F00EFE636932889B681044D4
S3150800A0C0AB423080DDD805B0BDE8F08F00F038FB34
S3150800A0D0E26A34492F4840F071FC98F800202D4B6D
S3150800A0E031882E4808F092FDE16A2C4808F0F2FD06
S3150800A0F06269348812682B4903462344254833800D
S3150800A10040F05CFC98F800203188224B234805B0C3
S3150800A110BDE8F04F08F07ABD94F9393098F8002078
S3150800A120B6F800B0039204EB83030135D3F83CA0DC
S3150800A130514608F0CFFD99F80010039A009103469E
S3150800A1405946384609F0F2F90021384608F026FF44
S3150800A15098F8002031885346384608F057FD51468E
S3150800A160384608F0B7FD636932889B681044AB42ED
S3150800A170308086D805B0BDE8F08F98F80020318881
S3150800A180094B064808F042FD4FE700BFC60F0020FE
S3150800A19010E60408B00F0020C80F002020C00120D8
S3150800A1A04C320508F44805080CE60408C40F0020DC
S3150800A1B0CA0F0020F8B50B780B3B0446202B34D881
S3150800A1C0DFE803F011433334333343333433333363
S3150800A1D03333333333333333333333333333333341
S3150800A1E033333333630090F82830D0F8D42090F90D
S3150800A1F03910D154406994F828308268013A93425C
S3150800A2004DD2013394F83820DBB284F8283062B195
S3150800A2100168C95C914208D1D4F8D4202521D154CB
S3150800A22094F82830013384F82830F8BD90F839308E
S3150800A23090F8E020013B5BB280F83930F2B9002B88
S3150800A240F3DA232384F83930F8BD90F8393090F8DA
S3150800A250E02001335BB280F839302AB9232BE4DDDC
S3150800A260002384F83930F8BD012A3FD0022ADCD110
S3150800A270232BDADD1A2384F83930F8BD012A2FD0CA
S3150800A280022AD2D1192BDCDDF8BD90F828301BB193
S3150800A290013B80F82830F8BD43790371F8BD237E69
S3150800A2A004F11C06ABB10025D4F8D4305B5704EB97
S3150800A2B08302252B294630460CBFD4F8D070D76BBD
S3150800A2C0FFF74CF83B780370237E0135AB42EBDC95
S3150800A2D060693146FEF798FF40F20113A380F8BD86
S3150800A2E0002BA2DA192380F83930F8BD192BB7DC10
S3150800A2F0F8BD00BF10B50446D0F8D4000A4B236059
S3150800A30008B13EF0DBFB04F12C00FEF775FF04F103
S3150800A3101C00FEF771FF204600F0A6F92046E4214E
S3150800A3203EF0CEFB204610BDC8E604082DE9F84FDE
S3150800A330D0E900960546A6EB09036FF00040834274
S3150800A34051D08A469346002B48D0B3EB430F4FEAC9
S3150800A350430831D98046AAEB090440463EF0B2FBD1
S3150800A360074680449BF800303B55002C0FDCA6EBD3
S3150800A3700A060134002E3C4426DC3444B9F1000FA9
S3150800A38011D1C5E90074C5F80880BDE8F88F2246E2
S3150800A39049463846A6EB0A063FF066FD0134002E0C
S3150800A3A03C4411DC344448463EF088FBC5E9007459
S3150800A3B0C5F80880BDE8F88FB8F1000FCADBA1EB35
S3150800A3C00904CAD14746CDE72046514632463FF0F2
S3150800A3D03DFD3444B9F1000FD3D0E4E7A1EB0904FD
S3150800A3E04FF00108B9E701483EF082FBA4E60408ED
S3150800A3F02DE9F04F85B0022580461E4600950E9B36
S3150800A4009DF83C709DF84090044600F011F9324BD7
S3150800A41048F81C3B314904F12C0A4046FEF7AAFECF
S3150800A4202E495046FEF7A6FE002598222C4904F12F
S3150800A4303C003FF00BFD11996661C4E9355550465D
S3150800A440C4F8DC5084F82850FEF7DEFE61698B6894
S3150800A4500422E2716BB304F1D40B24264FF0250ACB
S3150800A4600EE099428DF80F602FD00E70D4F8D830D0
S3150800A4700133C4F8D83061698B680135AB4217D906
S3150800A4800B68D4F8D8105B5DBB42D4F8DC30E8D151
S3150800A49099428DF80FA018D081F800A0D4F8D830CA
S3150800A4A061690133C4F8D8308B680135AB42E7D807
S3150800A4B0DBB223764046FEF7A7FE204684F8E090F6
S3150800A4C084F8387005B0BDE8F08F0DF10F025846D4
S3150800A4D0FFF72CFFCFE700BFC8E604084041050890
S3150800A4E0F0E304082DE9F04F87B01E469DF840506A
S3150800A4F0119B0095814604469DF848809DF84CA01E
S3150800A50000F096F8314B49F81C3B31494846FEF7AE
S3150800A51031FE2F4904F12C00FEF72CFE2D49982216
S3150800A52004F13C003FF092FCB26866610023042106
S3150800A530C4E93533E171C4F8DC3084F82830002AE0
S3150800A54041D004F1D40019461D4624274FF0250BA7
S3150800A55010E099428DF817702ED00F70D4F8D830C5
S3150800A5600133C4F8D8306669B3680135AB4215D9EA
S3150800A570D4E936133268525D4245EAD199428DF8DC
S3150800A58017B019D081F800B0D4F8D830666901330D
S3150800A590C4F8D830B3680135AB42E9D8DBB22376C4
S3150800A5A031464846FEF730FE204684F8E0A084F897
S3150800A5B0388007B0BDE8F08F0DF117020390FFF75A
S3150800A5C0B5FE0398CFE71346E9E700BFC8E60408D7
S3150800A5D040410508F0E3040810B5044600F016F8F3
S3150800A5E094F8E030012B0AD9022B08BF1A234FF042
S3150800A5F0000008BF84F8393084F8280010BD00230D
S3150800A600002084F8393084F8280010BD08B583790D
S3150800A610012B0AD00379032B07D08B4218BF43714D
S3150800A620C36801710BB108469847002008BD00BFF2
S3150800A63030B44D1E0E2D82600A4DC3604FF00202E3
S3150800A6404FF4A06388BF00210560427108250022E7
S3150800A650C3809DF808304574827430BC0174037158
S3150800A660704700BF00E7040810B504468068044B2D
S3150800A670236010B101213EF023FA204610BD00BF29
S3150800A68000E70408037901718B4218BF43717047CC
S3150800A69043790371704700BF007970478079704726
S3150800A6A000238371704700BF81717047C079704776
S3150800A6B038B5437C082B044628D0062B2BD0184DDA
S3150800A6C0284608F0C7FA284608F0FEFA95F8292021
S3150800A6D095F82A001349A37C121A0A70A3B92B8885
S3150800A6E0A2791149012A0B8002D02379032B05D1BF
S3150800A6F0BDE838400A48012108F050BCBDE838409A
S3150800A7000748032108F04ABC9BB2E9E70749044811
S3150800A71008F0F6FAD3E70649014808F0F1FACEE759
S3150800A72020C00120CA0F0020CC0F002060F60408C4
S3150800A73014EF040881747047806870478160704719
S3150800A740013930B40B2914D8DFE801F0222F3B0673
S3150800A750475461707E8C95154D4A4E4B12781B886E
S3150800A7604D4D4E4C4E4952005B0800202A702380FE
S3150800A770088030BC7047464A464B12781B88464CC0
S3150800A780464847495B089200227003800B80F0E731
S3150800A790404B3F4C40491B884048414A24780C703E
S3150800A7A05B08002103801180E3E7394C3A4A3948AF
S3150800A7B03A493B4B247800881470002208801A8096
S3150800A7C0D7E7344B324C1B883449354A324824780B
S3150800A7D004705B080B801380CBE72D4B2D4C2F495B
S3150800A7E01B782D482E4A24880C805B0000210370B4
S3150800A7F01180BEE7264A274B12781B88264C274825
S3150800A80027495B085200227003800B80B1E7204B72
S3150800A810204A1B781288204D204C214903EB43031C
S3150800A820520800202B7022800880A2E7184B194C8A
S3150800A8301A491B7818481A4A24880C8003EB4303E4
S3150800A84000210370118094E7114A124B12781B8875
S3150800A850114C124812495B0802EB4202227003802F
S3150800A8600B8086E70A4A0B4B12781B880A4D0B4C5D
S3150800A8700B49920078E7064B064C08491B780648B0
S3150800A880074A24880C809B0000210370118070E71A
S3150800A890CA0F0020CC0F0020C40F0020C80F0020CC
S3150800A8A0C60F0020436A13B190F821201A700020C1
S3150800A8B0704700BF41610276704700BF90F92120BA
S3150800A8C0436953F82200704790F82800704700BF84
S3150800A8D02DE9F04F044681B00D46FFF7E9FE94F8DE
S3150800A8E02830012B48D023B1022B02D001B0BDE895
S3150800A8F0F08F217CDFF88481564F2046FFF720FF32
S3150800A900002D40F08D80217C23790231C9B2204682
S3150800A910002B58D0FFF714FF237E002B69D0626AFC
S3150800A9206369127853F822204B494C4840F046F8A0
S3150800A9304A4B98F800203988494808F067F9A26810
S3150800A9404849464840F03AF8217C2046FFF7F8FE89
S3150800A950454B424942481C8808F0BCF9398898F8A2
S3150800A96000203E4B0C44241A3D48A1B2398001B060
S3150800A970BDE8F04F08F04AB9217CDFF80081354F71
S3150800A9802046FFF7DDFE35BB257965BBDFF8F0A06D
S3150800A990DFF8CC902E46013505EB4501C9B22046B5
S3150800A9A0FFF7CEFE94F92130002B1A46B8BFDA1C01
S3150800A9B0921006EB8206B3423AD0237EB34225DCD8
S3150800A9C0042DE7D1BBE7FFF7BBFE237E8BB194F9D5
S3150800A9D021206369A6E798F800203988234B204888
S3150800A9E008F014F9D0E7A26821491C483FF0E6FFB1
S3150800A9F0AAE7204D194B07CD186059609A60398827
S3150800AA0098F80020164808F001F998E7636998F85D
S3150800AA10002053F826303988484608F0F7F8CFE77B
S3150800AA2098F800203988114B0D4808F0EFF86AE7C6
S3150800AA30114B51464846B3F800B008F04BF9ABEB5A
S3150800AA40000081B298F800205346484608F0DEF820
S3150800AA50B3E700BFC60F0020F4480508B00F002072
S3150800AA6020C0012034E70408C80F00200CE60408BB
S3150800AA7038E704083CE70408CC0F0020C40F002080
S3150800AA8030E70408426938B5164B03600446AAB194
S3150800AA90037E9BB1002552F82500012158B13EF0EE
S3150800AAA00FF8237E0135AB4208DD626952F82500AE
S3150800AAB001210028F3D10135AB42ECDC606A10B104
S3150800AAC001213DF0FDFFE06910B101213DF0F8FFDD
S3150800AAD0A06810B101213DF0F3FF2046FFF7C4FD41
S3150800AAE0204638BD50E7040810B50446FFF7CAFFEC
S3150800AAF020462C213DF0E4FF204610BD38B54369B9
S3150800AB00B3B1027E05469AB1002453F82400012108
S3150800AB1058B13DF0D5FF2A7E0134A24208DD6B69A3
S3150800AB2053F8240001210028F3D10134A242ECDCB9
S3150800AB3038BD00BFF8B50B780E2B04463AD034D88A
S3150800AB400B2B65D00C2B2FD190F8213090F8205084
S3150800AB500021013B5BB28D4280F821308C4609DC2E
S3150800AB60BCF1000F1ED0EDB100218C4602E0013188
S3150800AB708D42F5DDE7697A181344D8B2831A12F8BC
S3150800AB80016B5BB2B342F2D1831A01315BB28D42DB
S3150800AB9084F821304FF0010CF0DC4FF0000C6146D0
S3150800ABA0002DE8D1002B41DBF8BD2B2BFCD14379D6
S3150800ABB00371F8BD90F8213090F8200001335BB29C
S3150800ABC0002184F821300F4600E00131884216DD65
S3150800ABD0E2690A449B1ADDB2AB1812F8016B5BB244
S3150800ABE0B342F2D1AB1801315BB2884284F8213006
S3150800ABF04FF00107F0DC20B100210F46E8E7002FEF
S3150800AC00F9D1227E9A42CFDC002384F82130F8BDA0
S3150800AC1003680A4ADB6893420DD1436A13B190F878
S3150800AC2021201A7040F20113A380F8BD237E013B50
S3150800AC3084F82130F8BD9847F4E700BFA5A80008B6
S3150800AC402DE9F04182B00226044600961D460B9B6C
S3150800AC509DF828809DF82070099EFFF7E9FC0023DF
S3150800AC60084984F8288003222160E2712376E3618B
S3150800AC7023840DB1656127762046666202B0BDE879
S3150800AC80F08100BF50E704082DE9F04182B0044680
S3150800AC9000930A9D9DF830709DF82C80DDE90836F2
S3150800ACA0FFF7C6FC0023094984F8287003222160AF
S3150800ACB0E2712376E361238415B1656184F818800F
S3150800ACC02046666202B0BDE8F08100BF50E704087E
S3150800ACD010B50446FFF79AFC94F82830022B01D0E9
S3150800ACE0002010BD94F82130217E01335AB29142DA
S3150800ACF084F82120DBB222680949DCBF002384F8E6
S3150800AD002130D2688A4207D1626A02B1137040F2D2
S3150800AD100113A380002010BD20469047F7E700BF27
S3150800AD20A5A80008704700BF90F82600704700BF26
S3150800AD3010B5034B03600446FFF796FC204610BD8A
S3150800AD4090E7040810B5054B03600446FFF78CFC32
S3150800AD5020462C213DF0B4FE204610BD90E704089D
S3150800AD602DE9F04104460D46FFF7A2FC217C224F4F
S3150800AD70224E0139C9B22046FFF7E2FC3DBBA26864
S3150800AD801F4920483FF01AFE1F4B1E491F481D88C1
S3150800AD9007F0A0FF31881B4B3A780D442D1AA9B24B
S3150800ADA01A48318007F032FF2379022B16D0012B7F
S3150800ADB01AD0217C01312046C9B2FFF7C1FC3A7886
S3150800ADC03188104B1148BDE8F04107F01FBF3A78AB
S3150800ADD031880F4B0D4807F019FFD0E762690D4916
S3150800ADE008483FF0EBFDE4E7A3690B49054804F181
S3150800ADF01C023FF0E3FDDCE7C40F0020C60F00206D
S3150800AE0010E60408B00F0020C80F002020C001205B
S3150800AE100CE60408F448050880E704081C303FF0EF
S3150800AE203DBE00BF70B582B00226044600961D4698
S3150800AE30DDE90663FFF7FCFB22460A4B42F81C3B9A
S3150800AE400023E3615360138184F826301DB1D5E9E8
S3150800AE500032C4E9053202232046A662E37102B035
S3150800AE6070BD00BF90E704084161704710B50446FD
S3150800AE70FFF7CCFBA06A10BD2DE9F047054604464E
S3150800AE804FF4006025F8040BDFF83C809DF820900D
S3150800AE900F462846414692461E46FEF76BF941463E
S3150800AEA004F11000FEF766F900232846514663842C
S3150800AEB084F82430FEF7F0F9277784F81D90A677F2
S3150800AEC02046BDE8F08700BF4041050810B5044696
S3150800AED01030FEF791F9201DFEF78EF9204610BDB9
S3150800AEE0807F70471030FEF78FB900BF0430FEF739
S3150800AEF08BB900BF0170704700787047407F704774
S3150800AF0041707047037F0C2B15D8DFE803F0152135
S3150800AF102B34414C5664707B8A8F0700C38C90F89B
S3150800AF2025205B08002163F30F0163F31F4193009B
S3150800AF30016280F824307047C38C00215B080A46FA
S3150800AF4063F30F0263F31F4280F82410026270470E
S3150800AF50C38C90F8252080F824205B0800220384FF
S3150800AF604284704790F82530C28C80F8243000233C
S3150800AF70028443847047C38C90F8252080F82420E7
S3150800AF805B08002263F30F0263F31F4202627047F5
S3150800AF9090F82520C38C52005B08002180F82420F5
S3150800AFA003844184704790F82530C28C02845B0084
S3150800AFB0002280F8243042847047C38C90F82520FC
S3150800AFC05B08002163F30F0163F31F41530001621D
S3150800AFD080F82430704790F82530C28C03EB430381
S3150800AFE05208002180F8243002844184704790F882
S3150800AFF02530C28C028403EB4303002280F82430F8
S3150800B00042847047C28C90F825305208002162F3BA
S3150800B0100F0162F31F4103EB4303016280F82430FA
S3150800B020704790F82520C38C9200B5E790F8253034
S3150800B030C28C02849B00002280F824304284704728
S3150800B0400378012B00D1704730B54378082B8FB0B1
S3150800B05004463FD0062B42D0234D284607F0FAFD7A
S3150800B060284607F031FE95F82A2095F829302988D0
S3150800B070E1849B1A84F825300321284607F08EFFC1
S3150800B0802046FFF73FFF23696268184901A83FF089
S3150800B09095FC237F28469BB101A9258C07F01AFE4B
S3150800B0A0618C281A00EBD07001EB600189B26184CB
S3150800B0B094F824200C4801AB07F0A8FD0FB030BD6A
S3150800B0C001A9258C07F006FE618C0D442D1AA9B23C
S3150800B0D06184EDE70649044807F012FEBCE7054916
S3150800B0E0014807F00DFEB7E720C00120544A0508BD
S3150800B0F060F6040814EF0408704700BF80697047BB
S3150800B1000020704710B5034B03600446FFF7ACFAFE
S3150800B110204610BDC8E7040810B5054B0360044671
S3150800B120FFF7A2FA20461C213DF0CAFC204610BDB6
S3150800B130C8E704082DE9F04106460C46FFF7B8FAB9
S3150800B140317CDFF85880114F3046FFF7F9FAACB971
S3150800B1500F4BB1680F481C8807F0BCFD3988B368E7
S3150800B16098F80020241A04EBD47401EB640189B220
S3150800B17039800848BDE8F04107F048BD98F8002036
S3150800B1803988054B034807F041FDE1E7C60F002063
S3150800B190C80F002020C001200CE60408C40F0020B8
S3150800B1A070B582B002261D460096069B0446FFF738
S3150800B1B03FFA044A6561002320462260A361E371D1
S3150800B1C002B070BDC8E7040810B50446FFF71EFABA
S3150800B1D0606910BD70B49DF80C509DF8204041611F
S3150800B1E09DF814108361017201239DF81C100374E5
S3150800B1F04174B5FBF4F304FB13514262DBB2069AC1
S3150800B200049EC26011F0FF0F4FF0000218BF013311
S3150800B2104660057780F82040C0E90D2270BC0270B0
S3150800B220C277C26383777047704700BF4161704732
S3150800B2300378042B70B5044660D0052B04D0032B85
S3150800B2400BD00023237470BDC16A0B78052BC36825
S3150800B25000F0BC800BB198472070A26901232374C3
S3150800B260002A61D0616A0B780B3B212BE9D801A033
S3150800B27050F823F0EFB400080BB4000841B40008F6
S3150800B280B7B4000875B4000843B2000843B2000812
S3150800B29043B2000843B2000843B2000843B20008AC
S3150800B2A043B2000843B2000843B2000843B200089C
S3150800B2B043B2000843B2000843B2000843B200088C
S3150800B2C043B2000843B2000843B2000843B200087C
S3150800B2D043B2000843B2000843B2000843B200086C
S3150800B2E043B2000843B2000843B2000843B200085C
S3150800B2F043B2000879B5000823B30008836990F9BA
S3150800B3001D20416A53F8220003685B699847636AFF
S3150800B3101B782B2B00F047810B2B1FD0012323749E
S3150800B32070BDE36A5BB170BD636A1B780B2B00F0D6
S3150800B33081812B2B85D1E36A002B40F0BC81D4E9AF
S3150800B3400D12E06B00F08AFCE36800222270002BE5
S3150800B3503FF479AF20469847207070BD94F91D20B8
S3150800B360A36953F82200FFF797F90028D6D0E368B7
S3150800B370002B00F0B481A36994F91D2053F822002C
S3150800B380036801219B689847E36813B120469847EC
S3150800B390207094F91D20A36953F82200FFF786F957
S3150800B3A0032820D02378032BB8D0052B7FF455AF7C
S3150800B3B0A56AE06B00232B7000F0AEFCE36BEB6331
S3150800B3C0E862A16AE06B00F071FC46E702220270AF
S3150800B3D013B19847E16A2070E06B00F067FCE06BF8
S3150800B3E000F074FC9AE794F82050E27F237F15FB5F
S3150800B3F002F59D42D6DAA36953F82500FFF750F9FE
S3150800B400237F0135AB42F6DCCCE794F91D00431ED9
S3150800B4105BB2002B6377C0F2408194F820100133A9
S3150800B420B3FBF1F201FB1233002B7FF40CAFE37F81
S3150800B430002B3FF408AF042900F0B280607770BD96
S3150800B44094F82020042A40F2ED8094F91D1004296E
S3150800B45000F02E81E37F002B00F01181891A49B292
S3150800B460013BDBB20029E377B6BF12FB03F3617732
S3150800B470637770BD94F82000042840F2BA8094F9E6
S3150800B4801D30022B40F32581227F01335BB29A429D
S3150800B490637740F3A78093FBF0F200FB1233002B8F
S3150800B4A07FF4D1AEA37FE27F013B9A42BFF6CBAED3
S3150800B4B00132E27770BD94F91D00227F431C5BB20E
S3150800B4C09A42637740F38E8094F8201093FBF1F24A
S3150800B4D001FB1233002B7FF4B6AEA37FE27F013B5C
S3150800B4E09A42BFF6B0AE0429E2D06077A7E7237880
S3150800B4F0022B00F0AB8094F91D3052F82300FFF7B9
S3150800B500CDF894F91D20A369054653F82200FFF7E4
S3150800B510C3F8012D3FF497AE03283FF494AE94F98F
S3150800B5201D20A36953F82200FFF7C0F8A36994F910
S3150800B5301D20064653F82200036800219B68984799
S3150800B5400546002800F00A81E36A1B78052B00D01F
S3150800B55000232370002E40F0F2800023E06BA562E2
S3150800B5602B7000F0D9FBE36BEB63E862A16AE06B32
S3150800B570BDE8704000F09ABBE36A002B3FF4DFAEEB
S3150800B580206BFFF785F800232370E16A0B78052BFB
S3150800B59001D100230B70E06BBDE8704000F086BB5C
S3150800B5A0013BE37770BD94F91D20A36953F8220087
S3150800B5B0FFF772F800283FF4B1AEE3680BB12046F6
S3150800B5C09847237F03222270002B3FF4A7AE00255D
S3150800B5D0A36953F82500FFF763F8237F0135AB42CB
S3150800B5E0F6DC9BE6637C013AD3B1012362770B70E4
S3150800B5F070BDA37FE27F013B9A42BFF624AE0428C2
S3150800B6003FF421AE94F91D30217F03445BB2013229
S3150800B610D2B29942E27763773FF715AE10FB02F292
S3150800B620627770BDE37F53B3042A3FF40CAE94F9F6
S3150800B6301D1013E7E3680422227013B120469847C9
S3150800B6402070A56A002D60D102232370E3680BB130
S3150800B6502046984700230121206B2370FFF712F834
S3150800B660E16A31B10B78052B95D1A36A002B00F05E
S3150800B6709180E06B0021BDE8704000F017BBE56AD9
S3150800B680002D51D0206BFFF703F8E16A00232370E1
S3150800B6900A78052A08BF0B707DE7637C4BB1002347
S3150800B6A06377D4E90D12E06BBDE8704000F0D6BAB6
S3150800B6B00323637770BDE368227013B12046984769
S3150800B6C02070206BFEF7E4FFE16AE06B00F0EEFA0B
S3150800B6D05BE7A17FE27F01398A4295DB70BDE27F95
S3150800B6E094F82050237F15FB02F59D424FF0030284
S3150800B6F02270BFF613AEA36953F82500FEF7C8FFFC
S3150800B700237F0135AB42F6DC08E600232B70E06B9D
S3150800B71000F002FBE36BEB63E862A16AE06B00F002
S3150800B720C5FA0123237470BDD4E90D12E06B00F04D
S3150800B73095FAE3682570002B7FF40CAE70BD012ED8
S3150800B74018D0022E16D0032E2CD0042E7FF47BADF3
S3150800B7502378032B7FF477AD267070BDAEB9E16A06
S3150800B760E06B0B78052B18BF33462370BDE8704095
S3150800B77000F09CBA0023A5622B7094F91D20A369DA
S3150800B780E06B53F822302B63EBE6012E3CD0022EF9
S3150800B790D9D170BDE06B00F089FAE06BBDE8704066
S3150800B7A000F094BA2378032B7FF44DADA36994F97E
S3150800B7B01D2053F822000368DB6A984702283FF4E5
S3150800B7C042ADE36813B1204698472070237894F871
S3150800B7D02050E27F042B1CBF04232370237F15FB14
S3150800B7E002F59D42BFF62FAD94F91D30AB424FF0DE
S3150800B7F00101A3690DD053F82500FEF755FF237FF5
S3150800B8000135AB42F0DC70BDE368002B7FF4A2ADD6
S3150800B81070BD53F825000021FEF734FF237F01355C
S3150800B8209D42E1DB70BD00BF41637047816370478D
S3150800B830C1637047F0B58E4E8E498BB007463046C9
S3150800B84007F05EFA304607F03FFA3046032107F064
S3150800B850A5FB97F82030042B40F0D380FA7F002A06
S3150800B86040F0F280BB7F013B9A4240F0BD8082499E
S3150800B8707F4807F045FA7E4807F0ECF97C4807F060
S3150800B88023FA7B48032107F089FB796901A8FDF7AC
S3150800B89071FC7A4904A8FDF76DFC794901A8FDF702
S3150800B8A047FD0246002800F0A6800823002207A8C4
S3150800B8B001A9FDF773FD07A904A8FDF7CBFC07A8A6
S3150800B8C0FDF79AFC00221146049B694807F09EF989
S3150800B8D00499674807F0FEF90C230822064601A9D1
S3150800B8E007A8FDF75BFD07A904A8FDF7B3FC07A8A1
S3150800B8F0FDF782FCFB7FF6B2002B70D05C48012175
S3150800B90007F04CFB049B5A480022314607F07EF9A3
S3150800B9100499574807F0DEF903213518544807F00B
S3150800B9203DFBFB7FEDB2002B40F08B800F230D22F1
S3150800B93001A907A8FDF732FD07A904A8FDF78AFCA7
S3150800B94007A8FDF759FC049B49480022294607F039
S3150800B9505DF90499464807F0BDF90F2213232C1800
S3150800B96001A907A8FDF71AFD07A904A8FDF772FCA7
S3150800B97007A8FDF741FCFB7F3D48012B0CBF0321BF
S3150800B9800121E4B207F00AFB049B3948002221464C
S3150800B99007F03CF90499364807F09CF9032104445A
S3150800B9A0334807F0FBFA039B132201A907A8FDF702
S3150800B9B0F5FC07A904A8FDF74DFCE4B207A8FDF7B6
S3150800B9C01BFC049B2A482146002207F01FF904A8FD
S3150800B9D0FDF712FC01A8FDF70FFC0BB0F0BD2448DB
S3150800B9E0032107F0DBFA8DE7264B21480522F921CA
S3150800B9F007F00CF93BE77B691D48114607F006F985
S3150800BA00E5E721493578304607F064F9BB7FFA7FC8
S3150800BA10013B281A9A42C4B205D01B4B3046032272
S3150800BA20214607F0F3F81949114807F053F9211A86
S3150800BA30C9B20139154B0E4889B2032207F0E6F858
S3150800BA4015E70E230C2273E71149304607F042F931
S3150800BA50C0F1F9000E4B81B20522304607F0D6F840
S3150800BA60BB7FFA7F013B9A423FF401AFBCE700BFB8
S3150800BA7020C00120C8FE040860F6040840410508F5
S3150800BA8000E80408F8E70408A0540508FCE70408D9
S3150800BA90343205080378052B70B5044632D1524A6C
S3150800BAA013780133DBB2072B2AD9C3680025012195
S3150800BAB0157001741BB39847E368207005461BB1DF
S3150800BAC02046984705462070002D7FD0042D16D1B4
S3150800BAD094F82050E27F237F15FB02F59D420EDA8B
S3150800BAE094F91D30AB424FF00101A36964D053F8B5
S3150800BAF02500FEF7D9FD237F0135AB42F0DC70BD8A
S3150800BB00137070BDFFF796FE94F82030E57F267F08
S3150800BB1015FB03F52B449E42A8BF1E46B5420FDA15
S3150800BB2094F91D30AB42A36953F8250003684FF01A
S3150800BB3000011B6905F1010539D09847AE42EFD1DE
S3150800BB40237A002523B91DE0237A0135AB4219DD96
S3150800BB50636853F82500FFF7C3F9237883424FEA51
S3150800BB608506F1D1636853F82500FFF7C7F9E37F27
S3150800BB708342E9D163689859FFF762FA237A013557
S3150800BB80AB42E5DC2278002AB9D117490B78013394
S3150800BB90DBB2072B0B70B2D9E56801232370237437
S3150800BBA00A70002DABD02046A847207070BD012131
S3150800BBB09847B542B4D1C3E753F825000021FEF7EC
S3150800BBC061FD237F01359D428ADB70BD0121206B13
S3150800BBD0FEF758FDE16A21B1E06BBDE8704000F060
S3150800BBE065B82946F8E700BFCE0F002000787047F1
S3150800BBF000230374704700BF01230374704700BF16
S3150800BC00007C704710B490F82040B2FBF4F304FBB4
S3150800BC10132414F0FF0FDBB218BF01335DF8044B91
S3150800BC20027781618377704790F91D20836953F8FD
S3150800BC3022007047006B704781627047806A00383F
S3150800BC4018BF0120704700BF002201230270037449
S3150800BC50704700BF4160704781607047F0B505685E
S3150800BC60104F2E684FF0000C0123BE4283B00446E5
S3150800BC70C0F80CC0037407D16B6861600A498B422F
S3150800BC800AD1A26003B0F0BD0192B0472568064903
S3150800BC906B68019A8B42F4D01146204603B0BDE882
S3150800BCA0F040184755BC000859BC000809B1C160E6
S3150800BCB0704701230374C160704700BFC36813B19E
S3150800BCC01846FFF7E7BE4368184700BFC36813B1B5
S3150800BCD01846FFF7ADBA8368184700BF10B5044683
S3150800BCE0C06818B1FFF78CFF207410BD207C10BD0A
S3150800BCF010B50446C06808B1FFF77AFF002323741D
S3150800BD0010BD00BF10B50446C06808B1FFF774FF40
S3150800BD100123237410BD00BFC0687047436810B57F
S3150800BD20044603B1984723682046DB69BDE81040FE
S3150800BD30184700BF704700BF10B4012480F8C940F7
S3150800BD4080F8C4105DF8044B80F8C52080F8C6302A
S3150800BD50704700BF02EBC20202EB8101084490F86B
S3150800BD60A43090F8A30003F00F0340EA03207047BD
S3150800BD7002EBC20202EB8101084490F8A53090F864
S3150800BD80A4001B0143EA1010704700BF02EBC20271
S3150800BD9002EB8101084490F8A20000F07F0070478A
S3150800BDA002EBC20202EB8101084490F8A20080F07F
S3150800BDB08000C009704700BF90F89D0000F00F0092
S3150800BDC0704700BF00220123A0F8C22080F8C930BE
S3150800BDD0704700BF20290CBF4FF47F42FF22012382
S3150800BDE0A0F8C22080F8C930704700BF012380F848
S3150800BDF0C21080F8C32080F8C9307047012380F844
S3150800BE00C71080F8C82080F8C9307047407E704750
S3150800BE10C3683BB1002001210622187283F8481036
S3150800BE2083F88120704700BF783003F0E7B900BF78
S3150800BE30043002F047BB00BFF0B54F2397B00C465D
S3150800BE4005461A4602A800213EF028F80022E271AB
S3150800BE50EA7DA97D0091019267782078A178E67835
S3150800BE6094F804E094F805C08DF80F708DF810006A
S3150800BE70A779A8688DF811108DF81260A9898DF830
S3150800BE8013E04F2302AA41F252168025FF248DF8AB
S3150800BE9014C08DF81570ADF808608DF80A508DF845
S3150800BEA00C4002F02BF817B0F0BD00BFF0B54F23D9
S3150800BEB097B00C4605461A4602A800213DF0EEFF4B
S3150800BEC00022E27115F8612C15F8621C00910192A6
S3150800BED067782078A178E67894F804E094F805C0A5
S3150800BEE08DF80F708DF81000A77955F8700C8DF83D
S3150800BEF011108DF8126035F86C1C8DF813E04F237D
S3150800BF0002AA41F252168025FF248DF814C08DF836
S3150800BF101570ADF808608DF80A508DF80C4001F0E0
S3150800BF20EDFF17B0F0BD00BF30B5044685B07830D8
S3150800BF3003F064F9E27DA37DCDE9003240F24325A2
S3150800BF400223A189A068ADF80C5003AA01F0D6FF18
S3150800BF5063680BB105B030BDFF210122A4F8C030DB
S3150800BF6084F8C21084F8C52005B030BD783003F0D7
S3150800BF70D5B800BF7C3003F0CDB800BF7C3003F0E5
S3150800BF8095B800BF7C3002F0F7BE00BF7C3002F0E7
S3150800BF90B3BF00BF08B5B0F99430012900EE903A56
S3150800BFA00CBFB0F99630B0F9923000EE103AF8EEC0
S3150800BFB0E00AB8EEC00A3CF07DFE9FED047ADFED9C
S3150800BFC0047A30EE070A20EE270A08BDDB0F49403F
S3150800BFD0E12E654210B50D4B82B00446002240F8AA
S3150800BFE0043B0B4B02F0B4FA0A4BE36704F17C00FE
S3150800BFF0019003F003F9084B636030330198E36757
S3150800C00003F0FCF8204602B010BD00BF80E8040823
S3150800C01028E8040838E8040844E8040810B40124A9
S3150800C02080F8C64080F8C3105DF8044B80F8C42039
S3150800C03080F8C530704700BF00EB8101D1F8B00029
S3150800C040C0F30B20704700BF00EB8101B1F8B200C6
S3150800C050C0F30B10704700BF00EB810191F8B000E8
S3150800C06000F07F00704700BF00EB810191F8B00037
S3150800C07080F08000C00970470F2070470022012316
S3150800C080A0F8BE2080F8C630704700BF20290CBF34
S3150800C0904FF47F42FF220123A0F8BE2080F8C63065
S3150800C0A0704700BF012380F8BE1080F8BF2080F8D3
S3150800C0B0C6307047704700BF407E7047C3683BB1C3
S3150800C0C0002001210622187283F8481083F881207F
S3150800C0D0704700BF783003F03BBB00BF043002F066
S3150800C0E0F1B900BFF0B5064697B00F4647220021C2
S3150800C0F004A83DF0D3FE96F8C6305A1CD2B20F2AD1
S3150800C1004FEA03138DF80A3043F2A2110ABF00233F
S3150800C11086F8C62086F8C630ADF8081010213A7899
S3150800C120BB787C788DF80B1006F184000DF11601AA
S3150800C1304FF2FF758DF80F208DF814308DF80E40EC
S3150800C140ADF80C5003F02AFB0DF1210106F17C0035
S3150800C15003F024FBFB787A68CDF83720002B14BF50
S3150800C16001220222032317498DF835208DF8323033
S3150800C17002AC4FF0FF320DF1530014F8013BD5B273
S3150800C1806B40844251F8233083EA1222F5D100230A
S3150800C1903B72317ED343727E01920091190A1D0CBF
S3150800C1A01C0E8DF853308DF85410B068B1898DF88F
S3150800C1B0555002AA4F238DF8564001F09FFE17B03E
S3150800C1C0F0BD00BF10E90408F0B5064697B00F4663
S3150800C1D04722002104A83DF061FE96F84E305A1C0D
S3150800C1E0D2B20F2A4FEA03138DF80A3043F2A2118E
S3150800C1F00ABF002386F84E2086F84E30ADF80810A0
S3150800C20010213A78BB787C788DF80B1006F10C0073
S3150800C2100DF116014FF2FF758DF80F208DF81430C9
S3150800C2208DF80E40ADF80C5003F0B8FA0DF1210167
S3150800C230301D03F0B3FAFB787A68CDF83720002B67
S3150800C24014BF01220222032318498DF835208DF8E0
S3150800C250323002AC4FF0FF320DF1530014F8013BB7
S3150800C260D5B26B40844251F8233083EA1222F5D1C5
S3150800C27000233B7216F8601CD34316F85F2C019214
S3150800C2800091190A1D0C1C0E8DF853308DF85410A8
S3150800C29056F8700C36F86C1C8DF8555002AA4F23C8
S3150800C2A08DF8564001F02AFE17B0F0BD10E90408D3
S3150800C2B030B5044685B0783003F04AFAE27DA37DAE
S3150800C2C0CDE9003240F643150223A189A068ADF8EE
S3150800C2D00C5003AA01F012FE63680BB105B030BD1D
S3150800C2E0FF210122A4F8C03084F8BF1084F8C220C8
S3150800C2F005B030BD783003F0AFB900BF7C3003F02D
S3150800C300A7B900BF7C3003F06FB900BF7C3002F0DC
S3150800C310B1BF00BF7C3003F07BB800BF012908B568
S3150800C32017D0B0F9A730B0F9A5205B4200EE102A65
S3150800C33000EE903AF8EEE00AB8EEC00A3CF0BAFC15
S3150800C3409FED097ADFED097A30EE070A20EE270A13
S3150800C35008BDB0F9A720B0F9A93052425B4200EEF9
S3150800C360902A00EE103AE5E7DB0F4940E12E6542D8
S3150800C37030B5144B044683B0002240F8043B124BF8
S3150800C38002F0E6F800251149E16704F17C00C4E9EA
S3150800C3902055C4E9225584F8875084F88F50A4F8AC
S3150800C3A0C850019003F0D4F9094B019884F8CA5093
S3150800C3B003F130026360E26703F0CAF9204603B06E
S3150800C3C030BD00BF18ED040828E80408D0E80408C2
S3150800C3D0DCE804080E4B1A7810B44AB90D4B1868F5
S3150800C3E003681C681146A446FF235DF8044B6047A2
S3150800C3F0012A02D05DF8044B7047074B186802689B
S3150800C40014680023A44619465DF8044BFF226047CA
S3150800C410D40F0020D80F0020DC0F0020124B10B5D7
S3150800C420187020B1012810D00024204610BDCC2059
S3150800C4303CF048FB0D4B19680446FFF7CBFD0C4A48
S3150800C4400C4B14602046A36010BDCC203CF03AFB90
S3150800C450064B19680446FFF78BFF074A054B14601D
S3150800C4602046A36010BD00BFD40F0020D00F0020C7
S3150800C470D80F0020D5C30008DC0F002010B4044CE8
S3150800C480044B216000225DF8044B1A70704700BF08
S3150800C490D00F0020D40F0020704700BF002070473F
S3150800C4A0704700BF002070470120704790F8500081
S3150800C4B0704700BF90F87A00704700BFA1F1E0000E
S3150800C4C0B0FA80F0400970472DE9F04385B004467C
S3150800C4D0ADF80A10039200F1220504270026002968
S3150800C4E04AD094F83030042BFDD8DFE803F0030E69
S3150800C4F07A7348000223D4F80910237240F2022204
S3150800C50001232161A28284F830300DF10A0203A9C1
S3150800C51004F1100005F000FF70B3D4F80920137871
S3150800C52084F83130527884F83220C4F80950294604
S3150800C530042AA3F10203DBB208BF84F83360042A95
S3150800C540237263752375216184F830701BD0052A20
S3150800C5505CD0022A4AD0237F002B78D0012BE38BAC
S3150800C5607CD04BB904F12008BDF80A10C4F809803C
S3150800C57084F830600029B4D105B0BDE8F08394F89A
S3150800C5803220042AE3D10DF10A0203A904F11000AE
S3150800C59005F0C2FE0028EFD094F82530FF2BE1D134
S3150800C5A094F82630012BDDD194F83830002B69D069
S3150800C5B094F82730002BD5D094F8222084F835300B
S3150800C5C0012194F8233084F8331084F8362084F84F
S3150800C5D03730C7E7D4F8091094F8322094F8313088
S3150800C5E0A6E794F8322094F831309EE70DF10A0256
S3150800C5F003A904F1100005F08FFE0028BCD094F8BA
S3150800C600253084F8343004F12008ADE70DF10A022C
S3150800C61003A904F1100005F07FFE0028ACD094F8B9
S3150800C6203330002B9ED0606800289BD094F83520C4
S3150800C630036804F12008CDE90028D3F8009094F89F
S3150800C640362094F8373094F83410C8478CE794F8B5
S3150800C6503130023B9BB20122E383227783B1BDF8D6
S3150800C6600A20039903E0E383013182B22BB1013B2F
S3150800C6709BB2501E002AF6D17EE7ADF80A20039138
S3150800C68026776FE794F82730012B7FF46BAF93E793
S3150800C69040F65C23994222D040F20D53994215D0B8
S3150800C6A043690BB9008B00B340F24C53994214D13D
S3150800C6B0B2F51A7F17D040F22F439A4213D040F2B0
S3150800C6C0D530101AB0FA80F04009704740F25A6324
S3150800C6D09A4208D04369002BE4D00020704742F202
S3150800C6E0E8139A42F6D1012070477047019A2BBB8E
S3150800C6F080F85D10D37803F00303032B1FD0022BB9
S3150800C7001CD192F902309178002BACBF0323022387
S3150800C71003EB4303034401F00F0183F8511091889A
S3150800C72083F85210937990F878209A4238BF80F8A7
S3150800C730783090F85E30013380F85E30704792F9B1
S3150800C7400230002BFADA90F85610012363F38701BA
S3150800C75080F856109178DBE72DE9F04385B004465A
S3150800C760ADF80A10039200F12205042700260029D5
S3150800C7704AD094F83030042BFDD8DFE803F0030ED6
S3150800C7807A7348000223D4F80910237240F2022271
S3150800C79001232161A28284F830300DF10A0203A92F
S3150800C7A004F1100005F0B8FD70B3D4F80920137829
S3150800C7B084F83130527884F83220C4F80950294672
S3150800C7C0042AA3F10203DBB208BF84F83360042A03
S3150800C7D0237263752375216184F830701BD0052A8E
S3150800C7E05CD0022A4AD0237F002B78D0012BE38B1A
S3150800C7F07CD04BB904F12008BDF80A10C4F80980AA
S3150800C80084F830600029B4D105B0BDE8F08394F807
S3150800C8103220042AE3D10DF10A0203A904F110001B
S3150800C82005F07AFD0028EFD094F82530E02BE1D109
S3150800C83094F82630012BDDD194F83830002B69D0D6
S3150800C84094F82730002BD5D094F8222084F8353078
S3150800C850012194F8233084F8331084F8362084F8BC
S3150800C8603730C7E7D4F8091094F8322094F83130F5
S3150800C870A6E794F8322094F831309EE70DF10A02C3
S3150800C88003A904F1100005F047FD0028BCD094F870
S3150800C890253084F8343004F12008ADE70DF10A029A
S3150800C8A003A904F1100005F037FD0028ACD094F870
S3150800C8B03330002B9ED0606800289BD094F8352032
S3150800C8C0036804F12008CDE90028D3F8009094F80D
S3150800C8D0362094F8373094F83410C8478CE794F823
S3150800C8E03130023B9BB20122E383227783B1BDF844
S3150800C8F00A20039903E0E383013182B22BB1013B9D
S3150800C9009BB2501E002AF6D17EE7ADF80A200391A5
S3150800C91026776FE794F82730012B7FF46BAF93E700
S3150800C920019A2BBB80F85910D37803F00303032B25
S3150800C9301FD0022B1CD192F902309178002BACBF84
S3150800C9400323022303EB4303034401F00F0183F897
S3150800C9504D10918883F84E10937990F874209A4276
S3150800C96038BF80F8743090F85A30013380F85A305E
S3150800C970704792F90230002BFADA90F85210012328
S3150800C98063F3870180F852109178DBE770B54FF4AE
S3150800C990802104464FF48062C4E91512002543F647
S3150800C9A00840042384F85150A4F8520084F85C30F7
S3150800C9B004F1640504F1740655F8043B184613B1EE
S3150800C9C01B689B689847AE42F6D10025E06C84F850
S3150800C9D050500123A4F8785084F85E30036884F830
S3150800C9E041509B6884F84250A4F8465084F87D501C
S3150800C9F0256684F87A5029469847284670BD00BFB0
S3150800CA002DE9F04F044690464FF480204FF480629B
S3150800CA10C4E9150243F60845002699460423A4F8F6
S3150800CA20525089B00F4684F8516084F85C3004F19E
S3150800CA30640504F1740A55F8046B304616B1336878
S3150800CA409B6898475545F6D10025D4F84CA084F83C
S3150800CA5050500123A4F8785084F85E30DAF8003094
S3150800CA6084F841501B6884F84250A4F8465084F86C
S3150800CA707D50256684F87A502946504698470646DA
S3150800CA80002849D0D0F800B0BBF1000F3FD004F120
S3150800CA90510303AA036080F80690009229462A46A5
S3150800CAA0E06C122304F084FEC6F800B0054618BBF5
S3150800CAB0DAF8002043465668394650462A46B047B3
S3150800CAC084F8500068B39DF81030092B2BD09DF8D8
S3150800CAD013009DF81D10BDF81420BDF8163084F813
S3150800CAE0520084F85410A4F87620A4F87430E0258F
S3150800CAF0284609B0BDE8F08F23680D289B682046B4
S3150800CB0018BFE1259847284609B0BDE8F08FD72514
S3150800CB10284609B0BDE8F08FD625284609B0BDE8F5
S3150800CB20F08FD425E4E701462B462A46E06C04F04C
S3150800CB3099FF236820469B689847D125D8E700BF08
S3150800CB402DE9F04F2DED028BD0F84C8090F85470FB
S3150800CB5090F850104FF0000980F85490D8F800204B
S3150800CB609BB00446126840461E469047002800F0CF
S3150800CB70918005464FF496702FF0FAFA494694F8D4
S3150800CB805030E06C4A4604F06DFF0146002840F03C
S3150800CB908880D8F80030A87194F850101B68404671
S3150800CBA09847002876D0867194F85010E06C04F106
S3150800CBB05103012208EE103A03F04AFA014600280A
S3150800CBC071D1B4F8762040F24C539A4277D0002FB0
S3150800CBD000F0D68004F104094B460025DFF864828C
S3150800CBE0DFF864B209930DF12C0A13AE2946B9464B
S3150800CBF029E00998DFF854C20C9094F85010E06CBC
S3150800CC008DF83420ADF840208DF84820ADF84A203C
S3150800CC10ADF85C208DF85E208DF86420CDF835607F
S3150800CC200F961196CDF82CC004F062FE0135E9B2D4
S3150800CC30002840F0CB8094F85E20032A00F2A480F6
S3150800CC40894540F2C580606FCDF800A04FF0000C12
S3150800CC5040450B46624601D05845CAD1774F0B97D7
S3150800CC6094F85010099FE06C0C978DF834C0ADF815
S3150800CC7040C08DF848C0ADF84AC0ADF85CC08DF824
S3150800CC805EC08DF864C0CDF835600F96119604F035
S3150800CC902FFECBE7D62108461BB0BDEC028BBDE8BC
S3150800CCA0F08F85F80690236809919B682046984777
S3150800CCB0099908461BB0BDEC028BBDE8F08FB4F8A5
S3150800CCC07430B3F51A7F08D040F22F42934204D04D
S3150800CCD040F2D53293427FF47AAF64202FF048FAB7
S3150800CCE094F8501094F85120E06C012304F014FFD6
S3150800CCF001460028D7D163690BB9238B5BB3B4F817
S3150800CD007430B3F51A7F6CD040F22F42934268D044
S3150800CD102346052053F8141F01909E88CDF82D1040
S3150800CD200B23CDE904330022079203920BAD0322AD
S3150800CD300923069500930292414D8DF82C0094F82C
S3150800CD40512094F85010E06CADF831602123CDF8ED
S3150800CD50335004F015F894F8512094F85010E06C0C
S3150800CD60002304F0D9FE002394F85010E06C1A460C
S3150800CD7004F078FE236820469B689847D1218AE705
S3150800CD8094F85E20032A23D994F85010E06C18EE24
S3150800CD90103A03F05DF90146002884D194F8501042
S3150800CDA094F85D3094F85120E06C04F0B5FE014625
S3150800CDB000287FF478AF4FF4C802012384F8810075
S3150800CDC02072C4F8822084F87A3064E701466AE75C
S3150800CDD0002394F85010E06C1A4604F043FED12163
S3150800CDE061E70BAD08230320F521CDE90110CDE954
S3150800CDF00535002207920392092204930092012026
S3150800CE00657E237EE27DA17DADF82C00607D8DF8E0
S3150800CE102E508DF82F30257D8DF830208DF8311065
S3150800CE208DF8320094F8512094F85010E06C8DF883
S3150800CE303350212303F0A4FF8DE700BFCCED04088F
S3150800CE4010010212E8215C0A5A060D05D8ED0408FD
S3150800CE5070B54D4BC164044603F1340223600023C8
S3150800CE604A4D6260C4E91933C4E91B3301264FF4FD
S3150800CE7080204FF480610422C4E9145084F85E606F
S3150800CE80A16584F85C2084F8413084F8433084F83E
S3150800CE904630A4F848302366A4F8783084F87A3007
S3150800CEA004F1680504F1740655F8043B184613B1F5
S3150800CEB01B689B689847B542F6D1E36C00220121AE
S3150800CEC084F8412084F84220A4F8462084F87D207E
S3150800CED084F850202266A4F8782084F87A2084F80A
S3150800CEE05E106BB39A6F72B3DA6FAAB3D3F8802069
S3150800CEF0A2B3D3F884209AB3D3F8882092B3D3F890
S3150800CF008C202AB3D3F8902072B3D3F894206AB34E
S3150800CF10D3F8982062B3D3F89C205AB3D3F8A0204C
S3150800CF2052B3D3F8A4204AB3D3F8A82042B3D3F80F
S3150800CF30AC203AB3D3F8B02022B1D3F8B4204AB122
S3150800CF40204670BD0E221E32204643F8224070BD90
S3150800CF500522F8E70F22F6E70A46F4E70222F2E787
S3150800CF600322F0E70422EEE70622ECE70722EAE7C7
S3150800CF700822E8E70922E6E70A22E4E70B22E2E7C5
S3150800CF800C22E0E70D22DEE7E4ED04080000083C89
S3150800CF90F0B590F8783085B000F1C907CDE900738F
S3150800CFA0054690F8572090F85010C06C40240DF1B3
S3150800CFB00E03ADF80E4003F0C5FE68B105F1640432
S3150800CFC0743554F8043B184613B11B685B689847D8
S3150800CFD0A542F6D105B0F0BDBDF80E3005F16404E2
S3150800CFE07435002BEDD0264656F8043B39461846CC
S3150800CFF013B11B681B689847AE42F5D1E1E700BF3D
S3150800D00070B513220C23064680F8892080F88A30EA
S3150800D01088B008460D46FBF705F9013086F88B00FF
S3150800D020002402E0EB5C82F88C302846FBF7FAF81D
S3150800D030E3B2984206EB030204F10104F2D8334442
S3150800D040002483F88C402846FBF7ECF80430B6F841
S3150800D0508630079480B2CDE90400CDE90244CDE9D3
S3150800D060004406F1890223F00103A6F886300692E9
S3150800D07096F8512096F85010F06C202303F080FEA5
S3150800D08008B070BDF0B590F8813089B00446132B0E
S3150800D09070D8DFE813F07900A400C400E9000F0196
S3150800D0A01E01490157018301D301020245021400FA
S3150800D0B051026F00650274029502BE027100B0F853
S3150800D0C08650290756D500F12206D9493046082246
S3150800D0D03DF0ECFC80B90127A4F8440084F87B00F5
S3150800D0E0D44984F84270162230463DF0DFFC002809
S3150800D0F040F08C8384F8447094F8803033B9B4F8DF
S3150800D1007E2042F208539A4200F0AD8394F84330E9
S3150800D110002B40F01D8394F84830002B40F018830C
S3150800D120092140F20472208CE66984F88910A4F873
S3150800D1308A2000230A2204F1890125F00305A4F8B0
S3150800D140900084F89230A4F88650C4F88C60CDE933
S3150800D1500233CDE90033CDE9052107930492202354
S3150800D16094F8512094F85010E06C03F009FE0D2352
S3150800D17084F8813009B0F0BDB0F88630D907F9D502
S3150800D180062384F88130F5E7B0F88230B0F88420B9
S3150800D19001339BB29A42A0F88230EBD200250323D2
S3150800D1A0A0F88650CDE90255CDE90055079580F8D7
S3150800D1B08930CDE9043300F189020C21A0F88A10E0
S3150800D1C0069290F8512090F85010C06C202303F076
S3150800D1D0D7FD0123A4F8825084F88130CAE7B0F855
S3150800D1E08230B0F8862001339BB2A0F88230D0078F
S3150800D1F000F19082B4F884209342BBD902EB8203F3
S3150800D2005B009BB2B3F5FA6F88BF4FF4FA63A4F8D4
S3150800D2108430002384F88130A4F88230AAE7B0F875
S3150800D2208630D907A6D5002223F021030321092534
S3150800D2301020A4F8863084F88110CDE9041184F80A
S3150800D2408950A4F88A00CDE90222CDE9002204F12A
S3150800D25089030792069394F8512094F85010E06CCD
S3150800D260202303F08DFD85E7B0F886309A0681D530
S3150800D27023F04103A4F8863000220323102004F18A
S3150800D28089010125A4F88A0084F88950CDE9053179
S3150800D290CDE90222CDE9002204930792202394F8CF
S3150800D2A0512094F85010E06C03F06AFD042384F8CA
S3150800D2B081305FE7B0F886305F067FF55BAFC168FF
S3150800D2C0002900F08982FFF79BFE052384F8813048
S3150800D2D050E7B0F88630DE077FF54CAF90F8492066
S3150800D2E0002A3FF44DAF23F4007323F00103A4F89A
S3150800D2F08630042200235048C4F8890004F18901C5
S3150800D300CDE90233CDE90033CDE90521079304922F
S3150800D310202394F8512094F85010E06C03F030FD67
S3150800D320112384F8813025E790F84830002B40F027
S3150800D3309E8190F84330002B40F099810A2384F8A7
S3150800D340813017E7B0F886301A067FF513AF002547
S3150800D35023F0010302200421032204F18906A4F81C
S3150800D360863084F88900A4F88A10CDE90665CDE9E7
S3150800D3700255CDE90055CDE90422202394F8512021
S3150800D38094F85010E06C03F0FBFC94F87C30002B0A
S3150800D39040F04982082384F88130EBE6B0F88630FD
S3150800D3A0DF077FF5E7AE23F48173002123F001033D
S3150800D3B0A0F88630057F407F84F87C1084F89810A2
S3150800D3C0CDE900110522E37F84F88920A27F84F83D
S3150800D3D08C5084F88D0094F8205094F8210084F835
S3150800D3E08E2084F88F304CF61842012340F60456F6
S3150800D3F084F8905084F89100A4F89220C4F89430E8
S3150800D40094F85120A4F88A60CDE90211079104F135
S3150800D410890094F850100690E06C20231025CDE979
S3150800D420045503F0ADFC092384F88130A2E600BF59
S3150800D43060ED04086CED040804100100B0F88630AD
S3150800D440DE057FF597AE13F0020100F08781428B67
S3150800D45080F88C2023F00103A0F88630C2F303215C
S3150800D4600523002211264FF40175893084F88D10A2
S3150800D47084F88960A4F88A50CDE90530CDE90222FE
S3150800D480CDE900220493079294F8512094F850109D
S3150800D490E06C202303F074FC50E790F84130002B31
S3150800D4A07FF468AE90F84330002B7FF463AE90F8B3
S3150800D4B04630002B7FF45EAE90F84830002B7FF4A0
S3150800D4C059AEC168B0F8862007930029CDE9023322
S3150800D4D0CDE9003318BF03264FF0040308BF022620
S3150800D4E022F011024FF4867004F189011A25A4F876
S3150800D4F08620A4F88A0084F88C6084F88950CDE9DF
S3150800D5000531049394F8512094F85010E06C2023C8
S3150800D51003F036FC01220B23227284F8813029E6B7
S3150800D520B0F88630DD0600F1C68058077FF522AED2
S3150800D530102384F881301DE6B0F886309A077FF507
S3150800D54019AE90F87D3013B1012380F846300023D8
S3150800D5500F2263726381A4F8863084F8812009E675
S3150800D560B0F8823001339BB2B3F57A7F7FF654AEBA
S3150800D57000220A23A0F8822080F88130FAE5B0F864
S3150800D58086305B077FF5F6AD0025A0F8865029465C
S3150800D590402289303CF082FC2946402204F1C90029
S3150800D5A03CF07CFC0A2384F84150A4F84250A4F8C5
S3150800D5B0465084F84850A4F87C5084F88130D9E560
S3150800D5C0B0F886309D057FF5D5AD90F87920002A0C
S3150800D5D03FF4D6AD23F00103A4F8863004220023D5
S3150800D5E0AC48C4F8890004F18901CDE90233CDE9D4
S3150800D5F00033CDE9052107930492202394F851209E
S3150800D60094F85010E06C03F0BBFB122384F88130C9
S3150800D610B0E5B0F88630D8077FF5ACAD9E49C4F8BA
S3150800D620891023F001034FF0FF32A4F88630C4F8BE
S3150800D6308D2000230B22FF2004F189011F25A4F861
S3150800D640920084F89150CDE90233CDE90033CDE953
S3150800D650052107930492202394F8512094F850103A
S3150800D660E06C03F08DFB132384F8813082E5B4F86F
S3150800D67086208A4BC4F889300821002322F08102CB
S3150800D68004F18900864DA4F88620C4F88D50CDE9AA
S3150800D6900233CDE90033CDE9051007930491202321
S3150800D6A094F8512094F85010E06C03F069FB0723B6
S3150800D6B084F881305EE5002223F00903A0F886305D
S3150800D6C0C569008C2272A4F894201927CDE9022294
S3150800D6D0CDE90022079240F60426012104F18902C9
S3150800D6E084F88970A4F88A60C4F88C50A4F890006D
S3150800D6F0A4F892100D230692CDE90433202394F85A
S3150800D700512094F85010E06C03F03AFB0C2384F88F
S3150800D71081302FE5002322F00102A4F88620A4F820
S3150800D720823084F88E305F480793CDE90233CDE91D
S3150800D730003302250623082104F1890284F8815062
S3150800D740C4F8890084F88D10CDE90532049382E582
S3150800D75094F87C30002B7FF41DAEE1E423F481734A
S3150800D76023F00103A0F88630057F407F84F89810DF
S3150800D770CDE9011100910522E37F84F88920A27F73
S3150800D78084F88C5084F88D0094F8205094F8210081
S3150800D79084F88E2084F88F3040F604564CF61842EA
S3150800D7A00123A4F88A6084F8905084F89100A4F8BC
S3150800D7B09220C4F8943094F851200791039194F874
S3150800D7C05010E06C102504F189062023CDE9055692
S3150800D7D0049503F0D5FACDE490F84920002A3FF4E1
S3150800D7E0CFAC23F4007323F00103A4F886302E4847
S3150800D7F00791042304F18902CDE90211CDE900114C
S3150800D800C4F88900CDE90532049381E52749162233
S3150800D81030463DF04BF990BB40F2011384F87B701B
S3150800D820A4F8443068E4B4F88630E069218CA4F89A
S3150800D830945023F00903CDE90665CDE90255CDE9F3
S3150800D8400055192640F604250122A4F8863084F8E6
S3150800D85089600D23A4F88A50C4F88C00A4F89010A7
S3150800D860A4F8922048E71249304613223DF01EF9E3
S3150800D87000287FF44BAC012384F87D3046E40D493B
S3150800D880132230463DF012F900287FF435AC84F8AF
S3150800D8907B7031E4560C0101010C08FF01040533C5
S3150800D8A08B9E300A240C03040410010084ED04083E
S3150800D8B0B0ED04089CED040870B50D2190F84350AE
S3150800D8C0C269038C80F8891041F2047188B0044655
S3150800D8D0A0F88A10C0F88C20A0F8903085B390F88C
S3150800D8E07B30062280F89220002B4AD0034653F854
S3150800D8F0142FC0F893209B88A0F897300022C4F80C
S3150800D9009920C4F89D20A4F8A120B4F8865094F86C
S3150800D910512094F85010E06C25F00105A4F88650C3
S3150800D92000231A258934CDE90233CDE9003307935C
S3150800D930CDE905540495202303F022FA08B070BDFA
S3150800D94006693046FAF76EFC84F8920002E0F35C4A
S3150800D95082F893303046FAF765FCEBB2984204EB4E
S3150800D960030205F10105F2D80F2BCED8C3F10F0239
S3150800D97003F19300D2B20132204400213CF08EFA22
S3150800D980C3E7034653F81C2FC0F893209B88A0F8DA
S3150800D9909730B3E7F0B590F878308BB000F1890589
S3150800D9A0CDE90053044690F8542090F85010C06C06
S3150800D9B040260DF12603ADF8266003F0C3F910F0F2
S3150800D9C0FB0F5ED194F88920531E322B59D8DFE815
S3150800D9D013F05A007400B100CA00E800F600090105
S3150800D9E0580058005800580058005800220158009E
S3150800D9F0580058005800580058005800490154016A
S3150800DA005800580058005800580058005800580048
S3150800DA105800580058005800580058005800580038
S3150800DA205800580058005800580058005800580028
S3150800DA3058005D0158003300B4F88630E069218C3F
S3150800DA40069523F001032C2240F20465A4F88630DB
S3150800DA5084F8892000230922A4F88A50C4F88C0087
S3150800DA60A4F89010CDE90233CDE90033CDE90422BC
S3150800DA70079394F8512094F85010E06C202303F093
S3150800DA807FF90BB0F0BD94F88830042B40F21A8168
S3150800DA9094F8431021B994F84810002900F012812F
S3150800DAA000230A2184F8413084F8433084F846304C
S3150800DAB084F8483084F8811006E194F88B60002ECB
S3150800DAC0DFD094F84310F300DBB2002940F0498117
S3150800DAD094F848E0084606E00131C8B203338642A6
S3150800DAE0DBB240F23781E21892F88E5092F88D70C8
S3150800DAF092F88FC005F00F02BEF1000FECD0052A90
S3150800DB00EAD117F0C80FE7D0062303FB004084F8D4
S3150800DB107E7084F87F5084F880C0D0F88C20B4F8E2
S3150800DB208630E261B0F89020228443F08003A4F89E
S3150800DB308630A6E7B4F8863094F88B2043F48071D3
S3150800DB40A4F88610002A40F0C28094F88D2094F834
S3150800DB508C10120202F4706243F481730A43A4F82B
S3150800DB60863062838DE7234694F8922053F88B1FFC
S3150800DB70E1619988218402F00F0194F8913094F8B4
S3150800DB80930084F87F20052984F87E3084F8800085
S3150800DB9000F0A180B4F8863043F01003A4F886306C
S3150800DBA06FE794F88B30002B7FF46BAFB4F88630B0
S3150800DBB023F0020343F00403A4F8863061E794F8DF
S3150800DBC08B30002B40F08E8094F84330002B00F009
S3150800DBD0B38094F84130002B40F0AE80012384F8DE
S3150800DBE041304EE794F88B30002B7FF44AAF04F1AE
S3150800DBF0210304F13F0101E08B4205D093F871201F
S3150800DC0003F8012F002AF7D1B4F8863043F0080349
S3150800DC10A4F8863035E794F88E30002B7FF431AFC0
S3150800DC20B4F88630B4F88C2041F2010143F00100C3
S3150800DC308A42A4F8860000F0DB8041F204018A4299
S3150800DC4000F0DF8041F209018A427FF41AAF2246CA
S3150800DC5043F0210352F88F1F616192882283A4F84A
S3150800DC6086300EE794F843301BB92369002B00F081
S3150800DC70A2802046FFF720FE03E7B4F88630E06965
S3150800DC80218C069523F001030C22DDE6B4F88630D4
S3150800DC90E669208C069523F0010340F604122B252D
S3150800DCA0A4F8863003210023A4F88A2084F8895032
S3150800DCB00C22C4F88C60A4F89000A4F8921084F89A
S3150800DCC09430CFE60133DAB284F88820D9E6062301
S3150800DCD084F88130D5E613F0C80F1CBF012384F8F9
S3150800DCE0473057E7638BB4F886200695C3F30321BC
S3150800DCF084F88C3084F88D10002322F00502132056
S3150800DD0006214FF44175A4F8862084F88E00A4F8FD
S3150800DD108A50CDE90233CDE90033CDE904110793E2
S3150800DD2094F8512094F85010E06C202303F028F85A
S3150800DD30102384F88130A4E694F84830002B3FF489
S3150800DD40A0AE94F84630002B7FF49BAE012384F8EE
S3150800DD50463096E684F87E7084F87F5084F880C052
S3150800DD608FE60021084605E00131C8B20333864232
S3150800DD70DBB2EFD9E21892F88E5092F88FC092F87B
S3150800DD808D7005F00F0EBCF1000F01D1052D0AD0DC
S3150800DD9094F84820002AE7D0BEF1050FE4D117F021
S3150800DDA0C80FE1D0B0E617F00C0F3ED194F8482022
S3150800DDB0002AD9D0F3E7B4F88620E069218C0793C6
S3150800DDC0CDE90233CDE90033069522F001020E268D
S3150800DDD040F204650923A4F8862084F88960A4F82B
S3150800DDE08A50C4F88C00A4F89010CDE9043340E6B4
S3150800DDF094F88F2084F8402043F04103A4F8863035
S3150800DE003FE69A050AD494F88F203AB994F89720F1
S3150800DE1012F0080218BF012284F8792043F400732F
S3150800DE2043F00103A4F886302BE601EB410104EB2D
S3150800DE304103012284F87C2084F87E7084F87F50A0
S3150800DE4084F880C0D3F88C10B4F88620E161B3F862
S3150800DE509030238442F08003A4F8863011E600BF90
S3150800DE6090F87A300BB90020704710B504462EF0AA
S3150800DE7079F9236EC01A00280EDB2EF073F994F890
S3150800DE807830184420662046FFF784FD2046FFF7C1
S3150800DE90F9F82046FFF77CF8002010BD30B5034698
S3150800DEA00C46B0F8865090F8512090F85010C06C87
S3150800DEB083F88C40C4F3032483F88D404FF44174EF
S3150800DEC089B0A3F88A40132483F88E4025F0050507
S3150800DED003F18904A3F8865006940625002483F8DE
S3150800DEE08950CDE90455CDE90244CDE900440794AB
S3150800DEF0202302F045FF09B030BD00BFF0B503F19D
S3150800DF000F0404F4FC7483B002AFADEB040D02AC4D
S3150800DF1003F1040E8DF80810C1F3032C4FEA2E21E5
S3150800DF204CF0200C05460026387EE170397F84F8CF
S3150800DF3001C0237184F802E06671A071E171E3B152
S3150800DF409EB2731E9BB2114604F108005A1C3BF0A0
S3150800DF507DFF06F10803009495F85A2095F85010AD
S3150800DF60E86C02F0B7FC10B90437BD46F0BD642072
S3150800DF702EF0FEF80437BD46F0BD0823EBE700BFD8
S3150800DF80F0B587B00446BDF8305084F80A2102205F
S3150800DF90042284F8090184F80B212812002284F847
S3150800DFA00D5184F80C2184F80E01187884F80F01B5
S3150800DFB05B7884F81031C1F303250B460826D4F89C
S3150800DFC00D11D4F809018DF808308DF80B2045F0AD
S3150800DFD020038DF80D208DF80F200DEB0602009218
S3150800DFE08DF809300C27012504AB8DF80A708DF8D9
S3150800DFF00C608DF80E5094F85A2003C394F850100C
S3150800E000E06C102302F066FC08B907B0F0BD642086
S3150800E0102EF0AEF807B0F0BD70B50446002503260D
S3150800E020082084F8096184F80C5184F80A2184F8D8
S3150800E0300B0188B01A7884F80D215A780C9B84F85D
S3150800E0400E211A7884F80F215B789DF8342084F81D
S3150800E0501031C1F303260B46A4F8125184F8145163
S3150800E0608DF80C3084F8112146F02003D4F80D11F0
S3150800E070D4F80901D4F811218DF80F508DF80D3018
S3150800E0808DF811508DF813500C2301258DF810309A
S3150800E0908DF81250102605AB03AD8DF80E6007C338
S3150800E0A00095142394F85A2094F85010E06C02F066
S3150800E0B011FC08B908B070BD64202EF059F808B0F4
S3150800E0C070BD00BF70B5044600250426082084F8F4
S3150800E0D0096184F80B0184F80C5184F80A211A782E
S3150800E0E084F80D2188B05B7884F80E31C1F30326D5
S3150800E0F00B461B48C4F81001FF2284F80F5184F818
S3150800E10014218DF80C3046F02003D4F80D11D4F8FC
S3150800E1100901D4F811218DF80F508DF80D308DF8BE
S3150800E12011508DF813500C2301258DF810308DF8F9
S3150800E1301250102605AB03AD8DF80E6007C3009587
S3150800E14094F85A2094F85010E06C142302F0C2FB9D
S3150800E15008B908B070BD64202EF00AF808B070BD82
S3150800E160000102FF70B50446002505260A2084F83A
S3150800E170096184F80B0184F80C5184F80A211A788D
S3150800E18084F80D2188B05B7884F80E31C1F3032634
S3150800E1900B468DF8083046F020038DF809304FF00D
S3150800E1A080704AF202021223C4F8100184F80F5153
S3150800E1B0A4F814218DF80A300E23D4F80D11D4F8DA
S3150800E1C00901D4F811218DF80C3001238DF80E3091
S3150800E1D004AB8DF80B508DF80D508DF80F5007C312
S3150800E1E0022284F81621B4F8155194F85A2094F8A6
S3150800E1F05010E06C1D8002AC1623009402F06AFBF6
S3150800E20008B908B070BD64202DF0B2FF08B070BD23
S3150800E210F0B50446062584F80A210420002284F86D
S3150800E220095184F80C2184F80B0187B0187884F812
S3150800E2300D0158780C9B84F80E01187884F80F01A4
S3150800E2405B7884F81031C1F303250B460826D4F809
S3150800E2500D11D4F809018DF808308DF80B2045F01A
S3150800E26020038DF80D208DF80F200DEB0602009285
S3150800E2708DF809300C27012504AB8DF80A708DF846
S3150800E2800C608DF80E5094F85A2003C394F8501079
S3150800E290E06C102302F01EFB08B907B0F0BD64203D
S3150800E2A02DF066FF07B0F0BDF0B50446072584F8E3
S3150800E2B00A210420002284F8095184F80C2184F8E4
S3150800E2C00B0187B0187884F80D0158780C9B84F8F0
S3150800E2D00E01187884F80F015B7884F81031C1F3C1
S3150800E2E003250B460826D4F80D11D4F809018DF834
S3150800E2F008308DF80B2045F020038DF80D208DF899
S3150800E3000F200DEB060200928DF809300C27012527
S3150800E31004AB8DF80A708DF80C608DF80E5094F8E1
S3150800E3205A2003C394F85010E06C102302F0D2FA76
S3150800E33008B907B0F0BD64202DF01AFF07B0F0BD8C
S3150800E34070B5044688B00B260D4684F80961C1F3FA
S3150800E350032684F80A2184F80D319DF830208DF8BB
S3150800E3600C500023082046F02005C4F8103184F824
S3150800E3700E2184F80C3184F80F3184F8143184F8AE
S3150800E3800B018DF80D501025D4F80901D4F80D119C
S3150800E390D4F811218DF80F308DF811308DF813301F
S3150800E3A08DF80E500C2301258DF810308DF812507B
S3150800E3B005AB03AD07C3009594F85A2094F850109E
S3150800E3C0E06C142302F086FA08B908B070BD642020
S3150800E3D02DF0CEFE08B070BD704700BF704700BF75
S3150800E3E0704700BF90F871305BB970B50446806815
S3150800E3F090F8463084B02BB92369DB071ED404B0E5
S3150800E40070BD7047437A002BF6D1637D002BF3D19C
S3150800E41094F86920002AEFD1418B01231125437214
S3150800E42084F86930A1812261227504F16B03009595
S3150800E430FFF7A6FD022384F87130E0E7012604F110
S3150800E4401605CDE9005604F16B03227DA1890393D5
S3150800E450FFF7E2FD30462DF08BFE00220095019273
S3150800E460227DA189039BA068FFF7D6FD237D33444F
S3150800E470304623752DF07CFE2B46227DA189A068A7
S3150800E480FFF720FE042384F8713004B070BD00BF86
S3150800E4900A2282760168002280F87120096A42758C
S3150800E4A010B4074C80F86920A14280F86A200261FE
S3150800E4B002D15DF8044B70475DF8044B084700BF6E
S3150800E4C0E1E3000810B590F86A3082B004463BBB19
S3150800E4D0227DA189A0680132D2B204F16D032275AA
S3150800E4E0009304F11803FFF793FE22681649936810
S3150800E4F08B4223D100230A21A17684F87130126A4F
S3150800E500124963758A4284F8693084F86A3023614F
S3150800E51017D10E220923A27684F8713002B010BDF5
S3150800E520027D81898068013204F16F03D2B22275B7
S3150800E530009304F11B03FFF76BFEC9E720469847D3
S3150800E540E7E720469047E4E791E40008E1E300089E
S3150800E55030B4816039B14C6EDCB18C6EECB1CC6EE6
S3150800E560B4B10C6FDCB10F4C0F4D81F848200B612C
S3150800E57000220A214FF0E043C0E91A340560C0E9D9
S3150800E580082230BC42750261A0F870208176704777
S3150800E590022401EB84046066E5E70124F9E7032415
S3150800E5A0F7E700BF0071005024EE040870B5837EBB
S3150800E5B00B2B84B0044605D00E2B26D00A2B0ED082
S3150800E5C004B070BD03699A05FAD523F400730121D6
S3150800E5D00A22036180F86A10827604B070BD036966
S3150800E5E013F4807234D15905EAD500F11B0123F4DE
S3150800E5F08063036180F86A200091027D818900F1B9
S3150800E6006F038068FFF750FEDAE703695B04D7D526
S3150800E61081898068FFF742FC2268254993684FF68E
S3150800E620FF708B42A0813ED100230A21A17684F88F
S3150800E6307130126A1F4963758A4284F8693084F812
S3150800E6406A302361BCD0204604B0BDE8704010474C
S3150800E65000F11B05012623F480720261CDE90056FC
S3150800E66000F16F03027D818980680393FFF7D4FC6C
S3150800E67030462DF07DFD002200950192227DA1896C
S3150800E680039BA068FFF7C8FC237D334430462375F7
S3150800E6902DF06EFD2B46227DA189A068FFF712FD9D
S3150800E6A00B23A3768CE7204604B0BDE870401847D4
S3150800E6B091E40008E1E3000870B590F87130023B78
S3150800E6C086B00446072B27D8DFE813F03C004D0038
S3150800E6D07B009A00A900D60008002800036999065D
S3150800E6E01AD5036882681D696F48002182F84610AA
S3150800E6F082F8481085424FF00102627540F0CE80DC
S3150800E70062680AB190472368DB69684A934240F019
S3150800E710C880012384F8713006B070BD03691A06F3
S3150800E720FAD5027D818980680132D2B204F16B0381
S3150800E7302275009304F11603FFF76AFD052384F892
S3150800E7407130E9E703695E07E6D5027D818980684D
S3150800E7500132D2B204F116032275FFF7B3FC032384
S3150800E76084F87130D8E703699D07D5D590F86830E5
S3150800E770C27D012B86BF002380F8683043F0700500
S3150800E780837DCDE9003288BF7025818980688DF840
S3150800E790175001230DF11702FFF7B0FB01202DF0EA
S3150800E7A0E7FC227DA189A0680132D2B21323227523
S3150800E7B0009304F16D03FFF7E3FB072384F8713038
S3150800E7C0AAE703699A07A7D590F86830C27D012B96
S3150800E7D086BF002380F8683043F07005837DCDE955
S3150800E7E0003288BF7025818980688DF8175001230B
S3150800E7F00DF11702FFF782FB062384F871308BE7C9
S3150800E80003691B0788D581898068FFF747FB0023C2
S3150800E8104FF6FF72A281236184F871307CE70369A1
S3150800E820DB067FF579AF00F118050126CDE900561C
S3150800E83000F16D03027D818980680393FFF7ECFB85
S3150800E84030462DF095FC002200950192227DA18983
S3150800E850039BA068FFF7E0FB237D3344304623750E
S3150800E8602DF086FC2B46227DA189A068FFF72AFC9D
S3150800E870082384F871304FE7036958067FF54CAFD3
S3150800E880227DA189A0680132D2B204F1180322754B
S3150800E890FFF718FC082384F871303DE72046A8479F
S3150800E8A037E72046984734E71DBD0008DDE3000832
S3150800E8B070B5437D82B004460D4613B90B7A022B18
S3150800E8C044D0A068437A13B990F8473033B9A18980
S3150800E8D02A78CBB29A4219D002B070BD637D002B5C
S3150800E8E0F5D194F86930002BF1D12A7A022AEED1B3
S3150800E8F0AA89112AEBD1418B80F84730012242724E
S3150800E90084F86920A18184F87130E1E76A780B12EE
S3150800E91043F020039A42DFD1EB88012B5BD0AB7919
S3150800E92094F86F20EE799A4271D094F86D209A4245
S3150800E93019D094F86B209A4239D02046FFF736FE54
S3150800E940204602B0BDE87040FFF7B6BE8B89012BA2
S3150800E950B7D18068827A002AB4D18372428BA281A9
S3150800E9600A23A376AEE794F86E20B242E1D12B7A59
S3150800E970A12BE2D12DF0F6FB2368BD4A5B696067DF
S3150800E98093422E7940F0E5816B7A012B00F0D08115
S3150800E990022BD2D1606A0028CFD002680A350095CA
S3150800E9A0B31E1568DBB200222146A847C5E794F8CE
S3150800E9B06C30B342C1D12B7AA32BBED12368AD4AA2
S3150800E9C09B699342B9D029790139C9B205F109027F
S3150800E9D020469847B1E72B7A012BAED0032B3CD0C3
S3150800E9E0022B63D0052B75D0042B00F09480062BE0
S3150800E9F000F0D180072B00F00A810A2B9DD16A7A94
S3150800EA0022756B7B00932B7BFFF79AFC95E794F8AE
S3150800EA107020B24289D12B7A022B00F0A380042BF6
S3150800EA2000F0DD80062B88D16A7AAB7A84F8292033
S3150800EA30072284F82820904D227F84F82A30002364
S3150800EA4084F82B302386E37EE562CDE900320A237B
S3150800EA5004F12802FFF752FA6FE72B8A002B7FF49E
S3150800EA606CAF6B8A002B7FF468AFAB7B94F86F2092
S3150800EA709A4200F0218194F86B209A4200F00B81AB
S3150800EA8094F86D209A427FF458AFEA7B94F86E307A
S3150800EA909A427FF452AF6B7A23752A7B23692276D2
S3150800EAA06A7B627643F04003236146E7AB89012B14
S3150800EAB04DD0112B00F0A080132B7FF43EAF6B7A5C
S3150800EAC02375AA7B23692276EA7B627643F01003D4
S3150800EAD0236132E72B8A002B7FF42FAF2B7B94F828
S3150800EAE06F209A4200F0CA8094F86B209A4200F090
S3150800EAF0F78094F86D209A427FF41FAF6A7B94F8EA
S3150800EB006E309A427FF419AF23696A7A227543F008
S3150800EB102003236111E72B7B94F86F209A4200F0BB
S3150800EB208F8094F86B209A4200F0968094F86D20B6
S3150800EB309A427FF402AF6A7B94F86E309A427FF469
S3150800EB40FCAE6A7A04F11803FFF70CFBF5E66B7A5C
S3150800EB502375AA7B2369E276EA7B227743F48073DE
S3150800EB602361EAE6032384F828306B7A84F829308F
S3150800EB70AB7AE27E84F82A30257F002384F82B308E
S3150800EB8023860523E362CDE900250A2304F128023A
S3150800EB90FFF7B4F9D1E62B7B94F86F209A4200F080
S3150800EBA0AC8094F86B209A4200F0B48094F86D20FB
S3150800EBB09A427FF4C2AE6A7B94F86E309A427FF42A
S3150800EBC0BCAE6A7A227504F11803009304F16D034A
S3150800EBD0FFF76AFB236820469B689847ADE605233E
S3150800EBE084F828306B7A84F82930AB7A84F82A308E
S3150800EBF0214D227F002323E76B7A2375AA7B23699D
S3150800EC00A275EA7BE27543F00103236195E62B7B47
S3150800EC10E27E9A4200F09180A27D9A4200F0A0809E
S3150800EC20227E9A427FF489AE6A7B637E9A427FF49B
S3150800EC3084AE23696A7A227543F0800323617CE6F1
S3150800EC406E7B94F8702096427FF46BAF6A7A04F173
S3150800EC501B03FFF787FA70E66E7B94F86C209642E2
S3150800EC607FF464AF6A7A04F11603FFF77BFA64E669
S3150800EC70D9E3000835BD000805000235697B94F81C
S3150800EC80702091427FF430AF23696A7A227543F483
S3150800EC900073236151E6E97B94F86C2091427FF476
S3150800ECA0EFAE6B7A23752A7B2369A2756A7BE275B8
S3150800ECB043F00403236140E6EE7B94F87020964205
S3150800ECC07FF4D9AE6B7A23752A7BE2760133DAB202
S3150800ECD06B7B2377227504F11B03FFF7F3F92CE608
S3150800ECE0697B94F86C2091427FF403AF23696A7AB2
S3150800ECF0227543F0020323611FE66E7B94F87020A9
S3150800ED0096427FF44EAF23696A7A227543F480638C
S3150800ED10236112E66E7B94F86C2096427FF446AF28
S3150800ED206A7A227504F11603009304F16B034FE720
S3150800ED30206A00287FF431AEFFE5697B227F914285
S3150800ED407FF46AAF23696A7A227543F480432361A4
S3150800ED50F3E5711EC9B205F109022046984713E684
S3150800ED60697BE27D91427FF45BAF23696A7A2275FB
S3150800ED7043F008032361E0E551B9037A03F00F0273
S3150800ED80072A56D013F00E0F0CBF0120002070473B
S3150800ED90132931D0012931D014292DD002293FD089
S3150800EDA0152929D0032932D0162925D0A1F108031F
S3150800EDB0DBB21E2B3FD84C4A22FA03F3DB073CD4BE
S3150800EDC001F0EF03092B40D0A1F12703012B3CD911
S3150800EDD00A293CD029293AD00B293AD02A2938D0F1
S3150800EDE0A1F10E03DBB21D2B35D8404A22FA03F3F4
S3150800EDF0DA0730D50A2321E000207047007A00F0B0
S3150800EE000F00013802288CBF002001207047007AC5
S3150800EE1000F00F00053802288CBF0020012070473B
S3150800EE20007A00F00F00033802288CBF002001206A
S3150800EE307047012070473329C2D10C238068C0F37C
S3150800EE401700D84000F0010070470D23F6E70E239F
S3150800EE50F4E70F23F2E7A1F10F03DBB21D2B09D963
S3150800EE600C290ED02D290CD00D2901D02E2924D1FC
S3150800EE700923E3E71D4A22FA03F3DB0703D50B232D
S3150800EE80DCE70823DAE71E2919D0052927D01D292A
S3150800EE9025D0062925D01F2923D007291DD02029AA
S3150800EEA01BD0A1F11003DBB21F2B0AD8104A22FA95
S3150800EEB003F3DA0705D51023C0E70429E3D10723AE
S3150800EEC0BCE7A1F11103DBB21F2B95D8094A22FA38
S3150800EED003F3DB0790D51123B0E70423AEE7062337
S3150800EEE0ACE70523AAE700BF0180094201004020DC
S3150800EEF00100048001020480B1B3132934D001292A
S3150800EF0049D0142947D0022949D0152947D00329C1
S3150800EF1050D016294ED0A1F10803DBB21E2B42D8D9
S3150800EF205E4A22FA03F3DB073FD401F0EF03092B0D
S3150800EF3044D0A1F12703012B40D90A2943D0292916
S3150800EF4041D00B2944D02A2942D0A1F10E03DBB2C5
S3150800EF501D2B42D8524A22FA03F3DA073DD54FF45D
S3150800EF6080616FF4806302E001216FF0010310B441
S3150800EF70B0F8444090F8432042EA042213401C0AA1
S3150800EF800A42A0F8444080F843305DF8044B14BFA9
S3150800EF9001200020704702216FF00203E7E70421F1
S3150800EFA06FF00403E3E73329BFD14FF480516FF4C0
S3150800EFB08053DCE708216FF00803D8E74FF40051C7
S3150800EFC06FF40053D3E74FF480416FF48043CEE7E4
S3150800EFD04FF400416FF40043C9E7A1F10F03DBB218
S3150800EFE01D2B0CD90C2914D02D2912D00D2901D08E
S3150800EFF02E2930D14FF400716FF40073B7E7284A11
S3150800F00022FA03F3DB0709D54FF400616FF40063B6
S3150800F010ADE74FF480716FF48073A8E71E291CD002
S3150800F020052931D01D292FD0062931D01F292FD0E7
S3150800F030072925D0202923D0A1F11003DBB21F2BE5
S3150800F0400FD8184A22FA03F3DA070AD54FF48031A3
S3150800F0506FF480338BE70429E0D180216FF08003B9
S3150800F06085E7A1F11103DBB21F2B15D80E4A22FA48
S3150800F07003F3DB0710D54FF400316FF4003376E75E
S3150800F08010216FF0100372E740216FF040036EE71E
S3150800F09020216FF020036AE70020704701800942AB
S3150800F0A00100402001000480010204801B2920D9A8
S3150800F0B0A1F12103DAB2122A05D8134BD340DB4358
S3150800F0C013F001031BD0A1F10E03DBB21D2B04D8EC
S3150800F0D00E4A22FA03F3DA0713D4A1F10F03DBB2BF
S3150800F0E01D2B0CD8094A22FA03F3DB0707D5007B48
S3150800F0F07047074BCB40DB4313F00103E3D10020F5
S3150800F1007047C07A704700BFE10304000100402041
S3150800F1100F0FF80B01440879704700BF012910B595
S3150800F1200B4604463FD91146002A3CD01278012ADC
S3150800F13057D0112A42D1032B40D9033BDAB23C2AD5
S3150800F14028BF3C22033104303AF080FEA168236CC4
S3150800F150C1F31701C3F31703994224D021EA030325
S3150800F16084F84330227A206C02F00F021B0A61F3FE
S3150800F1701700072AA4F84430206400D0FAB90123FE
S3150800F180053A022A98BF43F0080394F84E209A429B
S3150800F19009D094F8431084F84E3023EA020363F347
S3150800F1A0030184F8431094F84D303BB121462046BC
S3150800F1B051F8463BBDE810401B68184710BD511E64
S3150800F1C0A2F10103B3FA83F302294FEA5313A2F11A
S3150800F1D0030110D8022943F00203D6D843F00403EA
S3150800F1E0CEE7013BDAB23C2A28BF3C220131043083
S3150800F1F03AF02CFEAAE70229F0D9C1E7F0B4036C6D
S3150800F20090F82F6090F826C090F82A7090F833503E
S3150800F21090F8384090F83C104FF07F3203F0704376
S3150800F22046F0800647F0800745F0800544F08004E4
S3150800F23042604CF0800C43F0080241F08001002344
S3150800F24080F82F60082680F82A7080F83350866088
S3150800F25080F8384080F826C0F0BC80F83C1002647C
S3150800F2600373C0F84630A0F84A30A0F84C3080F84E
S3150800F2704E30704751B9C37E03F00F02072A56D0A5
S3150800F28013F00E0F0CBF012000207047132931D050
S3150800F290012931D014292DD002293FD0152929D08A
S3150800F2A0032932D0162925D0A1F10803DBB21E2B7B
S3150800F2B03FD8524A22FA03F3DA073CD401F0EF03A7
S3150800F2C0092B41D0A1F12703012B3DD90A293DD0AD
S3150800F2D029293BD00B293BD02A2939D0A1F10E0385
S3150800F2E0DBB21D2B36D8464A22FA03F3DB0731D5A3
S3150800F2F00A2221E000207047C07E00F00F00013886
S3150800F30002288CBF002001207047C07E00F00F0045
S3150800F310053802288CBF002001207047C07E00F007
S3150800F3200F00033802288CBF0020012070470120F7
S3150800F33070473329C2D10C22C37E808B43EA002052
S3150800F340D04000F0010070470D22F5E70E22F3E7E2
S3150800F3500F22F1E7A1F10F03DBB21D2B09D90C2906
S3150800F3600ED02D290CD00D2901D02E2924D1092201
S3150800F370E2E7234A22FA03F3DA0703D50B22DBE78F
S3150800F3800822D9E71E2919D005292CD01D292AD0EB
S3150800F39006292AD01F2928D0072922D0202920D09B
S3150800F3A0A1F11003DBB21F2B0AD8164A22FA03F37F
S3150800F3B0DB0705D51022BFE70429E3D10722BBE7FF
S3150800F3C0A1F11103DBB21F2B11D9A1F11203DBB294
S3150800F3D01F2B8FD80C4A22FA03F3DB078AD5122291
S3150800F3E0AAE70422A8E70622A6E70522A4E7074A11
S3150800F3F022FA03F3DA07E8D511229DE701800942CC
S3150800F40001004020010004800104008001020480FC
S3150800F410B1B3132934D0012949D0142947D0022978
S3150800F42049D0152947D0032950D016294ED0A1F125
S3150800F4300803DBB21E2B42D8664A22FA03F3DA0720
S3150800F4403FD401F0EF03092B44D0A1F12703012B88
S3150800F45040D90A2943D0292941D00B2944D02A2941
S3150800F46042D0A1F10E03DBB21D2B42D85A4A22FA2A
S3150800F47003F3DB073DD54FF480616FF4806302E048
S3150800F48001216FF0010310B4B0F8404090F83F2016
S3150800F49042EA042213401C0A0A42A0F8404080F8B7
S3150800F4A03F305DF8044B14BF01200020704702214D
S3150800F4B06FF00203E7E704216FF00403E3E733295B
S3150800F4C0BFD14FF480516FF48053DCE708216FF009
S3150800F4D00803D8E74FF400516FF40053D3E74FF40D
S3150800F4E080416FF48043CEE74FF400416FF4004348
S3150800F4F0C9E7A1F10F03DBB21D2B0CD90C2914D0D7
S3150800F5002D2912D00D2901D02E2930D14FF40071A2
S3150800F5106FF40073B7E7304A22FA03F3DA0709D51E
S3150800F5204FF400616FF40063ADE74FF480716FF438
S3150800F5308073A8E71E291CD0052936D01D2934D08A
S3150800F540062936D01F2934D007292AD0202928D0C1
S3150800F550A1F11003DBB21F2B0FD8204A22FA03F3BE
S3150800F560DB070AD54FF480316FF480338BE7042923
S3150800F570E0D180216FF0800385E7A1F11103DBB2AA
S3150800F5801F2B1CD9A1F11203DBB21F2B15D8144A65
S3150800F59022FA03F3DB0710D54FF480216FF480239A
S3150800F5A071E710216FF010036DE740216FF04003FB
S3150800F5B069E720216FF0200365E700207047094AB4
S3150800F5C022FA03F3DA07DDD54FF400316FF400337E
S3150800F5D059E700BF0180094201004020010004806C
S3150800F5E001040080010204801B2920D9A1F121030E
S3150800F5F0DAB2122A05D8134BD340DB4313F00103C2
S3150800F6001BD0A1F10E03DBB21D2B04D80E4A22FA39
S3150800F61003F3DA0713D4A1F10F03DBB21D2B0CD8C1
S3150800F620094A22FA03F3DB0707D5407E7047074BE2
S3150800F630CB40DB4313F00103E3D100207047007E83
S3150800F640704700BFE1030400010040200F0FF80BCC
S3150800F6500144087D704700BF012910B50B460446D2
S3150800F66044D91146002A41D01278012A62D0312A9B
S3150800F6704DD1022B4BD0023BDAB2282A28BF2822CA
S3150800F680023114303AF0E2FBE27EA18BE36B42EAE8
S3150800F6900121C3F31703994223D021EA030384F80F
S3150800F6A03F30E06B02F00F021B0A61F31700072ACE
S3150800F6B0A4F84030E06300D052BB0123053A022A81
S3150800F6C098BF43F0080394F84B209A4209D094F85F
S3150800F6D03F1084F84B3023EA020363F3030184F8EE
S3150800F6E03F10B4F84C300133A4F84C3094F84A3043
S3150800F6F03BB12146204651F8423BBDE810401B6805
S3150800F7001847E37A002BF4D1E37C002BF1D110BD26
S3150800F710511EA2F10103B3FA83F302294FEA5313E8
S3150800F720A2F1030110D8022943F00203CBD843F013
S3150800F7300403C3E7013BDAB2282A28BF282201318D
S3150800F74014303AF083FB9FE70229F0D9B6E700BFE9
S3150800F75030B4C36B90F8344090F83810082203F0A0
S3150800F76070434FF07F3544F08004C27641F0800143
S3150800F7701A430023456180F8344080F8381030BCBD
S3150800F780C26383830371C3720373C3740383C0F8AC
S3150800F7904230C0F84630A0F84A3070470378262B26
S3150800F7A012D00BD8012B01D0022B23D10B70437832
S3150800F7B04B7083788B700023C3717047FC2B19D16B
S3150800F7C00B700023C37170470B704378DB434B7093
S3150800F7D083780BB102238B70C3780B7103794B7155
S3150800F7E043798B7183795B0808BF01234B72002329
S3150800F7F0C371704700230B704B708B700023C37165
S3150800F800704700BF002070470020704700207047EF
S3150800F810002070470020704711F0800F42D1072B57
S3150800F82040D830B4044612B1C079072837D0E07CF6
S3150800F830002869D0A07E002868D094F82100002806
S3150800F84066D094F82800002864D094F82F00002881
S3150800F85062D094F83600002860D094F83D0000285D
S3150800F8605ED094F8440000285CD094F84B00002839
S3150800F8705AD094F85200002858D094F85900002815
S3150800F88056D094F86000002854D094F867000028F1
S3150800F89052D094F86E0038B194F8750000B3002081
S3150800F8A030BC7047002070470E25D9B1C1F302015C
S3150800F8B04FF0000061F3C500FAB1E1790131C9B230
S3150800F8C0E17101F00701C5EBC50541EA82132C4435
S3150800F8D003F047031843207300F07F0030BC7047DD
S3150800F8E00F25E2E7C5EBC50552B16219412313732B
S3150800F8F0E27901321846E271D2E703F00701E2E73E
S3150800F9002C4401202073CBE70125CEE70225CCE75E
S3150800F9100325CAE70425C8E70525C6E70625C4E77B
S3150800F9200725C2E70825C0E70925BEE70A25BCE77B
S3150800F9300B25BAE70C25B8E70D25B6E7C1EBC102DA
S3150800F94002442DE9F843072303FB0103127B1D7BC1
S3150800F9505306884604464FEAC10940F1CF8005F0B0
S3150800F960070501260827BB1B23441B7BC3F3C203D9
S3150800F970AB4200F0D480731CDBB2102B00F0BB80C6
S3150800F980C3EBC3022244DF00127BC2F3C202AA42BF
S3150800F99000F0C480B31CDBB2102B00F0AC80C3EBC4
S3150800F9A0C3022244DF00127BC2F3C202AA4200F05D
S3150800F9B0B580F31CDBB2102B00F09D80C3EBC302AD
S3150800F9C02244DF00127BC2F3C202AA4200F0A680DC
S3150800F9D0331DDBB2102B00F08E80C3EBC30222442A
S3150800F9E0DF00127BC2F3C202AA4200F09780731DA1
S3150800F9F0DBB2102B7FD0C3EBC3022244DF00127B9D
S3150800FA00C2F3C202AA4200F08980B31DDBB2102BF2
S3150800FA1071D0C3EBC3022244DF00127BC2F3C202D9
S3150800FA20AA427BD0F31DDBB2102B64D0C3EBC30212
S3150800FA302244DF00127BC2F3C202AA426ED006F14C
S3150800FA400803DBB2102B56D0C3EBC3022244DF00F7
S3150800FA50127BC2F3C202AA4260D006F10903DBB2E6
S3150800FA60102B48D0C3EBC3022244DF00127BC2F33B
S3150800FA70C202AA4252D006F10A03DBB2102B3AD0D0
S3150800FA80C3EBC3022244DF00127BC2F3C202AA42BE
S3150800FA9044D006F10B03DBB2102B2CD0C3EBC30208
S3150800FAA02244DF00127BC2F3C202AA4236D006F114
S3150800FAB00C03DBB2102B1ED0C3EBC3022244DF00BB
S3150800FAC0127BC2F3C202AA4228D006F10D03DBB2AA
S3150800FAD0102B10D0C3EBC3022244DF00127BC2F303
S3150800FAE0C202AA421AD0022E05D094F87530C3F382
S3150800FAF0C203AB421BD0E379AB4215D0A9EB080889
S3150800FB00A04401220023043488F80D20C8F80840D0
S3150800FB1088F80C3088F80E30BDE8F8831E46314662
S3150800FB202046FFF70BFF1EE7013DE571E6E70F26C6
S3150800FB307827F4E7D9B3C37C8B4240D0837E8B42C7
S3150800FB403FD090F821308B423DD090F828308B4238
S3150800FB503BD090F82F308B422BD090F836308B4222
S3150800FB6035D090F83D308B4233D090F844308B42F4
S3150800FB7031D090F84B308B422FD090F852308B42D0
S3150800FB802DD090F859308B422BD090F860308B42AC
S3150800FB9029D090F867308B4227D090F86E308B4288
S3150800FBA025D090F875308B4223D000207047083056
S3150800FBB070470523C3EBC303083018447047012375
S3150800FBC0F8E70223F6E70323F4E70423F2E706231C
S3150800FBD0F0E70723EEE70823ECE70923EAE70A2319
S3150800FBE0E8E70B23E6E70C23E4E70D23E2E70E2319
S3150800FBF0E0E70F23DEE700BF41292DE9F843044675
S3150800FC0049D0C37C8B4200F08E81837E8B4200F004
S3150800FC108D8190F821308B4200F08B8190F8283046
S3150800FC208B4200F0898190F82F308B4200F0878153
S3150800FC3090F836308B4200F0858190F83D308B4243
S3150800FC4000F0838190F844308B4200F0818190F86F
S3150800FC504B308B4275D090F852308B4200F07B8146
S3150800FC6090F859308B4200F0798190F860308B42D9
S3150800FC7000F0778190F867308B4200F0758190F834
S3150800FC806E308B4200F0738190F875308B4200F02D
S3150800FC907181BDE8F883021D002301214FF48070AD
S3150800FCA0C4F80F20C4F81620C4F81D206262C4F8F0
S3150800FCB02B20C4F83220C4F839202264C4F847201F
S3150800FCC0C4F84E20E374237784F8213084F82A3068
S3150800FCD084F82F3084F8383084F83D3084F846307C
S3150800FCE084F84B3084F8543084F85930A182618402
S3150800FCF02186E187A4F84C10A4F85A106083208561
S3150800FD00E086A4F84400A4F85200C4F85520A4F8E4
S3150800FD106000A4F86810A4F86E00A4F87610E371E1
S3150800FD2084F86230E26584F86730C4F8632084F8A2
S3150800FD307030C4F86A2084F87530C4F87120BDE8BC
S3150800FD40F8834FF00908C8EBC80323444FEAC809EB
S3150800FD501B7B03F007065B0640F1CF8001250827C9
S3150800FD607B1B23441B7BC3F3C203B34200F0D6803C
S3150800FD706B1CDBB2102B00F0BB80C3EBC302224422
S3150800FD80DF00127BC2F3C202B24200F0C680AB1C8F
S3150800FD90DBB2102B00F0AC80C3EBC3022244DF00B9
S3150800FDA0127BC2F3C202B24200F0B780EB1CDBB290
S3150800FDB0102B00F09D80C3EBC3022244DF00127BA8
S3150800FDC0C2F3C202B24200F0A8802B1DDBB2102B90
S3150800FDD000F08E80C3EBC3022244DF00127BC2F31D
S3150800FDE0C202B24200F099806B1DDBB2102B7FD0A5
S3150800FDF0C3EBC3022244DF00127BC2F3C202B24243
S3150800FE0000F08B80AB1DDBB2102B71D0C3EBC302A5
S3150800FE102244DF00127BC2F3C202B2427DD0EB1D40
S3150800FE20DBB2102B64D0C3EBC3022244DF00127B83
S3150800FE30C2F3C202B24270D005F10803DBB2102B3E
S3150800FE4056D0C3EBC3022244DF00127BC2F3C202C0
S3150800FE50B24262D005F10903DBB2102B48D0C3EBDE
S3150800FE60C3022244DF00127BC2F3C202B24254D05C
S3150800FE7005F10A03DBB2102B3AD0C3EBC3022244C6
S3150800FE80DF00127BC2F3C202B24246D005F10B0371
S3150800FE90DBB2102B2CD0C3EBC3022244DF00127B4B
S3150800FEA0C2F3C202B24238D005F10C03DBB2102B02
S3150800FEB01ED0C3EBC3022244DF00127BC2F3C20288
S3150800FEC0B2422AD005F10D03DBB2102B10D0C3EBDA
S3150800FED0C3022244DF00127BC2F3C202B2421CD024
S3150800FEE0022D05D094F87530C3F3C203B34244D04B
S3150800FEF0E379B34201D1013EE671A9EB0808A044B3
S3150800FF0001220023043488F80D20C8F8084088F830
S3150800FF100C3088F80E30BDE8F8831D462946204681
S3150800FF20FFF70CFD1CE74FF001080CE74FF002083D
S3150800FF3009E74FF0030806E74FF0040803E74FF018
S3150800FF40050800E74FF00608FDE64FF00708FAE651
S3150800FF504FF00808F7E64FF00A08F4E64FF00B08EA
S3150800FF60F1E64FF00C08EEE64FF00D08EBE64FF021
S3150800FF700E08E8E64FF00F08E5E60F257827CDE7E7
S3150800FF8070B4304A304C314E0260011D00224FF4E5
S3150800FF908075446001248160C0F80F10C0F81610FF
S3150800FFA0C0F81D104162C0F82B10C0F83210C0F816
S3150800FFB039100164C0F84710858145830585C586D3
S3150800FFC0A0F84450848244840486C4878273C27429
S3150800FFD0027780F8212080F82A2080F82F2080F8E0
S3150800FFE0382080F83D2080F8462080F84B20A0F87D
S3150800FFF04C40C0F84E10C0F85510C165C0F86310E3
S31508010000C0F86A10C0F871101121A0F85250A0F872
S315080100105A40A0F86050A0F86840A0F86E50A0F8C1
S315080100207640317080F8542070BC80F8592080F8E9
S31508010030622080F8672080F8702080F8752080F8A3
S31508010040B820704750EE040800083C00E10F002074
S31508010050002B46D000293ED010B4C47C8C424ED029
S31508010060847E8C424DD090F821408C423BD090F84A
S3150801007028408C4247D090F82F408C4245D090F8C2
S3150801008036408C4243D090F83D408C4241D090F89E
S3150801009044408C423FD090F84B408C423DD090F87A
S315080100A052408C423BD090F859408C4239D090F856
S315080100B060408C4237D090F867408C4235D090F832
S315080100C06E408C4233D090F875408C4231D0D620A0
S315080100D05DF8044B704708300171036042710020D6
S315080100E07047D82070470324C4EBC4040830204461
S315080100F04271017103605DF8044B002070470124C9
S31508010100F2E70224F0E70424EEE70524ECE70624E7
S31508010110EAE70724E8E70824E6E70924E4E70A24E6
S31508010120E2E70B24E0E70C24DEE70D24DCE70E24E6
S31508010130DAE70F24D8E700BFF0B5054683B00C46C9
S3150801014000294BD0C17CA14200F01781877EA742C6
S3150801015000F01C8190F82110A14200F0198190F855
S315080101602810A14200F0168190F82F10A14200F044
S31508010170B58090F83610A14200F00E8190F83D1036
S31508010180A14200F00B8190F84410A14200F00A81C7
S3150801019090F84B10A14200F0098190F85210A14243
S315080101A000F0088190F85910A14200F0078190F8F3
S315080101B06010A14200F0068190F86710A14200F094
S315080101C0058190F86E10A14200F0048190F875102F
S315080101D0A14200F00381D62003B0F0BD8068002853
S315080101E000F0C88005F1080637467979002900F03C
S315080101F0BC800139C9B2013101EB4101014403E077
S315080102000330884200F0B18007789742F8D18278A6
S31508010210186093080F2B28BF0F230127089A7548E2
S3150801022007FA03F3013B1380102100222CF086FF05
S315080102304FF0E20C4FF0FF3301A902226E488DF808
S3150801024004C08DF8054030F009FA6A483A4610218B
S315080102502CF074FFD82367488DF80330002210214B
S315080102602CF06CFF3A464FF0FF330DF1030162485B
S3150801027030F0F4F900244FF0FF333A4601A95E48FD
S315080102808DF8044030F094FC5A483A4610212CF077
S3150801029055FFB3799DF80440EBB195F8B8301C4386
S315080102A044F002045348002210212CF047FFDA25B6
S315080102B001A94FF0FF3302224F488DF805408DF80A
S315080102C0045030F0CBF94B48012210212CF036FFAF
S315080102D0002003B0F0BD04F0F904E3E70521C1EB02
S315080102E0C10105F1080046184158002942D0A74224
S315080102F056D095F82110A14256D095F82810A1425A
S3150801030056D095F82F10A14256D095F83610A1422D
S3150801031056D095F83D10A14256D095F84410A14201
S3150801032056D095F84B10A14256D095F85210A142D5
S3150801033056D095F85910A14254D095F86010A142AB
S3150801034052D095F86710A14250D095F86E10A14287
S315080103504ED095F87510A14207D10F21C1EBC10105
S315080103604718405800287FF440AF0022DB201A6066
S3150801037003B0F0BDD72003B0F0BDD0F80F1005F1DA
S315080103800F0608300029F5D00121E7E70221A6E783
S315080103900321A4E70421A2E70621A0E707219EE796
S315080103A00221DBE708219AE70321D7E7092196E726
S315080103B00421D3E70A2192E70521CFE70B218EE72E
S315080103C00621CBE70C218AE70721C7E70D2186E736
S315080103D00821C3E70E2182E70921BFE70F217EE73E
S315080103E00A21BBE70B21B9E70C21B7E70D21B5E7D0
S315080103F00E21B3E700100240A0C201202DE9F04FFB
S315080104004D788BB08B46691E3F290592029300F2FF
S31508010410588298462BF0A6FE9BF80220074612F052
S31508010420010F96484FF000024FF0100114BF8026C5
S315080104304026EA242CF082FE4FF0FF3309A9022256
S315080104408F488DF825608DF8244030F007F98B48E0
S31508010450012210212CF072FE07F59C5743460837F6
S31508010460002B00F03382ABB2844CDFF8148206937A
S315080104700DF1230A4FF000090097002210212046AA
S315080104802CF05CFE029B069A934228BF13461E4631
S31508010490079312254FF0FF33012209A940468DF82B
S315080104A0245030F0DBF84FF0FF33324614994046BA
S315080104B030F0D4F80122102120462CF03FFE00220C
S315080104C0102120462CF03AFEF3B21E4601933A2536
S315080104D04FF0FF33022209A940468DF825608DF8B1
S315080104E0245030F0BBF80122102120462CF026FEBC
S315080104F09BF800500022102120462CF01FFE45F0E3
S315080105002005022209A9F2264FF0FF3340468DF84D
S3150801051025508DF8246030F0A1F8012210212046DB
S315080105202CF00CFEC8230022102120468DF821301C
S315080105302CF004FE4FF0FF3301220DF12101404654
S3150801054030F08CF84FF0FF33012209A940468DF8A7
S31508010550249030F02DFB0122102120462CF0EEFDCF
S315080105609DF92430002BDDDA0022102120462CF0DB
S31508010570E5FD48F2CA054FF0FF33022209A94046B4
S31508010580ADF8245030F06AF80122102120462CF0EB
S31508010590D5FDF8270022102120468DF823702CF06E
S315080105A0CDFD4FF0FF3301225146404630F056F853
S315080105B04FF0FF33012209A940468DF8249030F007
S315080105C0F7FA0122102120462CF0B8FD9DF8245097
S315080105D015F00F0500F051810023CDE903332BF007
S315080105E0C1FD009BC01A002880F24881062D49D01A
S315080105F00E2D00F05E81042D00F04F811F48002268
S3150801060010212CF09BFD3A24022209A91C48ADF8B9
S3150801061024404FF0FF3330F021F818480122102109
S315080106202CF08CFDF82315488DF823300022102173
S315080106302CF084FD51464FF0FF330122104830F06B
S315080106400DF8002409A94FF0FF3301220C488DF853
S31508010650244030F0ADFA0948012210212CF06EFD34
S315080106609DF824309BF80220C3F3401363F300027C
S3150801067028468BF802200BB0BDE8F08F0010024027
S31508010680A0C201200022102120468DF823702CF0EB
S3150801069055FD4FF0FF330122514640462FF0DEFF4C
S315080106A04FF0FF33012209A940468DF8249030F016
S315080106B07FFA0122102120462CF040FD9DF82430B6
S315080106C09BF8022083F02003C3F3401363F300026F
S315080106D012F0010F8BF802204FF010014FF00002C3
S315080106E0204614BF80254025EA262CF027FD022244
S315080106F009A94FF0FF3340468DF825508DF824603F
S315080107002FF0ACFF0122102120462CF017FD002204
S31508010710102120462CF012FD3A254FF0FF33022214
S3150801072009A94046ADF824502FF098FF012210215F
S3150801073020462CF003FD149B0022102120461E782A
S315080107402CF0FCFC4FF0120C4FF0FF33022209A9E2
S3150801075040468DF824C08DF825602FF07FFF0122D1
S31508010760102120462CF0EAFC0022102120462CF00C
S31508010770E5FC4FF0FF33022209A98DF824504046C3
S31508010780019D8DF825502FF069FF01221021204681
S315080107902CF0D4FC9BF800500022102120462CF0A6
S315080107A0CDFC45F02005022209A9F2264FF0FF33B8
S315080107B040468DF825508DF824602FF04FFF012211
S315080107C0102120462CF0BAFCC8230022102120460D
S315080107D08DF822302CF0B2FC4FF0FF3301220DF1D7
S315080107E0220140462FF03AFF4FF0FF33012209A9B3
S315080107F040468DF8249030F0DBF90122102120467D
S315080108002CF09CFC9DF92430002BDDDA0022102106
S3150801081020462CF093FC48F2CA054FF0FF3302221A
S3150801082009A94046ADF824502FF018FF01221021DE
S3150801083020462CF083FC0022102120468DF82370D7
S315080108402CF07CFC4FF0FF330122514640462FF035
S3150801085005FF4FF0FF33012209A940468DF8249080
S3150801086030F0A6F90122102120462CF067FC9DF8EC
S31508010870245015F00F057FF4B2AE0025029B079AA6
S3150801088014999B1A9BB2114402931491002B7FF47D
S31508010890F4AD002D3FF4C6AEB0E6049B059A0133CC
S315080108A09BB20493002A3FF432AF93427FF42FAFF1
S315080108B0A4E6039B0133DBB2032B03937FF427AF33
S315080108C09CE6DA2528460BB0BDE8F08F029D0DF1AE
S315080108D0230AA7E670B584B00DF10A051C46002661
S315080108E0009503AB254603960446ADF80A60FFF763
S315080108F023FC40B9089B0093BDF80A2003992B46AF
S315080109002046FFF77BFD04B070BD00BF2DE9F04F0F
S3150801091085B01546894601932BF024FC4FF0000A51
S3150801092000F59C57504C49EA05090837D346554600
S315080109302BF018FCC01B002870DA00221021204673
S315080109402CF0FCFBF22503A94FF0FF33022247489E
S315080109508DF80D908DF80C502FF080FE0122102194
S3150801096020462CF0EBFB414E4FF0C8081DE08DF8F0
S315080109700A802CF0E3FB4FF0FF3301220DF10A0147
S3150801098030462FF06BFE4FF0FF33012203A93046A4
S315080109908DF80C5030F00CF90122102120462CF06C
S315080109A0CDFB9DF90C30AB423CDB2BF0DBFB034660
S315080109B00025DB1BAB422A464FF010012046D6DB49
S315080109C0F8230022102120468DF80B302CF0B6FBB7
S315080109D04FF0FF3301220DF10B0124482FF03EFEA3
S315080109E0002503A94FF0FF33012220488DF80C504A
S315080109F030F0DEF80122102120462CF09FFB9DF8ED
S31508010A000C5005F00F05042D22D00E2D06D10BF141
S31508010A10010B5FFA8BFBBBF1030F89D1284605B0A1
S31508010A20BDE8F08F2A46204610212CF087FB48F2B4
S31508010A30CA0503A94FF0FF3302220C48ADF80C5042
S31508010A402FF00CFE0122102120462CF077FBB7E788
S31508010A50019B0AF1010A1FFA8AFA002B3FF468AFD3
S31508010A609A457FF465AFD9E700100240A0C201207C
S31508010A702DE9F04F2DED028B9B4687B00B46AF4E05
S31508010A805B7800918978029300249DF84C30BBF875
S31508010A9000A0019311F0020F054613464FF010010D
S31508010AA022463046ABF8004008EE105A08EE903A56
S31508010AB00CBF0D462025DDF84890A14F2CF03EFBD2
S31508010AC0EA2005A94FF0FF3302228DF814009C484D
S31508010AD08DF815502FF0C2FD0122102130462CF059
S31508010AE02DFB0394009A18EE903A127818EE100A24
S31508010AF00021FFF70BFF0628054600F0A180002814
S31508010B0040F00E81C8230246102130468DF8113077
S31508010B102CF014FB4FF0FF3301220DF11101384679
S31508010B202FF09CFD4FF0FF33012205A938468DF8B9
S31508010B30145030F03DF80122102130462CF0FEFA0F
S31508010B409DF814305B0740F1F18030232A461021C5
S31508010B5030468DF813302CF0F1FA0DF113014FF0F0
S31508010B60FF33012238462FF079FD4FF0FF3301227A
S31508010B7005A938468DF8145030F01AF801221021CB
S31508010B8030462CF0DBFABBF800409DF81480AAEB3E
S31508010B900404D04524B224EAE474C8BF5FFA8AF88B
S31508010BA044454FF008034FF000024FF0100130465C
S31508010BB0A8BF44468DF812302CF0C0FA4FF0FF3327
S31508010BC001220DF1120138462FF048FD2246002177
S31508010BD0484639F063F94FF0FF334946A2B2384621
S31508010BE02FF0E6FF0122102130462CF0A7FA002249
S31508010BF0102130462CF0A2FA40F2CA4C4FF0FF33CE
S31508010C00022205A93846ADF814C02FF027FD0122A6
S31508010C10102130462CF092FABBF80030029A434470
S31508010C209BB29045A144ABF8003051D353454FD2FE
S31508010C30019B002B3FF456AF18462BF099FA51E762
S31508010C40F8233046002210218DF813302CF076FA5D
S31508010C500DF113014FF0FF33012238462FF0FEFC48
S31508010C60039C8DF814404FF0FF3305A9012238463D
S31508010C702FF09EFF3046012210212CF05FFA0099D1
S31508010C809DF814308A7883F01003C3F3001363F3D5
S31508010C90410212F0020F8A7030464FF010014FF0F0
S31508010CA000020CBF0C462024EA252CF047FA05A9B8
S31508010CB04FF0FF33022238468DF815408DF814504F
S31508010CC02FF0CCFC0122102130462CF037FA09E727
S31508010CD0F8231A488DF81330002210212CF02EFA29
S31508010CE00DF113014FF0FF33012215482FF0B6FC21
S31508010CF000244FF0FF3305A9012211488DF814404D
S31508010D002FF056FF012210210C482CF017FA0099F2
S31508010D109DF814308A78C3F3001363F341028A708D
S31508010D20284607B0BDEC028BBDE8F08FF0252846B2
S31508010D3007B0BDEC028BBDE8F08F00BF0010024082
S31508010D40A0C2012070B584B00DF10A051C46002623
S31508010D50009503AB25460396ADF80A6004469DF84F
S31508010D602460FFF7E9F948B9089B0093BDF80A2002
S31508010D70039901962B462046FFF77AFE04B070BD0B
S31508010D802DE9F04F2DED028B8BB000260DF11604DF
S31508010D909DF85C7000940796ADF816601D469DF89F
S31508010DA05860029607AB03979DF86090BDF864807A
S31508010DB0BDF868B0BDF86C701D9E04469246FFF7F3
S31508010DC0BBF9844628B160460BB0BDEC028BBDE881
S31508010DD0F08F029B8DF821300246039B61488DF8FE
S31508010DE0223010218DF820508DF82390ADF82480FB
S31508010DF0ADF826B02CF0A2F94FF0220C0DF11A012C
S31508010E004FF0FF33012258488DF81AC02FF026FCFF
S31508010E104FF0FF33082208A953482FF01FFC514809
S31508010E20012210212CF08AF9BDF8163052461021FC
S31508010E302046FFF76BFD84460028C4D11C9B6DB282
S31508010E40002B00F08580002D079938DA8B7843F05E
S31508010E5002038B70BBF1000F7CD0B84608EE104A2E
S31508010E601C9FCDF808A081465D46BDF81620ADF851
S31508010E70188006ABCDE9007918EE100AFFF7F8FDE0
S31508010E80062801468446ABEB050E0DF11A033A46D0
S31508010E90304632D0002996D13EB13468BDF81810D3
S31508010EA0D4F800A0ADF81AE0D047BDF81830ED1A0D
S31508010EB04345ADB250D3002D4ED00799D5E7887872
S31508010EC0BDF8162040F0010088701C9800903B463A
S31508010ED02046FFF793FA844600287FF474AF8021F1
S31508010EE0BDF8163052462046FFF710FD8446604687
S31508010EF00BB0BDEC028BBDE8F08FF82319488DF8CD
S31508010F001530002210212CF019F94FF0FF33012278
S31508010F100DF1150114482FF0A1FB4FF0FF33012203
S31508010F200DF11A0110488DF81A902FF041FE012291
S31508010F3010210C482CF002F99DF81A30079983F014
S31508010F4020038A78C3F3401363F341028A708CE75E
S31508010F50002DC4DAA021C3E718EE104ADDF808A06F
S31508010F60F8E700BF00100240A0C201202DE9F047B2
S31508010F700446806888B000284FD00806A37347D472
S31508010F80072A45D8E07C002800F02582A07E0028A3
S31508010F9000F0258294F82100002800F0248294F8B4
S31508010FA02800002800F0238294F82F00002800F07A
S31508010FB0228294F83600002800F0218294F83D0038
S31508010FC0002800F0208294F84400002800F01D82D1
S31508010FD094F84B00002800F01A8294F85200002871
S31508010FE000F0178294F85900002800F0148294F84A
S31508010FF06000B8B194F86700002800F00E8294F8F2
S315080110006E00002800F00B8294F87500002867D05E
S31508011010D426304608B0BDE8F087D726304608B052
S31508011020BDE8F0870C2000295CD0C1F3020502F067
S315080110300702C0EBC00042EAC505204405F07F055A
S315080110400573002DE4D0E27CAA4251D0A27EAA42C1
S3150801105000F0B18194F82120AA4200F0AE8194F8FB
S315080110602820AA4200F0AB8194F82F20AA4200F06A
S31508011070A88194F83620AA4200F0A58194F83D206B
S31508011080AA4200F0A28194F84420AA4200F09F8166
S3150801109094F84B20AA4200F09C8194F85220AA4267
S315080110A000F09B8194F85920AA4200F09A8194F89D
S315080110B06020AA4200F0998194F86720AA4200F0BC
S315080110C0988194F86E20AA4200F0978194F87520C9
S315080110D0AA4200F09681D626304608B0BDE8F087C8
S315080110E00F20A0E7C0EBC000204401250573AAE73D
S315080110F00122C2EBC202A118052700228B732046E2
S31508011100CDE90622CDE90422CDE90222019513464D
S3150801111011460097FFF734FE06464FF496702BF0FA
S3150801112027F8002E3FF475AFE37CAB4200F07981D6
S31508011130A37EAB4200F0778194F82130AB4200F0F0
S31508011140748194F82830AB4200F0718194F82F30FD
S31508011150AB4232D094F83630AB4200F06A8194F84B
S315080111603D30AB4200F0678194F84430AB4200F061
S31508011170648194F84B30AB4200F0618194F85230A7
S31508011180AB4200F05E8194F85930AB4200F05B81C6
S3150801119094F86030AB4200F0588194F86730AB425E
S315080111A000F0558194F86E30AB4200F0528194F804
S315080111B07530AB427FF42DAF0F27C7EBC703234426
S315080111C04FEAC70A1B7B03F007085B0640F1E2807A
S315080111D001254FF00809A9EB050323441B7BC3F33B
S315080111E0C203434500F0E2806B1CDBB2102B00F012
S315080111F0CA80C3EBC30222444FEAC309127BC2F376
S31508011200C202424500F0D180AB1CDBB2102B00F0C4
S31508011210BA80C3EBC30222444FEAC309127BC2F365
S31508011220C202424500F0C180EB1CDBB2102B00F074
S31508011230AA80C3EBC30222444FEAC309127BC2F355
S31508011240C202424500F0B1802B1DDBB2102B00F023
S315080112509A80C3EBC30222444FEAC309127BC2F345
S31508011260C202424500F0A1806B1DDBB2102B00F0D3
S315080112708A80C3EBC30222444FEAC309127BC2F335
S31508011280C202424500F09180AB1DDBB2102B7AD029
S31508011290C3EBC30222444FEAC309127BC2F3C2025B
S315080112A0424500F08280EB1DDBB2102B6BD0C3EBFD
S315080112B0C30222444FEAC309127BC2F3C202424562
S315080112C073D005F10803DBB2102B5CD0C3EBC30264
S315080112D022444FEAC309127BC2F3C202424564D0D3
S315080112E005F10903DBB2102B4DD0C3EBC30222442F
S315080112F04FEAC309127BC2F3C202424555D005F132
S315080113000A03DBB2102B3ED0C3EBC30222444FEAD9
S31508011310C309127BC2F3C202424546D005F10B034B
S31508011320DBB2102B2FD0C3EBC30222444FEAC30909
S31508011330127BC2F3C202424537D005F10C03DBB278
S31508011340102B20D0C3EBC30222444FEAC309127BF8
S31508011350C2F3C202424528D005F10D03DBB2102BB8
S3150801136011D0C3EBC30222444FEAC309127BC2F36D
S31508011370C202424519D0022D05D094F87530C3F33F
S31508011380C203434567D0E379434503D108F1FF38E2
S3150801139084F80780AAEB07072744002304340122AF
S315080113A0BC607A733B73BB7333E61D4629462046F8
S315080113B0FEF7C4FA0FE702229BE6032299E6042206
S315080113C097E6052295E6062293E6072291E6082284
S315080113D08FE609228DE6012025E60A2289E6022002
S315080113E021E60B2285E603201DE60C2281E6042070
S315080113F019E60D227DE6052015E60E2279E6062078
S3150801140011E60F2275E607200DE608200BE60920EE
S3150801141009E60A2007E60B2005E60D2003E60E205D
S3150801142001E60127C9E60227C7E60327C5E6042719
S31508011430C3E60627C1E60727BFE60827BDE609274B
S31508011440BBE60A27B9E60B27B7E60C27B5E60D274B
S31508011450B3E60E27B1E60F254FF07809A6E700BFD8
S315080114602DE9F04F85B0DFF830819DF838B0DFF807
S315080114702C91019000EB810617469A460024B06F1D
S3150801148003685D68454507D11D684D451BD1002593
S31508011490284605B0BDE8F08F5B4652463946A8474F
S315080114A0E02805461ED137B307F11E030199374ACD
S315080114B051F8230003685B69934237D1B06F03681B
S315080114C01D684D45E3D05B4652463946A8470D2867
S315080114D0054630D1E3B2022B2FD864202AF048FE04
S315080114E00134CCE70D284ED1E3B2022BF5D92846B3
S315080114F005B0BDE8F08F26483A4610212BF01EFEAE
S315080115004FF4F5754FF0FF33022203A92148ADF8D0
S315080115100C502FF0A3F81E48012210212BF00EFEC5
S3150801152066202AF025FEB06F0368ADE75146984755
S31508011530B06F0368A8E70028A9D05FB1019B134AD9
S315080115401E3753F8270003685B699342A0D05146BA
S3150801155098479DE73A460E4810212BF0EFFD4FF4C8
S31508011560F5744FF0FF3303A902220A48ADF80C407F
S315080115702FF074F80648012210212BF0DFFD6620B2
S315080115802AF0F6FD84E7002898D081E7A1C400086F
S3150801159000100240A0C201209DC4000805F80008F9
S315080115A02DE9F04F2DED068B93B01D4609930DF1EC
S315080115B0300E002385730DF1340C856807930F46A9
S315080115C0C0F808E019460393019316461A460623FE
S315080115D01224CDF818C000934FF0010C4FF40063A4
S315080115E0CDE90444ADF83030CDF808C03C24802359
S315080115F080468DF83240FFF7C3FBC8F8085000282B
S315080116005FD1BDF83C30DFF8A0A1DFF8A0B109EE43
S31508011610903ABDF83E300AEE103A9DF838300B93F1
S315080116209DF83930B94608EE106A08F1740608EED5
S31508011630907A34460A9609EE103A054608F1B40737
S315080116404E460FE0136A5B451ED1936954498B4296
S3150801165025D1D369534A934240F08780A74205F1C1
S31508011660010533D054F8040F5FFA85F90028F5D03F
S31508011670026813695345E5D098470028EED12068DA
S315080116800268136A5B45E0D019EE101A98470028DC
S31508011690E4D020684249026893698B42D9D01AEE90
S315080116A0102A19EE901A9847002875D0099B0093BD
S315080116B0494618EE103A32464046FFF7D1FED12880
S315080116C0CCD013B0BDEC068BBDE8F08F0A9EDFF8CF
S315080116D0D890DFF8D8A0DFF8C8B0002403E0B742F5
S315080116E004F1010446D056F8040FE5B20028F6D0F5
S315080116F0026813694B451CD1136A534521D1936975
S315080117005B4528D1D369274A934240D1099B009367
S3150801171018EE902A18EE103A29464046FFF7A0FE21
S3150801172000F0F703D12BDAD013B0BDEC068BBDE878
S31508011730F08F98470028D2D130680268136A53455A
S31508011740DDD019EE101A98470028DFD030680268F4
S3150801175093695B45D6D01AEE102A19EE901A984766
S315080117600028BCD130680268CCE70B999847002855
S315080117709CD173E7099B18EE102A18EE901A404679
S31508011780FFF7F4FB13B0BDEC068BBDE8F08F0B99A0
S3150801179098470028A3D1B9E72068026859E700BF2E
S315080117A015F80008A5C4000811F80008A9C400081E
S315080117B02DE9F04F89B004AD1C46009505AB00250F
S315080117C0129F059506469046ADF81050FEF7B4FCF3
S315080117D010B109B0BDE8F08F0246424B4248ADF858
S315080117E01C2010210693ADF81E4022252BF0A6FCDD
S315080117F00DF112014FF0FF3301223C488DF81250CA
S315080118002EF02CFF4FF0FF33082206A937482EF099
S3150801181025FF3548012210212BF090FCBDF8103028
S31508011820424610213046FFF771F80028D1D11FB37F
S3150801183005998B7843F002038B70ECB1DFF8A8B0F9
S31508011840DFF8A8A081462546CDE90079BDF8102024
S31508011850ADF812400DF112033046FFF709F90628D3
S3150801186014D00028B5D1BDF81230ED1A9C42ADB29C
S3150801187002D80DB10599E7E7BDF810304246304662
S31508011880A021FFF743F809B0BDE8F08FF82300223D
S31508011890102158468DF80E302BF050FC4FF0FF33CF
S315080118A001220DF10E0150462EF0D8FE4FF0FF33FE
S315080118B001220DF10F0150468DF80F902FF078F99E
S315080118C00122102158462BF039FC05999DF80F3055
S315080118D08A7883F02003C3F3401363F341028A70C5
S315080118E0B2E700BF8006000100100240A0C2012035
S315080118F02DE9F04F9FB00AAC0025984600940BAB32
S315080119000B95044689461646ADF82850FEF714FC91
S3150801191010B11FB0BDE8F08F02464FF4D06700F151
S3150801192080404FF410230225102100F50430ADF84C
S3150801193030700EAF8DF833500D938DF83280222515
S315080119402BF0FCFB39464FF0FF33012243488DF853
S3150801195038502EF083FE4FF0FF3308220CA93F487A
S315080119602EF07CFE3E48012210212BF0E7FBBDF844
S315080119702830324610212046FEF7C8FF0028C8D174
S315080119800B998B78092543F002038B70AB464FF010
S31508011990000ACDE9007ABDF82820ADF82AB00DF184
S315080119A02A032046FFF764F806282CD00028B0D170
S315080119B0BDF82A30ED1A082BADB202D90DB10B9933
S315080119C0E5E7BDF828303246A0212046FEF79EFFFE
S315080119D000289ED1289B0390CDE90673BDF83A707D
S315080119E0CDF804804FF0400C022506230093CDE97B
S315080119F0047C32464946204602958023FFF7C0F902
S31508011A001FB0BDE8F08FF82315488DF826305246E9
S31508011A1010212BF093FB4FF0FF3301220DF1260124
S31508011A200E482EF01BFE4FF0FF3301220DF1270160
S31508011A300A488DF827A02FF0BBF801221021084883
S31508011A402BF07CFB0B999DF827308A7883F02003CD
S31508011A50C3F3401363F341028A7098E7A0C20120D9
S31508011A6000100240F0B587B00DF10A0400941F4634
S31508011A70002403AB0394ADF80A4006461546FEF763
S31508011A805BFB044630B14FF496702AF071FB204691
S31508011A9007B0F0BD02464FF4A0631D488DF8134008
S31508011AA010210594ADF8103022248DF812702BF010
S31508011AB045FB4FF0FF3301220DF1090115488DF859
S31508011AC009402EF0CBFD4FF0FF33082204A9114837
S31508011AD02EF0C4FD0E48012210212BF02FFBBDF874
S31508011AE00A302A4610213046FEF710FF0446002820
S31508011AF0C9D1BDF80A302A4680213046FEF706FFCD
S31508011B0004464FF496702AF033FB204607B0F0BD21
S31508011B1000100240A0C20120F0B587B00DF10A04F9
S31508011B2000941F46002403AB154606460394ADF8F8
S31508011B300A40FEF701FB024610B1104607B0F0BD98
S31508011B404FF410631B488DF8132010210592ADF848
S31508011B5010308DF8127022242BF0F0FA4FF0FF3373
S31508011B6001220DF1090114488DF809402EF076FD80
S31508011B704FF0FF33082204A90F482EF06FFD0D48D8
S31508011B80012210212BF0DAFA2A46BDF80A30102173
S31508011B903046FEF7BBFE02460028CED12A46BDF8DE
S31508011BA00A3030468021FEF7B1FE0246104607B0DC
S31508011BB0F0BD00BF00100240A0C2012030B583B0BD
S31508011BC0F82362488DF80330002210212BF0B6FA6B
S31508011BD00DF103014FF0FF3301225D482EF03EFD62
S31508011BE0002501A94FF0FF33012259488DF8045009
S31508011BF02EF0DEFF5548012210212BF09FFA9DF8A1
S31508011C00044004F0C004802C49D041D8002C00F0CF
S31508011C108380402C3AD1D8234C488DF803302A4684
S31508011C2010212BF08BFA0DF103014FF0FF3301223E
S31508011C3047482EF013FD4FF0FF33012201A944480E
S31508011C408DF804502EF0B4FF0122404810212BF0E4
S31508011C5075FA9DF8042012F0020244D02A463B4840
S31508011C6010212BF06BFA4CF6DA144FF0FF3301A969
S31508011C7002223748ADF804402EF0F0FC0122334821
S31508011C8010212BF05BFA334B02221A7003B030BDD8
S31508011C90C02CFBD12F4B01221A7003B030BDD823BB
S31508011CA02A488DF803302A4610212BF047FA0DF100
S31508011CB003014FF0FF33012225482EF0CFFC4FF0E8
S31508011CC0FF33012201A922488DF804502EF070FF36
S31508011CD001221E4810212BF031FA9DF8042012F03A
S31508011CE00202BCD02A46194810212BF027FA4CF6D5
S31508011CF0DA3401A94FF0FF3302221548ADF8044042
S31508011D002EF0ACFC1148012210212BF017FA114BC9
S31508011D1003221A7003B030BD22460C4810212BF05D
S31508011D200DFA4DF2DA1501A94FF0FF3302220848E0
S31508011D30ADF804502EF092FC0448012210212BF034
S31508011D40FDF9044B1C7003B030BD00BF0010024002
S31508011D50A0C20120E00F002070B54FF4005182B0F7
S31508011D6004466D482BF0E4F9002800F0BA816B4B64
S31508011D701B78032B00F2C482DFE803F0C3BEBC0262
S31508011D800126674D2B7803F0F003102B00F08B82A8
S31508011D90A06F28B10368634ADB68934240F06B82FF
S31508011DA0E06F28B103685F4ADB68934240F06182BD
S31508011DB0D4F8800028B103685A4ADB68934240F098
S31508011DC05682D4F8840028B10368564ADB689342E0
S31508011DD040F04B82D4F8880028B10368514ADB6881
S31508011DE0934240F04082D4F88C0028B103684D4AEA
S31508011DF0DB68934240F03582D4F8900028B1036835
S31508011E00484ADB68934240F02A82D4F8940028B104
S31508011E100368444ADB68934240F01F82D4F898006D
S31508011E2028B103683F4ADB68934240F01482D4F82C
S31508011E309C0028B103683B4ADB68934240F009825B
S31508011E40D4F8A00028B10368364ADB68934240F00B
S31508011E50FE81D4F8A40028B10368324ADB689342AC
S31508011E6040F0F381D4F8A80028B103682D4ADB684D
S31508011E70934240F0E881D4F8AC0028B10368294AB6
S31508011E80DB68934240F0DD81D4F8B00028B10368DD
S31508011E90244ADB68934240F0D281D4F8B40028B1D1
S31508011EA00368204ADB68934240F064812B78402B13
S31508011EB000F0658100F2D380202B00F0E981302BF8
S31508011EC036D11948002210212BF038F94FF4F57450
S31508011ED04FF0FF33022201A91448ADF804402EF051
S31508011EE0BDFB1148012210212BF028F940232B7044
S31508011EF002B070BD002644E7094D13232B70002656
S31508011F0046E7074D2B7803F0F003102B00F02881E4
S31508011F1011232B7000263BE700080240E00F002042
S31508011F20E10F00200DF8000800100240A0C20120B0
S31508011F30112BDDD1A06F002384F8B83028B10368CE
S31508011F40884A9B68934240F0D981E06F28B10368BB
S31508011F50844A9B68934240F0CF81D4F8800028B127
S31508011F600368804A9B68934240F0C481D4F8840090
S31508011F7028B103687B4A9B68934240F0B981D4F83B
S31508011F80880028B10368774A9B68934240F0AE817E
S31508011F90D4F88C0028B10368724A9B68934240F0D2
S31508011FA0A381D4F8900028B103686E4A9B689342CE
S31508011FB040F09881D4F8940028B10368694A9B686F
S31508011FC0934240F08D81D4F8980028B10368654A98
S31508011FD09B68934240F08281D4F89C0028B103683B
S31508011FE0604A9B68934240F07781D4F8A00028B1F3
S31508011FF003685C4A9B68934240F06C81D4F8A4005C
S3150801200028B10368574A9B68934240F06181D4F826
S31508012010A80028B10368534A9B68934240F0568149
S31508012020D4F8AC0028B103684E4A9B68934240F045
S315080120304B81D4F8B00028B103684A4A9B68934299
S3150801204040F04081D4F8B40028B10368454A9B683A
S31508012050934240F0358112232B7002B070BD512B8B
S3150801206000F00B81802B0DD1002233462046114604
S31508012070FFF796FA002870D0D2283FF439AFA0238B
S315080120802B7035E7502B7FF433AFC82336488DF8CC
S315080120900430002210212BF051F84FF0FF330122B2
S315080120A001A932482EF0DAFA00244FF0FF33012253
S315080120B00DF103012D488DF803402EF079FD2A48CC
S315080120C0012210212BF03AF89DF803305B067FF5C3
S315080120D00FAF51232B702AF045F8254B14301860A1
S315080120E006E70546C823024610211F488DF8023027
S315080120F02BF024F84FF0FF3301220DF102011B48A2
S315080121002EF0ACFA4FF0FF3301A9012217488DF8DA
S3150801211004502EF04DFD1448012210212BF00EF823
S315080121209DF8043013F0200540F0C5800E480022C2
S3150801213010212BF003F8CA2601A94FF0FF3302221A
S315080121400A488DF805508DF804602EF087FA06487E
S31508012150012210212AF0F2FF09E690232B70C7E627
S31508012160002615E609F8000800100240A0C2012061
S31508012170E40F002098472B78402B7FF49BAEE82389
S3150801218061488DF80330002210212AF0D7FF0DF19E
S3150801219003014FF0FF3301225C482EF05FFA002459
S315080121A04FF0FF3301A9012258488DF804402EF05B
S315080121B0FFFC5548012210212AF0C0FF9DF8043082
S315080121C013F001047FF494AED82322464E488DF8C5
S315080121D0033010212AF0B2FF0DF103014FF0FF334E
S315080121E001224A482EF03AFA4FF0FF33012201A99B
S315080121F046488DF804402EF0DBFC434801221021A5
S315080122002AF09CFF9DF804603F48224610212AF0D7
S3150801221095FF46F008064FF0FF3301A902223B4815
S315080122208DF80560DA248DF804402EF017FA364841
S31508012230012210212AF082FF50232B7058E6984775
S315080122402BE6984720E6984715E698470AE6984701
S31508012250FFE59847F4E59847E9E59847DEE59847A5
S31508012260D3E59847C8E59847BDE59847B2E5984745
S31508012270A7E598479CE5984792E529F073FF244B13
S315080122801B68C01A0028FFF633AE80232B70EBE6D5
S3150801229029F068FF1E4B1B68C01A0028FFF628AEF6
S315080122A030232B700DE629F05DFF194AC83020232B
S315080122B010602B706CE52046FFF780FC202535E77A
S315080122C09847C8E69847BDE69847B2E69847A7E60D
S315080122D098479CE6984791E6984786E698477BE6AD
S315080122E0984770E6984765E698475AE698474FE64D
S315080122F0984744E6984739E698472EE6984724E6EC
S31508012300044D002644E500BF00100240A0C201208A
S31508012310E40F0020E10F00200368FBB170B40479D3
S31508012320A4B11388BBB143790E68056836781B1BBF
S31508012330EE540379013B037113880C68013B0134A0
S315080123409BB213800C600479002CEBD1437903719D
S3150801235070BC01207047002070BC70470020704790
S3150801236000B583B0481EADF8062007280DD8DFE86A
S3150801237000F02B04424C5A10101DBDF8062002B17C
S315080123800122334820212AF0D9FE012003B05DF845
S3150801239004FB3049BDF80620086819464FF47A73DC
S315080123A02EF05CF9012003B05DF804FB2949BDF85C
S315080123B00620086819462EF007FD012029F0D8FEE7
S315080123C0012003B05DF804FB0022102120482AF001
S315080123D0B5FE022029F0CCFE1D48012210212AF063
S315080123E0ADFE1D4801224FF400412AF0A7FE012047
S315080123F003B05DF804FBBDF806300BBB1648012295
S315080124004FF400412AF09AFEBFE7BDF8062002B153
S31508012410012210210E482AF091FE2CF053FA0120D0
S3150801242003B05DF804FB0B4A4FF47A7310680DF19B
S31508012430060101222EF012F9012003B05DF804FB12
S31508012440054800224FF400412AF078FE9DE700BFB7
S3150801245000040240E80F00200000024029F088BE6F
S3150801246010B5094B044601224FF4004107481C6088
S315080124702AF064FE0A2029F07BFEBDE81040044AD2
S315080124800449054800F0B6BCE80F002000000240E8
S31508012490612301080000002020C001202DE9F04F2A
S315080124A087B08146BDF840A0CDF800A0119E0D4623
S315080124B014461F4600F0B2F800287BD0BAF1000F87
S315080124C078D0A7F108039AB2C3F3CC0305F10F013B
S315080124D0013322F00702A24407350493531807F182
S315080124E0070B1FFA8AF00593ABB202900393CBF35D
S315080124F0CC0B072F70D9049B039D06EB030AB04644
S3150801250018F8013B0093294602232246484600F063
S3150801251033FD0835D045ADB2F2D1BDF8148007F0C8
S315080125200705002D40D09AF800A0A8F107011AF076
S31508012530010F89B241D1A8F10601012D89B24FEAED
S315080125405A0331D0DA073DD4A8F10501022D89B223
S315080125504FEA9A0328D0DB0739D4A8F10401032DE1
S3150801256089B24FEADA031FD0D8073AD4A8F1030192
S31508012570042D89B24FEA1A1316D0DA0736D4053D67
S31508012580A8F10201ADB289B24FEA5A1365B1DB0768
S3150801259031D408F1FF38012D1FFA88F14FEA9A1A4A
S315080125A002D01AF0010F2BD1029B0134A4B29C422E
S315080125B05E449ED107B0BDE8F08F2246484600F03A
S315080125C0CFFCB8E72246484600F0CAFCBCE72246DB
S315080125D0484600F0C5FCC0E7DDF80C803D46B2462A
S315080125E09FE72246484600F0BBFCBFE7224648461D
S315080125F000F0B6FCC3E72246484600F0B1FCC8E73E
S315080126002246484600F0ACFCCEE700BF10B4BDF840
S31508012610044001945DF8044BFFF740BF70B4BDF860
S315080126200C40B0F84260C58F013C14449642A4B2EE
S3150801263018D3A54201D9A24211D9B0F84040828FD8
S31508012640013B0B448C429BB207D39A420FD999425C
S3150801265094BF0020012070BC70479A42F7D9002028
S3150801266070BC7047A542FAD8A242F8D9E5E701201D
S31508012670F6E700BF10B48C680023A44601215DF873
S31508012680044B604710B48C680023A44603215DF807
S31508012690044B604710B48C680023A44602215DF8F8
S315080126A0044B604710B48C680023A44605215DF8E5
S315080126B0044B60472DE9F0411446127880460E46D0
S315080126C0FF2A0AD0B568002305214046A84700B36A
S315080126D06278FF2A04F10104F4D16578FF2D0FD041
S315080126E0FE2D4AD0EF2D11D8DF2D15D905F00F0291
S315080126F00023B56802214046A84702342278DFE75D
S31508012700B568002305214046A84710B1A2780234CE
S31508012710D6E70020BDE8F081CF2D09D905F00F02D3
S315080127200023B56803214046A84702342278C7E743
S31508012730BF2D18D92D01002302351A460421B76881
S3150801274005F0FE054046B8472846FFF787FE0122F1
S3150801275000230421B7684046B8472846FFF77EFE9E
S3150801276002342278ACE7BD2DD0D82B06CED4284624
S31508012770FFF774FE02342278A2E70120BDE8F08152
S31508012780013AF8B51FFA82FE0EF1010E0E4F0F4EF1
S315080127909E44002213F8014B04F00F0C551C240922
S315080127A016F80CC007F802C0ADB2345D7C5502328A
S315080127B0734592B2EED18C68034B4FF480620821BF
S315080127C0A0470120F8BD00BFEC0F00205CEE04080D
S315080127D0013AF8B55FFA82FE0EF1010E0D4F0E4E63
S315080127E09E44002213F8014B04F00F0C551C2409D2
S315080127F016F80CC007F802C0EDB2345D7C550232FA
S315080128007345D2B2EED18C68024B80220621A047CD
S315080128100120F8BDEC1300205CEE04080120704786
S315080128202DE9F04F85B017460A3A044688460193C2
S315080128300C2A58D8DFE802F0605757575769888F2E
S315080128405757579607004B68B3F80A901A88D3F872
S315080128500CA04FEA49091FFA89F9002A43D00297C1
S31508012860DFF8ACB15746184600269A4602E0D8F872
S3150801287004000288057A02FB056505F0FF055A463C
S3150801288041462046FFF716FF2A4641462046FFF7EE
S3150801289009FF05F10802D2B241462046FFF702FFB9
S315080128A0002241462046FFF7F5FE5C2241462046B6
S315080128B0FFF7F8FE012241462046FFF7EBFE3B46AD
S315080128C04A4641462046FFF75BFF0022414620461D
S315080128D0FFF7D8FE0836BAF80010F2B291424F4413
S315080128E01646C4D8029F019B3A464146204605B082
S315080128F0BDE8F04F00F054BC0222FFF7BBFE414A87
S3150801290041462046FFF7D6FEEDE70122FFF7BAFE5C
S31508012910414620460022FFF7BDFE4146C122204618
S31508012920FFF7C0FE414620460122FFF7B3FE019B91
S315080129301A78414652082046FFF7B4FE002241465E
S315080129402046FFF79FFECEE72F4AFFF7B3FE012089
S3150801295005B0BDE8F08F2D4AFFF7ACFE012005B0A2
S31508012960BDE8F08F4B6858891A88D3F80C9081080E
S315080129700291002AB7D00397DFF894B04F465FFA61
S3150801298081FA18460026994602E0D8F8040002881A
S31508012990057A02FB056505F0FF055A4641462046BC
S315080129A0FFF788FE2A4641462046FFF77BFE6A1C4A
S315080129B0D2B241462046FFF775FE0022414620461F
S315080129C0FFF768FE5C2241462046FFF76BFE0122AF
S315080129D041462046FFF75EFE3B46524641462046A3
S315080129E0FFF7F6FE002241462046FFF74BFE013669
S315080129F0B9F80010029BF2B291421F441646C4D898
S31508012A00039F70E76CEE040808EF0408FCEE04085F
S31508012A10ECEE04084218435C507800EB032080B2C0
S31508012A20704700BF0020704790F92900013080B235
S31508012A30704700BF704700BF08B5FFF7FBFF10F0EE
S31508012A40FD0F14BF0320062008BD00BF0621FFF7AE
S31508012A50E1BF00BF0821FFF7DDBF00BF807A7047DD
S31508012A60C07A70472DE9F84FD0F808B09BF800A056
S31508012A70054650468946FFF7DDFF012807465846B1
S31508012A8014BFFF260F26FFF7E9FF04465846FFF74E
S31508012A90E7FF60298046584630D9FFF7DBFF28B3A0
S31508012AA00BEB00026124C84519D3444517D8504693
S31508012AB0FFF7C2FF0AE04C4528D093783340034418
S31508012AC044451A4404F1010409D0E4B21378FF2BF2
S31508012AD0F1D1444502F1010204F10104F5D10022C4
S31508012AE0EA6185F820201046BDE8F88F5846FFF7B9
S31508012AF0ADFF40B10BEB00024124D4E7FFF7A6FF77
S31508012B00B9F1400FF5D80BF11102CCE717F0FD0F1B
S31508012B1012D003F00F0102391B09A9776B77537895
S31508012B2003F00F011B0985F82010EB7793781B0931
S31508012B302B771046BDE8F88FEB77537885F8203068
S31508012B40D3782B7713796B775379AB771046BDE832
S31508012B50F88F00BF2DE9F04F8A4685B01946914690
S31508012B600646FFF77FFF044600284CD096F82070EA
S31508012B7096F91E2096F91D30B168F57F91F8008007
S31508012B8000973A44A9EB02029A441FFA82FB1FFAFC
S31508012B908AFA5A4651462B463046FFF73FFD80B31F
S31508012BA0E91DC1F3C40167B34046FFF745FF251880
S31508012BB039B37B1E01F1FF38DBB25FFA88F80133BE
S31508012BC008F101085B4405EB08099BB203934F46DC
S31508012BD0544615F8013B0093214600235A463046D0
S31508012BE000F0CAF90834BD42A4B2F2D1039B0BF135
S31508012BF0010B1FFA8BFB9B4547444D4601D0C14447
S31508012C00E6E796F91C0005B0BDE8F08F2DE9F0411D
S31508012C101D46436A904607460C4698472B7840441A
S31508012C209BB11FFA80F80026214642463846FFF72F
S31508012C3091FF15F8013F80B204443044A4B286B22C
S31508012C40002BF1D13046BDE8F0811E463046BDE87D
S31508012C50F08100BF8268002380F828309AB192F982
S31508012C60053080F8293092F90C1090F82B2080F85D
S31508012C702A105B1A402A9BB203D0DBB202FB03F38C
S31508012C809B0980F82C3070478268012380F8283028
S31508012C909AB192F90F3080F8293092F9101090F80C
S31508012CA02B2080F82A105B1A402A9BB203D0DBB28C
S31508012CB002FB03F39B0980F82C307047014B4362F2
S31508012CC0704700BF252A0108014B4362704700BFC0
S31508012CD0292A010870B50D46097871B106460024FE
S31508012CE03046FFF7BFFE96F91C3015F8011F1C4444
S31508012CF0A4B20029F4D1204670BD0C46204670BD09
S31508012D0083688B421AD08160B1B190F82830B3B983
S31508012D1091F9053080F8293091F90C1080F82A10BC
S31508012D2090F82B205B1A402A9BB203D0DBB202FB38
S31508012D3003F39B0980F82C300B4B43627047012B38
S31508012D4008D091F90D3080F8293091F90E1080F8E4
S31508012D502A10E5E791F90F3080F8293091F910101A
S31508012D6080F82A10DCE700BF252A010810B40C6890
S31508012D70A4465DF8044B604710B582B00C680DF1A6
S31508012D8006034622A047BDF8060002B010BD00BFE3
S31508012D9010B582B00C680DF106034722A047BDF8AD
S31508012DA0060002B010BD00BF30B54168044683B0C5
S31508012DB00D680DF106034622A8476168BDF806307D
S31508012DC00D68238020460DF106034722A84761684E
S31508012DD0BDF806300D686380204600234822A847BF
S31508012DE06168E0740D6804F13C0320461722A84780
S31508012DF003B030BD2DE9F041222300254FF001082B
S31508012E0004460E468374C0E902558561A0F8108010
S31508012E1080F834801746FFF751FF104A104B666059
S31508012E20A262A36384F82C500220B76000F05CFC10
S31508012E30314637682B460A222046B847A36B064611
S31508012E4003209847A36B284698471EB12046FFF7EB
S31508012E50ABFF46463046BDE8F08100BF01000040A1
S31508012E60E936010870B5044602206568A36B9847E0
S31508012E70A36B012098472E68294620460023142271
S31508012E80B04704F13C032E68294620461722B0476D
S31508012E90A36B0020BDE87040184700BFF8B58369E9
S31508012EA0044603B198476668A36B02209847A36B4B
S31508012EB00120984735683146002315222046A84740
S31508012EC0054630B13768314604F13C0317222046DE
S31508012ED0B847A36B002098472846F8BDF8B583691B
S31508012EE0044603B198476668A36B02209847A36B0B
S31508012EF00120984735683146002316222046A847FF
S31508012F00054630B13768314604F13C03172220469D
S31508012F10B847A36B002098472846F8BD10B582B07C
S31508012F2043688DF807101C6819460F220DF107032F
S31508012F30A04702B010BD00BF416810B40C68002359
S31508012F40A44610225DF8044B604700BF416810B4DF
S31508012F500C680023A44611225DF8044B604700BFA4
S31508012F6030B44468C1852568028603462146AC46C5
S31508012F702E3330BC3222604770B445689DF80C6028
S31508012F8080F8333080F832602C68C185028629467C
S31508012F90A44600F12E0370BC3B22604780F834102A
S31508012FA0704700BFC37C302B08D0282B0AD0022BD0
S31508012FB014BF0123032380F8343070474FF6FF739B
S31508012FC083867047FF23F6E703880022013B828048
S31508012FD0C3800272704700BF838802884188134400
S31508012FE09BB28B42838012D210B4C488037A2244DE
S31508012FF092B2914298BF01F1FF3203F101030372C4
S3150801300098BF92B2C2805DF8044B01207047002038
S31508013010704700BF4389C28810B4013B84884C803D
S3150801302000205DF8044B08808B80CA80704700BF7A
S3150801303030B44B794A88012B1ED0032B19D1A2F142
S3150801304008039BB29A4214462CBF002101211A4655
S31508013050C3888588934234BF0023012343EA0100CC
S31508013060A5428CBF002000F001000B40184330BC7C
S31508013070704714460021EBE702F10804A4B2A24204
S3150801308094BF00210121E3E730B485884489C068EB
S31508013090521BA408D2B29DF8085012FB04F28C0800
S315080130A0490014FA82F201F0060145B1845C03F085
S315080130B0030303FA01F12143815430BC7047032508
S315080130C0845C8D40EDB224EA0504F0E7F0B50C798D
S315080130D083B00D460646002723061BD46B79032BBE
S315080130E006D8DFE803F0130B0F026B88013B6B80F0
S315080130F0640014F0FF04EFD103B0F0BD6B8801330F
S315080131006B80F5E72B88013B2B80F1E72B88013390
S315080131102B80EDE76A88B3889342DFD8F388934218
S31508013120DCD3298873898B42D8D90097AB79304685
S31508013130FFF7AAFFD2E700BFF0B50C7983B00D46B9
S3150801314006460127A309AB71B1886A8891420AD854
S31508013150F188914207D3708929888842304602D975
S315080131600097FFF791FF6B79032B06D8DFE803F089
S315080131700F130B026B88013B6B80A40014F0FF044C
S31508013180E0D103B0F0BD2B88013B2B80F5E72B88F6
S3150801319001332B80F1E76B8801336B80EDE700BFC4
S315080131A030B5143A4D6885B0342A27D8DFE802F0DD
S315080131B0451B1B2926262626262626262626262694
S315080131C026262626262626266149262626264E260A
S315080131D0262626262626262F262626262626262677
S315080131E026263D4176002846FFF7F6FE002853D0ED
S315080131F06A89E8685200002136F050FE012005B0C0
S3150801320030BD28461946FFF705FF0120F7E719469D
S3150801321028460393FFF70CFF039B0028EED02846A8
S315080132201946FFF753FF0120E9E76A891A80012049
S31508013230E5E76A881A800120E1E72846FFF7C4FE18
S31508013240D6E719462846FFF777FFD7E75A88A988A8
S315080132509142D3D8E9889142D0D31988688988429E
S31508013260CCD900209B7900902846FFF70DFF012055
S31508013270C5E75A88A9889142C0D8E9889142BDD341
S31508013280198868898842B9D901249B790094284606
S31508013290FFF7FAFE2046B2E70020B0E70220AEE7C4
S315080132A02DE9F04F87B00746BDF8405000950C460A
S315080132B090461E46FFF7B2F910B907B0BDE8F08F80
S315080132C0072E40F2E980A6F1080A2AF0070A0AF150
S315080132D0080AA2441FFA8AFAA1464FF0FF0B49468B
S315080132E009F10809CDF800B00023424638461FFA0D
S315080132F089F9FFF741FED145F1D106F00703002B05
S3150801330040F08B80072D40F2AA80A5F1080323F02F
S31508013310070AC2441FFA8AFA03930AF108039BB201
S315080133200593C1464FF0FF0B01234A46CDF800B07D
S3150801333021463846FFF720FE4B46534509F1080951
S315080133401FFA89F9F0D105F00703049315F007036D
S3150801335074D1039B23F00709C1441FFA89F9711E29
S3150801336009F1080321449BB289B20593C2464FF07D
S31508013370FF0B01235246CDF800B038460391FFF7FB
S31508013380FBFD53464B450AF1080A03991FFA8AFAC7
S31508013390EFD1BDF8103073B183F007030133FF2273
S315080133A003F0070302FA03F3DBB20093059A01233C
S315080133B03846FFF7E1FD013DA844072E1FFA88F8B4
S315080133C065D9A6F1080929F0070909F10809A144EF
S315080133D01FFA89F9FF25214608340095002342463C
S315080133E03846A4B2FFF7C8FDA145F4D106F0070691
S315080133F0002E3FF462AF86F00706731C03F007063A
S31508013400FF23B340DBB210934246494638460023B0
S3150801341007B0BDE8F04FFFF7AFBD83F007030133EF
S31508013420FF2203F0070302FA03F3DBB200935146C6
S31508013430002342463846FFF79FFD63E783F00703FB
S31508013440013303F007030BFA03FB5FFA8BF30093CF
S31508013450059A012321463846FFF78EFD79E7002DA7
S31508013460A9D085F00703013303F00702FF23934030
S31508013470DBB200932146012342463846FFF77CFD1D
S31508013480711E214489B22B46CDF8148083E7A146E3
S31508013490002E3FF412AFAEE73346A2462FE700BF30
S315080134A02DE9F04F85B0A3F10806BDF838901F46FF
S315080134B026F0070601F108031E4491448A4615467B
S315080134C0B6B21FFA89F9072F2CD9B34654464FF0DD
S315080134D0FF0821460834CDF8008000232A46A4B205
S315080134E00390FFF749FDB4420398F2D107F00703A9
S315080134F033B90135ADB24D45E5D105B0BDE8F08F1B
S3150801350083F007030133FF2203F0070302FA03F3EB
S31508013510DBB20093594600232A460390FFF72CFD98
S315080135200398E6E73B46D346E2E700BF2DE9F041BB
S3150801353082B00446BDF82080CDF800800D461646B7
S315080135401F46FFF76BF810B902B0BDE8F0813B469C
S31508013550324629462046CDF8208002B0BDE8F04122
S31508013560FFF79EBF002070472DE9F041A2F117052C
S31508013570496882B0174606461C46302D1AD8DFE838
S3150801358005F066191919191919191919191919198C
S31508013590191919191919191F39191919191F191960
S315080135A0191919191919391919191919191919195C
S315080135B019585F00234602B0BDE8F041FFF7D6BBB4
S315080135C00191FFF7E5FB65880199ED43054430460E
S315080135D0FFF7D2FB23880199DB430344ADB223806D
S315080135E065803A4630462346FFF7C0FB012002B004
S315080135F0BDE8F0810191FFF7CBFB65880199ED43A1
S3150801360005443046FFF7B8FB228863790199ADB2C4
S3150801361065800233D543054403F0030363713A46D3
S31508013620304625802346FFF7A1FB012002B0BDE8FD
S31508013630F081FFF7A1FB2080012002B0BDE8F081EF
S31508013640FFF7A6FB2080012002B0BDE8F0812346E2
S3150801365017220191FFF78AFB01993046FFF78CFB88
S31508013660B4F8048001996FEA080880443046FFF7E8
S3150801367083FB27880199FF4307443046FFF788FBF8
S31508013680E3880199DB43054630461D44FFF780FB75
S315080136906388DB4318441FFA88F8BFB2ADB2E080ED
S315080136A00120A4F80080A780658002B0BDE8F081FA
S315080136B0044942688A4200D0704752684260FFF75F
S315080136C073BB00BF1C000020054B42689A4218BF15
S315080136D05A60044A18BF43601A60FFF765BB00BF0A
S315080136E01C00002069350108704700BFF8B5084E6F
S315080136F0084F0223054633700A2400E038B1012237
S315080137002946384633F0BCFD013C3070F6D1F8BD88
S315080137106C1600207016002070B5084E0223054667
S3150801372033700A2400E038B101222946002033F01B
S31508013730A7FD013C3070F6D170BD00BF6C160020A4
S31508013740024B312283F87820704700BFA418002065
S3150801375030B40F4D0F4C104A017040F6B83145612F
S31508013760846141F2883502240186426308210022D8
S31508013770C0E90E54C0E9032230BCC0E90722C0E9FA
S315080137800922A0F84010427042804260C262704726
S31508013790006CCA8800943577801A0600F0B52F4B5D
S315080137A02F4E304F044693E8030087B0C823009094
S315080137B08DF80410052269462B482CF04FFF237813
S315080137C02A4836F81310012229F0B8FC237828482C
S315080137D037F81310012229F0B1FC0A2028F0C8FC99
S315080137E02578A1230022042D02938DF80C2010D8E8
S315080137F036F815101D4829F0A1FC052202A91A4818
S31508013800C8232CF02BFF36F815101848012229F089
S3150801381095FC0A2028F0ACFC2578AD230022042D5E
S3150801382004938DF8142011D836F815100F4829F08D
S3150801383085FCC823052204A90B482CF00FFF36F88E
S3150801384015100A48012229F079FC257837F8151050
S315080138500748002229F072FC07B0F0BDC82E0508FA
S31508013860D0070020D8070020F8C20120000C02402A
S315080138700008024030B56A4B024693E8030091B04E
S31508013880147800908DF80410D3E9060102908DF89A
S315080138900C10D3E9080104908DF81410D3E902013C
S315080138A006908DF81C10D3E90A0108908DF82410AA
S315080138B0D3E90C010A908DF82C10D3E90E010C906E
S315080138C08DF83410D3E91001042C0E908DF83C10B4
S315080138D000F2A380534D544835F81410002229F0FC
S315080138E02DFCC8236946052250482CF0B7FE35F849
S315080138F014104D48012229F021FC35F814104A48C4
S31508013900002229F01BFCC8236946052247482CF0EA
S31508013910A5FE35F814104448012229F00FFC35F8A4
S3150801392014104148002229F009FCC823052202A9DE
S315080139303E482CF093FE35F814103B48012229F035
S31508013940FDFB35F814103848002229F0F7FBC82387
S31508013950052204A935482CF081FE35F814103248A1
S31508013960012229F0EBFB35F814102F48002229F023
S31508013970E5FBC823052206A92C482CF06FFE35F86D
S3150801398014102948012229F0D9FB35F814102648C4
S31508013990002229F0D3FBC823052208A923482CF0C5
S315080139A05DFE35F814102048012229F0C7FB35F8C9
S315080139B014101D48002229F0C1FBC82305220AA9B3
S315080139C01A482CF04BFE35F814101748012229F035
S315080139D0B5FB35F814101448002229F0AFFBC823AB
S315080139E005220CA911482CF039FE35F814100E4899
S315080139F0012229F0A3FB35F814100B48002229F0FF
S31508013A009DFB05220EA90948C8232CF027FE35F887
S31508013A1014100548012229F091FB11B030BD00BFF1
S31508013A20A8E40408D0070020000C0240F8C20120CF
S31508013A3030B5474B024693E803008BB014780090E3
S31508013A408DF80410D3E902018DF80C100290D3E920
S31508013A501A018DF814100490D3E906018DF81C108B
S31508013A600690D3E91C01042C8DF8241008906CD813
S31508013A70384D394835F81410002229F05FFBC82360
S31508013A806946052235482CF0E9FD35F81410324807
S31508013A90012229F053FB35F814102F48002229F08A
S31508013AA04DFBC823694605222C482CF0D7FD35F86D
S31508013AB014102948012229F041FB35F8141026482B
S31508013AC0002229F03BFBC823052202A923482CF032
S31508013AD0C5FD35F814102048012229F02FFB35F8C9
S31508013AE014101D48002229F029FBC823052204A920
S31508013AF01A482CF0B3FD35F814101748012229F09D
S31508013B001DFB35F814101448002229F017FBC823A9
S31508013B10052206A911482CF0A1FD35F814100E4806
S31508013B20012229F00BFB35F814100B48002229F065
S31508013B3005FB052208A90948C8232CF08FFD35F88D
S31508013B4014100548012229F0F9FA0BB030BD00BF5F
S31508013B5088E40408D0070020000C0240F8C20120BE
S31508013B6030B5304B024693E8030087B014780090CD
S31508013B708DF80410D3E91E018DF80C100290D3E9D3
S31508013B802001042C8DF81410049048D8264D274896
S31508013B9035F81410002229F0D1FAC82369460522FE
S31508013BA023482CF05BFD35F814102048012229F032
S31508013BB0C5FA35F814101D48002229F0BFFAC823A2
S31508013BC0694605221A482CF049FD35F8141017489C
S31508013BD0012229F0B3FA35F814101448002229F005
S31508013BE0ADFAC823052202A911482CF037FD35F88C
S31508013BF014100E48012229F0A1FA35F814100B48C1
S31508013C00002229F09BFA052204A90948C8232CF0A9
S31508013C1025FD35F814100548012229F08FFA07B059
S31508013C2030BD00BF88E40408D0070020000C02401C
S31508013C30F8C2012030B583B004788DF8041008164F
S31508013C400A14AD230912032C8DF801008DF8022000
S31508013C508DF803108DF8003013DC0B4D0B4835F841
S31508013C601410002229F06AFA0522694608484FF419
S31508013C707A732CF0F3FC35F814100448012229F064
S31508013C805DFA03B030BD00BFD0070020000C02402A
S31508013C90F8C2012030B5164B04789942A8BF1946D7
S31508013CA083B00D1608140A12A723032C8DF80410E5
S31508013CB08DF801508DF802008DF803208DF800303B
S31508013CC013DC0C4D0C4835F81410002229F036FA8D
S31508013CD00522694609484FF47A732CF0BFFC35F87A
S31508013CE014100548012229F029FA03B030BD00BF96
S31508013CF000FE7F00D0070020000C0240F8C2012018
S31508013D002DE9F04301290B464FF6FF78B8BF012389
S31508013D1083B043450778A8BF43468DF80430A622E9
S31508013D201B120026032F8DF80330ADF800208DF8FD
S31508013D30026002DD03B0BDE8F083DFF888900C4627
S31508013D40054639F817101D48324629F0F7F94FF498
S31508013D507A73694605221A482CF080FC39F817103F
S31508013D601648012229F0EAF944452D78A8BF4446A8
S31508013D70211622148DF80440A8232412032D8DF848
S31508013D8001108DF802208DF803408DF80030D1DC42
S31508013D9039F815100948324629F0D0F969464FF421
S31508013DA07A73052206482CF059FC39F81510034890
S31508013DB0012229F0C3F903B0BDE8F083000C0240E3
S31508013DC0F8C20120D007002030B54FF6FF7399429B
S31508013DD00478A8BF194683B00D1608140A12A82339
S31508013DE0032C8DF804108DF801508DF802008DF81A
S31508013DF003208DF8003013DC0A4D0B4835F81410F2
S31508013E00002229F09BF90522694608484FF47A737E
S31508013E102CF024FC35F814100348012229F08EF9F8
S31508013E2003B030BDD0070020000C0240F8C20120C3
S31508013E302DE9F04F067883B04FF0A0080423032E2E
S31508013E40CDF800808DF8043002DD03B0BDE8F08FAF
S31508013E503D4D0C46074635F816103C48002229F018
S31508013E606DF94FF47A736946052239482CF0F6FB49
S31508013E7035F816103548012229F060F93E784FEADF
S31508013E80146BC4F3074AC4F30729A123E4B2032E2A
S31508013E908DF801B08DF802A08DF803908DF80440D5
S31508013EA08DF80030D1DC35F816102848002229F0A3
S31508013EB045F94FF47A730522694625482CF0CEFB5D
S31508013EC035F816102148012229F038F93E788DF87F
S31508013ED001B0AD23032E8DF802A08DF803908DF85D
S31508013EE004408DF80030B0DC35F81610174800226A
S31508013EF029F024F94FF47A730522694614482CF0FF
S31508013F00ADFB012235F81610104829F017F93C784F
S31508013F10CDF800800022032C8DF8042095DC35F8B5
S31508013F2014100A4829F00AF969464FF47A730522EA
S31508013F3007482CF093FB35F814100448012229F0A0
S31508013F40FDF803B0BDE8F08FD0070020000C024051
S31508013F50F8C2012070B56C4B024693E8030092B093
S31508013F60147800908DF80410D3E9020104908DF8B5
S31508013F701410D3E9040106908DF81C10D3E9060143
S31508013F8008908DF82410D3E908010A908DF82C10B1
S31508013F90D3E90A010C908DF83410D3E90C010026F7
S31508013FA0A522A023042C109002928DF80C608DF89E
S31508013FB03C600E938DF8441000F2A380534D54488B
S31508013FC035F81410324629F0B9F8C823052269468E
S31508013FD050482CF043FB35F814104D48012229F0BE
S31508013FE0ADF835F814104A48324629F0A7F8C8231F
S31508013FF0052202A947482CF031FB35F8141044482C
S31508014000012229F09BF835F814104148324629F067
S3150801401095F8C823052204A93E482CF01FFB35F85C
S3150801402014103B48012229F089F835F8141038484C
S31508014030324629F083F8C823052206A935482CF00B
S315080140400DFB35F814103248012229F077F835F8B6
S3150801405014102F48324629F071F8C823052208A9F9
S315080140602C482CF0FBFA35F814102948012229F0BE
S3150801407065F835F814102648324629F05FF8C82342
S3150801408005220AA923482CF0E9FA35F81410204824
S31508014090012229F053F835F814101D48324629F043
S315080140A04DF8C82305220CA91A482CF0D7FA35F879
S315080140B014101748012229F041F835F8141014484C
S315080140C0324629F03BF8C82305220EA911482CF0DF
S315080140D0C5FA35F814100E48012229F02FF835F8DB
S315080140E014100B48324629F029F8052210A9094867
S315080140F0C8232CF0B3FA35F814100548012229F023
S315080141001DF812B070BD00BF10E50408D0070020E5
S31508014110000C0240F8C201202DE9F04F83B00129B5
S315080141209DF830909DF834809DF838A014461E46B7
S31508014130054600F0AB80022900F0A5802846FFF766
S3150801414009FF544A2F786C63A242A8BF2246131668
S315080141508DF8013013148DF804208DF802301212EF
S31508014160A723032F8DF803208DF8003007DD2E864F
S3150801417085F8409085F8418003B0BDE8F08F464C3C
S31508014180464834F81710002228F0D8FF4FF47A73FE
S315080141906946052242482CF061FA34F817103F485F
S315080141A0012228F0CBFF012E95F800B02E86334662
S315080141B0B8BF01231912A6220027BBF1030F8DF8F8
S315080141C004308DF80310ADF800208DF80270CFDCAD
S315080141D034F81B1031483A4628F0B0FF4FF47A7389
S315080141E0052269462E482CF039FA34F81B102B485B
S315080141F0012228F0A3FF95F800B08DF8027032125B
S31508014200A823BBF1030F8DF804608DF80320ADF8E0
S315080142100030ADDC34F81B1020483A4628F08EFFF2
S315080142204FF47A73052269461D482CF017FA34F8BB
S315080142301B101A48012228F081FF2E7885F8409034
S315080142409023032E85F841808DF802A08DF80390FE
S315080142508DF80480ADF800308EDC34F816100F485E
S315080142603A4628F06BFF69464FF47A7305220C48E3
S315080142702CF0F4F934F816100848012228F05EFFEC
S3150801428003B0BDE8F08FFFF7F5FA57E7FFF7D0FB64
S3150801429054E700BF00FE7F00D0070020000C024053
S315080142A0F8C2012030B58DB00024264B00941A6B54
S315080142B0254842F001021A631A6B02F001020092C4
S315080142C0009A01945A6C42F480725A645B6C0894A1
S315080142D003F4807301930222032306A9CDE9062379
S315080142E0019D28F06FFD1948194B1A4A03604FF4CE
S315080142F080310123CDE90344029405948460046165
S31508014300047680F82040C462C46080F83040416079
S315080143108262C361436127F03DFF60B9012201232F
S3150801432000240A48049402A9CDE9022328F0D2F808
S3150801433020B90DB030BD22F06BFBEFE722F068FB28
S315080143400DB030BD003802400000024064C00120B3
S31508014350002001400100000F10B50168164A88B017
S3150801436000239142CDE90233CDE90433069301D006
S3150801437008B010BD02F58C320093516C0F4841F418
S3150801438080715164516C01F4807100910099019317
S31508014390116B41F001011163126B049302F00102E2
S315080143A001920323062202A9CDE90223019C28F0E2
S315080143B009FD08B010BD00BF002001400000024001
S315080143C00A4808B50A4B036000231022C0E90533E1
S315080143D08383C0E90123C0E9033328F035F900B91D
S315080143E008BDBDE8084022F013BB00BFACC00120E0
S315080143F00064004030B50168184A89B0002391422B
S31508014400CDE90233CDE90433069301D009B030BDB5
S3150801441002F5EA320093116C114841F000711164FA
S31508014420116C01F00071009100990193136B43F02F
S3150801443008031363136B03F0080301930923019A15
S3150801444006930022032302A903240225CDE9024586
S31508014450CDE9042328F0B6FC09B030BD006400405C
S31508014460000C024030B51348134B036083B0002398
S31508014470CDE9003328F002FA88B93C2400250D4815
S3150801448000226946CDE9004528F00EFA70B90948B7
S315080144906946102228F008FA20B903B030BD22F087
S315080144A0B7FAEAE722F0B4FA03B030BD22F0B0FA5F
S315080144B0EDE700BFD4C001200074004010B50168C3
S315080144C0164A88B000239142CDE90233CDE9043377
S315080144D0069301D008B010BD02F5E2320093116CC3
S315080144E00F4841F000511164116C01F0005100911F
S315080144F000990193116B41F001011163126B049349
S3150801450002F0010201920323302202A9CDE9022316
S31508014510019C28F057FC08B010BD00BF007400408C
S315080145200000024010B582B00024304B00941A6B8B
S3150801453042F480021A631A6B02F480020092009A0E
S3150801454001941A6B42F400121A631B6B03F40013ED
S315080145502246019307210C20019B28F00BF90C2018
S3150801456028F040F9224608210E2028F003F90E20EA
S3150801457028F038F922460921102028F0FBF81020E6
S3150801458028F030F922460A21112028F0F3F81120E3
S3150801459028F028F9224621462F2028F0EBF82F206B
S315080145A028F020F9224605213A2028F0E3F83A2096
S315080145B028F018F9224603213B2028F0DBF83B2096
S315080145C028F010F922460421452028F0D3F8452081
S315080145D028F008F922460621462028F0CBF846207D
S315080145E002B0BDE8104028F0FDB800BF003802400F
S315080145F02DE9F04F00248DB0CDE90644CDE90844F4
S31508014600654B00940A941A6BDFF89481DFF894B12C
S31508014610DFF89491614DDFF894A142F010021A6314
S315080146201A6B02F010020092009A01941A6B42F07A
S3150801463004021A631A6B02F004020192019A0294A7
S315080146401A6B42F080021A631A6B02F08002029218
S31508014650029A03941A6B42F001021A631A6B02F06A
S3150801466001020392039A04941A6B42F002021A6336
S315080146701A6B02F002020492049A05941A6B42F02C
S3150801468008021A631B6B03F00803059340460122CF
S315080146901021059B28F052FD2246584642F2C321B5
S315080146A028F04CFD2246484648F2010128F046FD0D
S315080146B0224628464FF6106128F040FD2846012279
S315080146C0802128F03BFD224650464FF44C7128F0D4
S315080146D035FD22464046032128F030FD00260027F5
S315080146E006A9404613220123CDE90623CDE9086729
S315080146F028F068FB584606A942F2C3220123CDE9F0
S315080147000623CDE9086728F05DFB06A9484648F265
S3150801471001020123CDE90623CDE9086728F052FBFA
S315080147204FF0010C404606A94FF680720023CDF8DA
S3150801473020C0CDE9062328F045FB06A928464FF6F1
S3150801474090620123CDE90623CDE9086728F03AFBF3
S31508014750484606A94FF480720223CDE90623CDE91E
S3150801476008670A9428F02EFB284606A90822002382
S31508014770CDE90623089428F025FB4FF44C72012352
S3150801478006A95046CDE90867CDE9062328F01AFBA4
S315080147900DB0BDE8F08F00BF00380240000C0240A2
S315080147A000100240000802400000024000040240D6
S315080147B00B480C4908B50C4B03604FF480420023A3
S315080147C0C0E90233C0E90533C0E907334160026134
S315080147D028F09CFE00B908BDBDE8084022F018B9CA
S315080147E0E8C00120801A06000054004070B502682E
S315080147F0184B88B000249A42CDE90244CDE9044415
S31508014800069401D008B070BD134D00942B6B134864
S3150801481043F002032B632B6B03F002030093C022C0
S315080148201223CDE9022301220323CDE9042302A998
S3150801483004230693009E28F0C5FA01942B6C43F4D1
S3150801484000132B642B6C03F400130193019B08B02E
S3150801485070BD00BF00540040003802400004024009
S31508014860BFF34F8F0549064BCA6802F4E06213434A
S31508014870CB60BFF34F8F00BFFDE700BF00ED00E03F
S315080148800400FA05704700BFF8B5B94B93F9003033
S31508014890F3B9B84C2378002B00F0BC80012B00F04B
S315080148A08180B548B54DB64EB0F900302968B6F9DC
S315080148B00020052BDBBF06230380D81E03201329FE
S315080148C063DC14218242296067DB043B3380F8BD2F
S315080148D0012BFCD1A74C2278002A00F0CC80012AB2
S315080148E07CD0A84AA84DA9491068B5F90070B1F954
S315080148F00060A74B0E2800F3A78093ED007ADFED41
S31508014900A56AB4EEE67AF2EE067A0F20F1EE10FA0F
S3150801491067EE277A106011DDFDEEE77A17EE900A49
S31508014920B8EEE77AC2ED007ADFED9B7AB4EEE77A64
S31508014930F1EE10FA40F3B88098481060002FC0F2E3
S315080149409780C82FC4BFC8232B80002EC0F28D8044
S31508014950C82EC4BFC8230B80F3F714FE82A3D3E97C
S315080149600023F3F779FE8E4E04460D463068F3F7B9
S3150801497009FE22462B46F4F7E1F80028A7D020467F
S315080149802946F4F719F93060F8BDB1F5875FC4BF58
S315080149904FF487512960824297DA012A97DC02236C
S315080149A03380F8BD7F4B1B780B3B082B3FF679AF5D
S315080149B001A252F823F000BFDB4B0108FB4B0108AB
S315080149C0414B0108B94B01081F4B0108A3480108CF
S315080149D0F94A0108A3480108CD4A0108714B1B7819
S315080149E00B3B082B3FF67DAF01A252F823F000BF1F
S315080149F0EB4C0108CF4C0108854C0108594C0108BC
S31508014A000B4D0108E3480108A74C0108E3480108D2
S31508014A101D4C010863490A780C2A00F087810E2A81
S31508014A2000F098810B2A7FF43CAF5348534D544EFE
S31508014A30DFF880C1B0F900302968B6F900200127EE
S31508014A408CF80070277034E7D3ED007AB2EE067A57
S31508014A5067EE877A07EE100AB8EEC77AB4EEE77AF8
S31508014A60F1EE10FA7FF560AF56E700230B8073E786
S31508014A7000232B8069E74B4801780C2900F09081C7
S31508014A800E2900F07A810B297FF42BAF3D4A3E4D62
S31508014A903E49DFF820C11068B5F90070B1F9006028
S31508014AA023708CF8003024E7B0F5167FFFF646AF81
S31508014AB03D4CC31784FB00C4C3EBA40303EB830378
S31508014AC0B0EB43031CBFC01A106037E7374B93F9A5
S31508014AD00030002B40F0D6812748354A03881478E0
S31508014AE0264D274E2968B6F900201B1B1BB20380E9
S31508014AF0304C01272770DCE62C4B93F90030002B4C
S31508014B0040F07B811C482A4B04881B781B4D1C4EA0
S31508014B102968B6F9002023441BB20380E8E7234B32
S31508014B2093F90030002B40F0BC811348134D0388DC
S31508014B30134E2968B6F9002014331BB20380D7E750
S31508014B401A4B93F90030002B40F066810A480B4D49
S31508014B5003880B4E2968B6F90020143B1BB2038063
S31508014B60C6E700BFAFF30080BA490C022B87863F20
S31508014B70A0070020541C002070060020E007002032
S31508014B80700B0020FC0B00202CBD01202ABD012042
S31508014B9068330020A38BAE3F00BA5B49A0BB0D006A
S31508014BA0040C002064B70120676666665D2F002045
S31508014BB0D4020020CC070020A54B93F90030002B26
S31508014BC040F03881A348A44D0388A44E2968B6F954
S31508014BD00020013B1BB203808AE7A14F9D489E4DE9
S31508014BE09E4EB0F900302968B6F900204FF0010C45
S31508014BF087F800C0002727705BE6954B93F90030CC
S31508014C00002B40F05C819348934D0388934E2968A5
S31508014C10B6F9002001331BB2038069E7914B93F97A
S31508014C200030002B40F0B0818F4A106844F24F6380
S31508014C3098428E4B1B7840F34C826FF0270101FB9B
S31508014C40030010608A4D8B49B5F90070B1F900600F
S31508014C50834B01241C704CE6824B93F90030002BE0
S31508014C6040F0B081804A1068B0F5167FACBF0538B0
S31508014C7000F1FF307E4D7F49B5F90070B1F900604A
S31508014C801060E5E7774B93F90030002B40F042813D
S31508014C90754A774D10687749B5F90070B1F9006022
S31508014CA014381060D4E76F4B93F90030002B40F0AD
S31508014CB07A816D4A106844F24F6398426B4B1B78B0
S31508014CC040F31182282111FB03001060BAE7654BF6
S31508014CD093F90030002B40F08F81634A1068B0F5D4
S31508014CE0167FACBF0A300130C4E75D4B5E4A604DA2
S31508014CF060491068B5F90070B1F900604FF0010C10
S31508014D0083F800C000232370F3E5564B93F900306E
S31508014D10002B40F06481544A554D10685549B5F940
S31508014D200070B1F900601430106091E7484A92F9B1
S31508014D300030002B47D0013B5BB249494548464DF7
S31508014D40464E137001230B70B6F90020B0F90030F6
S31508014D502968AEE53E480278013252B2022A38DCA9
S31508014D6002703F4A3B483C4D3C4EB0F90030296839
S31508014D7001241470B6F900209BE53A490B780133F2
S31508014D805BB2022B2CDC0B70354B374A384D39494F
S31508014D901068B5F90070B1F9006001241C70A8E526
S31508014DA0304C94F9003013B3013B5BB22C482E4AC0
S31508014DB02F4D3049237001230370B5F9007010682F
S31508014DC0B1F9006095E52C4C02252A20257008705A
S31508014DD0B3E72A4D032429222B7004700A70C0E711
S31508014DE0274D032429232A700C700370CCE7224926
S31508014DF002252A220D700270D8E7012B6CD11B4BB4
S31508014E00164E1A7834881348134DB0F900302968BC
S31508014E10224412B232806BE6012B40F089800F4E94
S31508014E200C4832880C4DB0F900302968143A12B290
S31508014E3032805DE6012B40F08980084E05483288AC
S31508014E40054DB0F900302968013A12B232804FE6B1
S31508014E505D2F002070060020E0070020700B00205F
S31508014E60CC0700205E2F0020FC0B0020D402002076
S31508014E702CBD01202ABD01205C2F00205F2F0020B8
S31508014E80602F0020012B6FD19B4E9C4B32881C78DA
S31508014E909B489C4DB0F900302968121B12B232802A
S31508014EA026E6012B40F0B580934E95483288954DFC
S31508014EB0B0F900302968143212B2328018E6012B93
S31508014EC01AD18D4E8E4832888E4DB0F90030296838
S31508014ED0013212B232800BE6022B40F02D81874B4C
S31508014EE0884D1C7829688648834EB0F90030B6F992
S31508014EF0002021442960FBE5022B40F01D81814DEC
S31508014F007F4829687C4EB0F90030B6F90020013196
S31508014F102960EDE5012B40F08A807B4D7B4A2F887D
S31508014F207B491068B1F900600A3F3FB22F808FE6CE
S31508014F30022B40F00181734D714829686E4EB0F914
S31508014F400030B6F9002014392960D1E5022B40F06A
S31508014F50F3806C4D6A482968674EB0F90030B6F996
S31508014F60002001392960C3E5022B40F0E580654D33
S31508014F70624B2C68197862485F4EB0F90030B6F971
S31508014F800020611A2960B3E5012B5DD15E4D5B4BAB
S31508014F902F881B785E495D4AB1F900601068FF1ACF
S31508014FA03FB22F8054E6012B5DD1544B564D1F78E5
S31508014FB02B885749554AB1F9006010681F443FB21A
S31508014FC02F8045E6012B5DD14F4D504A2F88504918
S31508014FD01068B1F90060053F3FB22F8038E6012B12
S31508014FE06AD1494D494A2F8849491068B1F9006083
S31508014FF00A373FB22F802BE6012B50D1424D434A47
S315080150002F8843491068B1F9006005373FB22F80F0
S315080150101EE6022B40F090803A4D39482968364EF3
S31508015020B0F90030B6F900201431296060E5022B89
S3150801503070D13749354A0E88334D1068B5F9007075
S315080150400A3E36B20E8003E6022B6CD130492B4B51
S315080150500E881B782C4D2D4AB5F900701068F61A82
S3150801506036B20E80F4E5022B5DD1244B28491E7811
S315080150700B88254D254AB5F9007010681E4436B2CD
S315080150800E80E5E5022B45D12149204A0E881E4DA1
S315080150901068B5F90070053E36B20E80D8E5022BC8
S315080150A038D11B49194A0E88174D1068B5F9007091
S315080150B0053636B20E80CBE5022B2BD11449134A9D
S315080150C00E88114D1068B5F900700A3636B20E8091
S315080150D0BEE5B0F5167FA6BF6FF0090101FB030017
S315080150E0C01A1060AEE5B0F5167FA6BF0A2111FBFE
S315080150F00300C0181060A5E5700B0020D40200203B
S3150801510070060020E00700202CBD0120FC0B0020C2
S315080151102ABD01200D4A0E4D0E491068B5F90070D9
S31508015120B1F9006094E50A4D0A49084AB5F90070D3
S31508015130B1F9006010688BE50748084D084EB0F9CB
S3150801514000302968B6F90020D2E400BFFC0B002024
S315080151502CBD01202ABD012070060020E007002091
S31508015160700B002008B5F6F741FD00F0FD03012B91
S3150801517003D0042818BF002008BD032008BD00BFBE
S315080151802DE9F04122492348DFF8A480224F234E16
S31508015190FDF7B6FD1F48FDF75DFD1E48FDF794FDB9
S315080151A01C480321FDF7FAFE1D4B1A481B6B00220A
S315080151B01146FDF72BFD1B4B1B4993F900201B4894
S315080151C035F0FCFB002498F800300021D3B197F99B
S315080151D00050AC4217D056F824000121F5F764FABD
S315080151E0254697F9003056F82500AB4203684FF07B
S315080151F000011B6908BF012101349847032CE2D13C
S31508015200BDE8F081254656F82500F5F74DFAE8E799
S3150801521060F6040820C00120682F0020280000201D
S315080152206C070020B80B0020DC3D05088C03002024
S31508015230541C00202DE9F04F60496148614F624DC9
S3150801524091B0FDF75DFD5E48FDF704FD5C48FDF78D
S315080152503BFD5B4890F82A3090F829600321F61A3D
S31508015260FDF79CFE594B56489B6A00221146FDF7ED
S31508015270CDFC97F90030F6B2002B40F0898003ACDB
S315080152802968204635F00AFCB6B223464C48324610
S315080152904121FDF7BBFC97F90130002B6ED1296836
S315080152A0204635F0FBFB2346454872004121FDF7B0
S315080152B0ADFC97F902304FEA4608002B54D129680C
S315080152C0204635F0EBFB23463D4806EB0802412113
S315080152D0FDF79CFC97F90330002B3BD12968204642
S315080152E035F0DCFB3648DFF8F490DFF8F4A0DFF898
S315080152F0F4B02346B20041218046FDF787FC3546C6
S31508015300002759F8041B4046FDF7E4FC0321C0F1C8
S315080153103C044046FDF742FE9AF90030BB42A4B26E
S315080153200ED02A4659F8043C214640460137FDF776
S315080153306DFC3544042FADB2E3D111B0BDE8F08F51
S315080153409BF800102A46404669BB214B1B68FDF7AE
S315080153505DFCE6E71F4A55F8233092F900201E49FD
S31508015360204635F02BFBBDE71A4A55F8233092F94A
S3150801537000201949204635F021FBA4E7154A55F8BE
S31508015380233092F900201449204635F017FB8AE7A5
S31508015390104A55F8233092F900200F4903AC2046EC
S315080153A035F00CFB70E700963C230021FEF7BEF8AA
S315080153B000214046FDF7F2FDB3E700BF60F6040899
S315080153C020C0012038030020A40700206C07002014
S315080153D0400B0020B80B0020F0520508D80A00201F
S315080153E0652F0020541C00202DE9F04FDFF8CC93DF
S315080153F099F9005093B02DB1012D00F0088113B031
S31508015400BDE8F08FDFF8B8B3DFF8B8A3D74CBBF91E
S315080154100030DAF80070D64AD6490392204607FBCF
S3150801542003F7FDF76DFC20460121FDF7B7FDD248CC
S31508015430D24ADFF880C3D24EDFF88C83A0FB07314E
S31508015440A2FB07E24FF41673890903FB1171D20B0C
S3150801545048F6A043ACFB01C103FB1273C908A0FBC4
S31508015460030300919B09C74905A835F0A7FA05ABBF
S3150801547036220A212046FDF7C9FBDAF80000C2499F
S31508015480C24B81FB00C183FB00720144C717C7EBFE
S315080154902111C7EBA20202EB420CC1EB0117A0EBEB
S315080154A0CC0CA0EB4700BA4F00910CEB8C0C87FB98
S315080154B000174FEA4C0C83FB0C13A7EBE0704FEA7D
S315080154C0EC7CCCEBA303B349019005A835F076FA39
S315080154D03E2205AB0A212046FDF798FBAE49204638
S315080154E0FDF70EFC2046FDF7B5FB2046FDF7ECFB64
S315080154F094F82A3094F8297020460321FF1AFDF7FB
S315080155004DFD9B4A2946936820462A46FDF77EFBB0
S31508015510BBF90030A14986FB0320DA17C2EBA002CA
S3150801552002EB8200A3EB4003FFB2BFB21BB212B279
S3150801553005A835F043FA3A4605AB7D212046FDF725
S3150801554065FBBBF900C0964B9649B3F9003086FB5B
S315080155500C024FEAEC70C0EBA20086FB032600EBB7
S315080155608002ACEB420CDA17C2EBA60202EB820E02
S315080155700FFA8CF6A3EB4E0300B2CDE900061BB277
S3150801558012B205A835F01AFA05AB7A007D21204634
S31508015590FDF73CFB7E00DAF800208349DFF82CA2F0
S315080155A005A835F00BFABA1905AB7D212046FDF79A
S315080155B02DFB79492046FDF7A3FB20460321FDF77C
S315080155C0EDFCAB463E4658F8041B2046FDF782FB28
S315080155D00321C0F178052046FDF7E0FC9AF9003071
S315080155E05B45ADB200F0FC80324658F8043C2946CA
S315080155F020460BF1010BFDF709FB3E44BBF1030FF6
S31508015600B6B2E0D199F90050012D7FF4F8AE574CA6
S315080156106149574D03952046FDF772FB2046FDF774
S3150801562019FB2046FDF750FB94F82A3094F82960B7
S3150801563020460321F61AFDF7B1FC0022AB68204685
S315080156401146FDF7E3FA594B1868B0F5167FF6B21D
S31508015650C0F2D080DFF87881554FB8F90030B7F934
S315080156600010454C454A534D03440B44A4FB030122
S31508015670A2FB03C24FF41670890900FB1131D20B44
S3150801568048F6A04000FB1233A5FB0151A4FB030316
S31508015690C90805AC00919B094749204635F08EF9A2
S315080156A0B6B2324623467D213048354DDFF824917E
S315080156B0DFF824A1DFF824B1FDF7A8FAB8F900301C
S315080156C03649DFF8A88085FB0320DA17C2EBA0026A
S315080156D002EB8200A3EB40031BB212B2204635F05F
S315080156E06DF9720023467D212048FDF78FFAB7F937
S315080156F000302A4985FB0325DA17C2EBA50202EB1E
S315080157008200A3EB40031BB212B2204635F056F9CC
S315080157107200234632447D214046FDF777FA1E4939
S315080157204046FDF7EDFA03214046FDF737FC3546BD
S31508015730002759F8041B4046FDF7CCFA0321C0F1AE
S3150801574078044046FDF72AFC9AF90030BB42A4B218
S3150801575063D02A4659F8043C214640460137FDF7ED
S3150801576055FA3544032FADB2E3D148E620C00120EE
S315080157706C07002014EF0408B5814E1BD55204E9C5
S3150801578067666666F03D050889888888ABAAAA2AED
S3150801579056555555083E050860F60408284F05086C
S315080157A0700B00202C3E0508403E0508FC0B002026
S315080157B02ABD0120CDCCCCCC4C3E0508A007002043
S315080157C070060020E0070020100700205D2F00204A
S315080157D02CBD01201C0700205E2F0020541C002030
S315080157E01D4B19783246204609BB039B1B68FDF7FA
S315080157F00DFAF9E6194B1A49DFF86C80194F83FB44
S315080158000023C217C2EBA30202EB820305ACA0EB8D
S315080158104303204635F0D2F842E79BF800102A46A2
S31508015820404671B9039B1B68FDF7F0F991E70097AC
S3150801583078230021FDF77AFE00212046FDF7AEFB0D
S31508015840D2E6009678230021FDF770FE0021404636
S31508015850FDF7A4FB7DE700BF541C0020676666665A
S31508015860284F05082ABD01202CBD01202DE9F04F3E
S31508015870A74DA849DFF8E4A293B02846FDF740FAF8
S315080158802846FDF7E7F92846FDF71EFA95F8293067
S3150801589095F82A209AF900409B1ADBB2029324B1A3
S315080158A0012C76D013B0BDE8F08F9B4B03931E46AF
S315080158B003212846FDF772FBF3682246214628464E
S315080158C0FDF7A4F9954BBDF808901A68944905ACFB
S315080158D0204635F073F823464A4669212846FDF7DE
S315080158E095F9904B8E49B3F90020204635F066F8B4
S315080158F023464FEA490269212846FDF787F98A4B6B
S315080159008749B3F9002020464FEA490635F056F88B
S315080159102346284609EB06026921FDF777F9834BE9
S3150801592093F90030022B00F0E18081499A1E204646
S3150801593035F044F87648DFF82882DFF828B223469E
S315080159404FEA890269210746FDF760F94D460026A7
S3150801595058F8041B3846FDF7BDF90321C0F1640464
S315080159603846FDF71BFB9BF90030B342A4B200F0A1
S3150801597097802A4658F8043C214638460136FDF7F1
S3150801598045F94D44042EADB2E2D19AF90040012CF5
S3150801599088D1614B5E4803931C460321FDF7FEFA45
S315080159A00022E3685A481146FDF730F9614B624A0D
S315080159B01C68624BBDF808901D68614982FB042387
S315080159C0E217C2EBA30202EB82036420A4EB4303B2
S315080159D000FB04F005AC90FBF5F00090204634F08E
S315080159E0EDFF23464A4669214948FDF70FF9554A0D
S315080159F0554B92F90020204653F8221034F0DEFF69
S31508015A00234643484FEA49026921FDF7FFF8474B08
S31508015A1093F90030022B4FEA49054BD044499A1EA7
S31508015A20204634F0CBFF09EB0502234669213848A5
S31508015A30374FDFF83481DFF834A1DFF818B1FDF705
S31508015A40E5F8424A424B92F90020204653F82210C3
S31508015A5034F0B4FF23464FEA890269213846FDF737
S31508015A60D5F84D46002658F8041B3846FDF732F995
S31508015A700321C0F164043846FDF790FA9AF900301B
S31508015A80B342A4B21DD02A4658F8043C21463846EA
S31508015A900136FDF7BBF84D44042EADB2E3D101E75B
S31508015AA02C4B19782A463846A9B9039B1B68FDF77A
S31508015AB0ADF85EE7284B93E8030005908DF81810BA
S31508015AC0B1E79BF800102A463846B1B9039B1B6813
S31508015AD0FDF79CF8D7E7CDF8009064230021FDF780
S31508015AE025FD00213846FDF759FA42E71A4B93E896
S31508015AF0030005908DF818101CE7CDF80090642373
S31508015B000021FDF713FD00213846FDF747FABAE7EC
S31508015B1020C0012060F604086C070020380900201F
S31508015B20403E05086A2F00206C2F0020B80B002084
S31508015B30603E0508040C002067666666FC0B0020BB
S31508015B40703E0508642F002054070020612F0020AD
S31508015B5048070020541C0020583E0508A0070020CD
S31508015B60280700205F2F002038070020602F00201B
S31508015B702DE9F04F6F49704891B0FDF7C1F86E48AD
S31508015B80FDF7A2F86C480321FDF708FA6B4B1B7861
S31508015B90002B00F097806A496748FDF7B1F8664817
S31508015BA0FDF758F86448FDF78FF863480321FDF7B8
S31508015BB0F5F9644B6048DB6A00221146FDF726F8C1
S31508015BC05E4B1B78002B00F09680012B00F0AA8013
S31508015BD0DFF8949199F90030F6224FF6FB78002BFD
S31508015BE018FB032803F1FF3298FBF2F81FFA88F82D
S31508015BF03CDD0024DFF874B14F4FDFF874A1264667
S31508015C0013E0ADB2721C514603A834F0D7FEA91DA4
S31508015C1003AB89B210223846FCF7F8FF013499F92B
S31508015C200030E4B29C42264620DA03213846FDF7C5
S31508015C30B5F99BF90030B34214FB08F5E1D13F4BA6
S31508015C401B78012B14FB08F513D0022B20D0002B4F
S31508015C50D7D114FB08F5ADB2691D0E23009389B29D
S31508015C600A230F223846FDF71BFBCBE711B0BDE827
S31508015C70F08FADB2691D0E230093384689B20A2307
S31508015C800F22FDF753FC00213846FDF787F9B9E7DE
S31508015C9014FB08F5ADB2691D0E230093384689B287
S31508015CA00A230F22FDF742FC291D102300933846CB
S31508015CB00E2289B20C23FDF7F3FA00213846FDF7C7
S31508015CC06DF99FE7204B1C482D220521FCF79EFF05
S31508015CD01E4B19482D220F21FCF798FF1C4B16481D
S31508015CE039220521FCF792FF1A4B13483922642100
S31508015CF0FCF78CFF4FE7184B0F4828221821FCF7B1
S31508015D0085FF164B0C4834220F21FCF77FFF144BF5
S31508015D10094834227021FCF779FF084B1B78012BBF
S31508015D207FF456AF0F4B044828221821FCF76EFF63
S31508015D304EE700BFC8FE040820C00120541C0020FD
S31508015D4060F604086C070020FCE70408A05405085F
S31508015D5034320508F8E70408843E0508A43E050818
S31508015D60AC3E0508B83E0508B80B0020662F002092
S31508015D70B84E05082DE9F04F2DED028BC94CCA49DD
S31508015D80DFF880A3DFF880B393B02046FCF7B8FFAD
S31508015D902046FCF75FFF2046FCF796FF94F82A3069
S31508015DA094F8296020460321F61AFDF7F7F8BF4B48
S31508015DB0002211465B682046FCF728FF204603218E
S31508015DC0FDF7ECF8BA4ABB4B92F90020F6B253F844
S31508015DD02210B6B205A834F0F1FD05AB20463246CD
S31508015DE06E21FCF713FF9AF8003023B19BF90020C6
S31508015DF0012A00F08D81B04BB04AB149750005A85A
S31508015E0034F0DCFD05ABA7482A466E21FCF7FEFEF9
S31508015E109AF80030012B2C4600F0B381022B00F0D2
S31508015E20FD80002B40F07981A34BA44AA449344450
S31508015E3005A834F0C3FD05AB9A4822466E21FCF746
S31508015E40E5FE9AF80030012B00F09581022B00F04F
S31508015E50ED8094480121FDF7A1F89AF800303BB18D
S31508015E609BF90030012B00F0F881022B00F00A8221
S31508015E70944A9FED950A136AD2699B1A002BB8BFFB
S31508015E805B4207EE903AF8EEE77AB40067EE807A5D
S31508015E909FED8E0ABDEEE78A0234B8EEC87A77EE30
S31508015EA0C77A27EE800A32F041FEFDEEC07A18EE77
S31508015EB0102A17EE903A092BCCBF8549854905A8C2
S31508015EC034F07CFD05AB774822460021FCF79EFE9F
S31508015ED09AF800303BB19BF90030012B00F0C781DD
S31508015EE0022B00F0CA817C4A9FED7C0A136AD269AB
S31508015EF09B1A002BB8BF5B4207EE903AF8EEE77A99
S31508015F0067EE807A9FED710ABDEEE78AB8EEC87A28
S31508015F1077EEC77A27EE800A32F008FEFDEEC07AE0
S31508015F2018EE102A17EE903A092BCCBF6C496D4929
S31508015F3005A834F043FD05AB5A4822464B21FCF728
S31508015F4065FE694B93F90030002B40F0F780674BEB
S31508015F50DFED676AC3ED006A9AF800303BB19BF939
S31508015F600030012B00F07F81022B00F09081614AFD
S31508015F70136AD2699FED550ADFF890919B1A002B97
S31508015F80B8BF5B4207EE903AF8EEE77A354687EEF8
S31508015F90A67A0027BDEEC78AF8EEC87A37EE677A81
S31508015FA027EE000A32F0C2FDFDEEC07A18EE102A7D
S31508015FB017EE903A092BCCBF4F49504905A834F042
S31508015FC0FDFC05AB224696213648FCF71FFE3548EF
S31508015FD003218046FCF7E2FF59F8041B4046FCF70B
S31508015FE079FE0321C0F164044046FCF7D7FF9BF90B
S31508015FF00030BB42E4B200F097802A4659F8043CC7
S31508016000214640460137FCF701FE3544032FADB260
S31508016010E2D113B0BDEC028BBDE8F08F9BF90030DD
S31508016020012B00F03881022B7FF4FEAE9BF900307C
S31508016030022B7FF40EAF06EB4604204A30491E4D6B
S3150801604005A834F0BBFC224605AB6E21154803941E
S31508016050FCF7DCFD05A91348FCF73CFE2946044676
S315080160601048FCF737FEE4B2C3B2039A0D4800960E
S31508016070013304F16D01FDF759FA0A480021FCF7CD
S315080160808DFF95E80300039AADF81810059004F101
S315080160906E0105AB0348FCF7B9FD02480321FCF77D
S315080160A07DFFD6E620C0012060F604086C070020B3
S315080160B0A007002008070020DC2E0508D02E0508B9
S315080160C0D43E0508E03000203F11A0390000C8423F
S315080160D0EC3E0508F83E0508243100209694F1386F
S315080160E0043F0508103F050840420020881D00208E
S315080160F074D13546741A00201C3F0508283F050847
S31508016100E43E0508541C00205C2F0020FC060020F4
S31508016110012B6FD0022B00F0BD809BF90020022ACB
S3150801612000F0F18074007FE69AF800102A4640468E
S31508016130B9B9AA4B1B68FCF769FD5EE7022B05D1C5
S31508016140A74BDFEDA86AC3ED006A05E7012B40F00E
S315080161504181DFEDA57AA24BF0EE676AC3ED007ABD
S31508016160FAE6009664230021FDF7E0F9002140468E
S31508016170FCF714FF41E79BF90030022B7FF469AE67
S3150801618007E09BF90030012B36D0022B7FF44CAE89
S315080161903444964B18680368DB6B98470546002814
S315080161A000F0E880924B934A934905A834F006FC1F
S315080161B005A99248FCF78EFD032105468F48FCF791
S315080161C0EDFEEBB2013322468C4800966D21FDF7B0
S315080161D0ADF98A480021FCF7E1FE05AB22466E219E
S315080161E08648FCF713FD85480321FCF7D7FE9AF884
S315080161F000302BE6740025467C4B18680368DB6B78
S3150801620098470746002800F08380794B794A7A49EE
S3150801621005A834F0D3FB05A97848FCF75BFD0321F3
S3150801622007467648FCF7BAFEFBB201332A4673489D
S3150801623000966D21FDF77AF970480021FCF7AEFE4C
S3150801624005AB2A466E216D48FCF7E0FC6B48032135
S31508016250FCF7A4FE9AF80030E0E5694A9FED690A61
S315080162605368126A09E6684A5368126A82E6674AF7
S315080162709FED670A5368126A3AE6644A9FED640A13
S31508016280536834E65E4A9FED5F0A5368F4E55E4A51
S3150801629053686EE67400A5B2564A5E49544F05A87E
S315080162A034F08CFB2A4605AB6E2154480395FCF75E
S315080162B0ADFC05A95148FCF70DFD394605464F4881
S315080162C0FCF708FDEDB2C3B2039A4C4800960133B8
S315080162D005F16D01FDF72AF948480021FCF75EFE34
S315080162E097E8030005AB039AADF81810059005F178
S315080162F06E014248FCF78AFC40480321FCF74EFE32
S315080163009AF800308DE5012B7FF4A0AD74003FE7C4
S31508016310DFF8E08039484146FCF7DCFC5FFA80F992
S3150801632009F101032A46354800966D21FDF7FEF865
S3150801633039463248FCF732FE98E8070005AF03C72D
S3150801634005AB3A706E212A462C48FCF75FFC2B48B0
S315080163500321FCF723FE264A2F4905A834F02EFB14
S3150801636005AB26482A4609F16E01FCF74FFC9AF857
S31508016370003053E5DFF87C8020484146FCF7AAFC4B
S31508016380C7B27B1C22461D4800966D21FDF7CEF843
S3150801639029461A48FCF702FE98E8070005AD03C529
S315080163A005AB2A706E2122461448FCF72FFC1348C8
S315080163B00321FCF7F3FD0E4A174905A834F0FEFA46
S315080163C005AB0E48224607F16E01FCF71FFC9AF849
S315080163D000303BE5024BD3ED006ABDE56C070020B2
S315080163E0881D0020DBAC2D47E4385E46681C00207A
S315080163F0DC2E0508D02E0508D43E050820C001204C
S31508016400E03000203F11A039741A00202431002001
S315080164109694F138E43E0508DC3E050800B5264B9E
S3150801642093F9003083B0DBB1012B2FD0022B33D087
S31508016430032B2BD0042B35D0072B27D0062B34D092
S31508016440052B0FD11D4A1E4B11780A2253F821003C
S3150801645001A935F0F3F901461A4825F005FE01E0D0
S3150801646025F0D0FD184B93F90030012B02D003B06B
S315080164705DF804FB15484368B3F5E13FF7D04FF4DF
S31508016480E13125F0F1FD03B05DF804FB0D484FF449
S31508016490E13125F0E9FDE5E70A484FF4613125F0D8
S315080164A0E3FDDFE725F076FDDCE706484FF4966164
S315080164B025F0DAFDD6E700BF282E0020BD350020DD
S315080164C0D45A050858C50120582000209CC501202A
S315080164D02DE9F04FA14FA24C97F90030A149032BA2
S315080164E0A9B040F36581072B40F39C800B2B40F341
S315080164F0ED820E2B40F39D83122B40F30182162B5E
S3150801650040F37C842046FCF7FBFB2046FCF7DCFBCA
S3150801651020460321FCF742FD0522934BDFF87C92C6
S31508016520DFF87C82914FF3212046FCF76FFB9049F7
S315080165302046FCF7E5FB2046FCF78CFB2046FCF7DA
S31508016540C3FB94F82A3094F8295020460321ED1A02
S31508016550FCF724FD874B88495A681BA834F02EFAA4
S31508016560002211461BAB2046FCF750FB834B84499E
S315080165701E68A9FB06235B09A8FB0320C3EB031CC2
S315080165800009720900EB4000A6EB8C06A3EBC003D9
S31508016590A7FB02C200961BA8002634F00FFA1BAA15
S315080165A00323012107A80096F4F766FC754B764983
S315080165B01A68A9FB02035B09A8FB03C00009C3EB20
S315080165C0031CA2EB8C0C4FEA521E00EB4000A7FB02
S315080165D00E72CDF800C0A3EBC0031BA834F0EEF988
S315080165E003231BAA1946009611A8F4F745FC07A828
S315080165F0F4F726FD11A8F4F723FD644BEDB21968EB
S315080166001BA834F04BFA1BABAA0028212046FCF73D
S31508016610FDFA11A8F4F75AFC07A8F4F757FC29B0B4
S31508016620BDE8F08F534B03932046FCF769FB2046E0
S31508016630FCF74AFB20460321FCF7B0FC4A4BDFF87E
S315080166406481534DDFF860910522F3212046FCF75A
S31508016650DDFA05224F4BF9212046FCF7D7FA4449C2
S315080166602046FCF74DFB2046FCF7F4FA2046FCF7DA
S315080166702BFB94F82A3094F8296020460321F61A50
S31508016680FCF78CFC039B44495A681BA834F096F91D
S31508016690002211461BAB2046FCF7B8FA98F90030E0
S315080166A0F6B2B6B255F823101BA834F0F7F93246FC
S315080166B01BAB41212046FCF7A9FA98F901301BA822
S315080166C055F8231034F0EAF972001BAB4121204634
S315080166D0FCF79CFA98F902304FEA460A55F8231056
S315080166E01BA834F0DBF906EB0A021BAB4121204655
S315080166F0FCF78CFA98F90330DFF8B0A055F82310A7
S315080167001BA834F0CBF91BABB20020464121FCF79C
S315080167107DFAA34635464FF0040859F8041B584636
S31508016720FCF7D8FA0321C0F13C045846FCF736FCBD
S3150801673097F900304345A4B200F0D6802A4659F8A5
S31508016740043C2146584608F10108FCF75FFA35442E
S31508016750B8F1080FADB2E0D161E700BF703F002084
S3150801676020C00120C8FE040834320508065BB005BE
S3150801677060F60408400B0020403F0508241B002052
S31508016780443F0508103A0020543F0508F80B00203D
S315080167901C0B0020F8E70408783F050889888888D3
S315080167A0ABAAAAAA340300208C0A0020541C002094
S315080167B0AF4D03952046FCF7A3FA2046FCF784FA69
S315080167C020460321FCF7EAFB0522AA4BDFF8EC92E7
S315080167D0DFF8F0A2F9212046FCF718FAA649204667
S315080167E0FCF78EFA2046FCF735FA2046FCF76CFAD8
S315080167F094F82A3094F8296020460321F61AFCF702
S31508016800CDFB6A689D491BA834F0D8F800221146C9
S315080168101BAB2046FCF7FAF9994A9A4B92F90020E4
S31508016820F6B2B6B253F822101BA834F037F932463D
S315080168301BAB8A212046FCF7E9F9934B93491A7851
S315080168401BA834F0BBF872001BAB8A212046FCF763
S31508016850DDF98F4B8D491A7875001BA834F0AEF80F
S3150801686072191BAB8A212046FCF7D0F9894A8A4B53
S3150801687092F900201BA853F8221034F00FF91BAB2C
S31508016880B20020468A21FCF7C1F9A34635464FF0E6
S31508016890000859F8041B5846FCF71CFA0321C0F1F5
S315080168A087045846FCF77AFB97F900304345A4B2AA
S315080168B00ED02A4659F8043C2146584608F10108E3
S315080168C0FCF7A4F93544B8F1040FADB2E1D1A6E657
S315080168D09AF800102A465846002940F0A081039BE1
S315080168E01B68FCF793F9E4E79AF800102A4658461C
S315080168F0002940F03982039B1B68FCF787F91DE7DD
S315080169005B4D03952046FCF7FBF92046FCF7DCF9BD
S3150801691020460321FCF742FB604BDFF8ACA10522B8
S31508016920F3212046FCF772F90522524BF92120463C
S31508016930FCF76CF950492046FCF7E2F92046FCF7CA
S3150801694089F92046FCF7C0F994F82A3094F8298089
S315080169502688049620460321A8EB0308FCF71EFBAC
S315080169606A684F491BA834F029F8002211461BAB67
S315080169702046FCF74BF94B4A4B4B92F900204FEA5C
S31508016980560BABF10F055FFA88F81FFA88F853F82A
S315080169902210ADB21BA834F081F8424629461BAB3A
S315080169A02046FCF733F9414A414B92F900201BA8CE
S315080169B053F8221034F072F84FEA480229461BAB05
S315080169C02046FCF723F93B4A3B4B92F900204FEA54
S315080169D0480653F822101BA834F060F808EB0602A3
S315080169E01BAB29462046FCF711F9ABF1140B1FFA2C
S315080169F08BFB46464FF00F095AF8041B2046FCF755
S31508016A0069F90321ABEB00052046FCF7C7FA97F9AC
S31508016A1000304B45ADB200F0BA8132465AF8043C13
S31508016A202946204609F10109FCF7F0F84644B9F16F
S31508016A30120FB6B2E0D1214D2148A96CFCF74AF9EB
S31508016A40049B181A00EBD07403211D48FCF7A6FA1B
S31508016A5097F90030122BC4F34F0400F0B3824FEAC2
S31508016A608802AB6C16482146FCF7D0F8D7E500BF7B
S31508016A70400B0020F8E7040860F60408343F0508CF
S31508016A809E0300204C0A00204C030020383F0508CD
S31508016A904D03002040420020040B00203432050833
S31508016AA06C3F0508282E0020600A0020C9B701207E
S31508016AB0100B002058200020580A00207C0A0020CC
S31508016AC020C00120541C0020B80A0020B64B0393AD
S31508016AD02046FCF715F92046FCF7F6F8204603216F
S31508016AE0FCF75CFAB14B0522F3212046FCF78EF838
S31508016AF00522AF4BF9212046FCF788F8AD49204617
S31508016B00FCF7FEF82046FCF7A5F82046FCF7DCF86A
S31508016B1094F82A3094F82960258820460321F61A24
S31508016B20FCF73CFA039BA4495A680DF16C084046E8
S31508016B3033F044FF0022434611462046FCF766F827
S31508016B409E4B1A78F6B2002A40F018819C4B0FCB5F
S31508016B5088E80F00B6B2434632468A219948DFF8DB
S31508016B606492DFF894A2DFF88CB2FCF74FF8964AE4
S31508016B70964B92F90020404653F8221033F08EFFC7
S31508016B80434672008A218F48FCF740F8904A914B98
S31508016B9092F90020404653F82210740033F07EFF24
S31508016BA0434632198A214846FCF730F88A4A8B4B04
S31508016BB01278690853F8223048460A31B200FCF7C0
S31508016BC025F835464FF008085AF8041B4846FCF7DD
S31508016BD081F80321C0F187044846FCF7DFF997F9E4
S31508016BE000304345A4B20ED02A465AF8043C214641
S31508016BF0484608F10108FCF709F83544B8F10C0FC5
S31508016C00ADB2E1D10BE59BF800102A4648460029AA
S31508016C1040F0B381039B1B68FBF7F8FFE4E7009696
S31508016C2087230021FCF782FC00215846FCF7B6F9B8
S31508016C303FE65D4B03932046FCF762F82046FCF7D6
S31508016C4043F820460321FCF7A9F9584B644D052260
S31508016C50F3212046FBF7DAFF0522554BF921204699
S31508016C60FBF7D4FF53492046FCF74AF82046FBF7C1
S31508016C70F1FF2046FCF728F894F82A3094F82960A1
S31508016C80B4F8008020460321F61AFCF787F9039B1E
S31508016C9054495A681BA833F091FE002211461BABD2
S31508016CA02046FBF7B3FF504A504B92F90020F6B243
S31508016CB053F822104FEA5809B6B21BA833F0EEFE74
S31508016CC01BAB324609F10A012046FBF79FFF296BE8
S31508016CD02046FBF7FFFF0321A9EB000320461FFA15
S31508016CE083FAFCF75BF997F900300C2B00F0BE81AB
S31508016CF02B6B344832465146FBF788FF696B31489E
S31508016D00FBF7E8FFA8EB000000EBD07403212D4840
S31508016D10FCF744F997F900300D2BC4F34F0400F042
S31508016D2098814FEA46094A466B6B26482146FBF786
S31508016D306DFFA96B2348FBF7CDFFA8EB000000EB1D
S31508016D40D07403211F48FCF729F997F900300E2B57
S31508016D50C4F34F0400F0958106EB0902AB6B1948A1
S31508016D602146FBF753FF5AE400963C230021FCF722
S31508016D70DDFB00215846FCF711F9DFE402EB82023C
S31508016D801B49C2EB0212404633F018FEE2E6194BE4
S31508016D90197832462046002940F02381039B1B6857
S31508016DA0FBF734FF39E600BF400B002034320508F3
S31508016DB0F8E7040860F60408743F0508F4B60120EC
S31508016DC07C3F050820C00120841D0020440A0020BC
S31508016DD0BC3E0020FC0A00202C0A0020F00A0020F4
S31508016DE07C0A0020703F05086E1A0020340A00202C
S31508016DF08C3F0508541C00209C0A0020C24B0393B3
S31508016E002046FBF77DFF2046FBF75EFF2046032160
S31508016E10FCF7C4F8BD4BBE4D0522F3212046FBF70E
S31508016E20F5FE0522BB4BF9212046FBF7EFFEBA49D1
S31508016E302046FBF765FF2046FBF70CFF2046FBF7CC
S31508016E4043FF94F82A3094F82960B4F800B0204634
S31508016E500321F61AFCF7A2F8AB4BB0495A680DF1B3
S31508016E606C08404633F0AAFD0022114643462046E7
S31508016E70FBF7CCFEAA4AAB4B92F90020F6B253F8BF
S31508016E8022104FEA5B0AB6B2404633F007FE434684
S31508016E9032460AF10A012046FBF7B8FEE96C20469C
S31508016EA0FBF718FF0321AAEB00092046FCF776F841
S31508016EB097F90030132B1FFA89F977D0EB6C9A48AA
S31508016EC049463246FBF7A2FE296D9748FBF702FFB2
S31508016ED0ABEB000000EBD07903219348FCF75EF891
S31508016EE097F90030142BC9F34F0950D07400224684
S31508016EF08D482B6DDFF818A249460546FBF786FE35
S31508016F001523344404961E4628460321FCF746F801
S31508016F1097F900309E4228466ED1844B84491B78E6
S31508016F204046002B79D0DAF8542033F047FD414624
S31508016F302846FBF7CFFE049B009381465B46224613
S31508016F4000212846ABEB0909FCF7F0FA09EBD979D8
S31508016F5000212846FCF722F8C9F34F014346224689
S31508016F602846FBF753FE049B162E1C44A4B20AF1CD
S31508016F70040A3FF454AB1626C6E700968723002178
S31508016F80FCF7D4FA00214846FCF708F82CE6674BCB
S31508016F9019787200002940F0A9805B4B62481B688A
S31508016FA004921446FBF732FE049AA1E75F4B19785F
S31508016FB0002940F0BF80544B20461B683246FBF738
S31508016FC025FE7BE7594B19784FEA8802002940F0DC
S31508016FD0BD80039B54481B680392FBF717FE039A6F
S31508016FE03FE5CDF800805B460021FCF79FFA0021BA
S31508016FF02046FBF7D3FF10E5DAF85410FBF76AFED3
S31508017000ABEB000000EBD070C0F34F01DAF8543057
S3150801701022462846FBF7FAFDA5E7DAF85410059348
S315080170202846FBF757FE059B81461946039BABEBA2
S31508017030090922461B68284609EBD979FBF7E6FDBB
S31508017040DAF85430C9F34F0122462846FBF7DEFD2C
S3150801705089E7364B1978720001BB039B32481B68D6
S3150801706004929146FBF7D2FD049A5DE62F4B1978F7
S3150801707000292FD1039B20461B683246FBF7C6FD24
S3150801708036E62A4B197806EB0902B1B9039B26485D
S315080170901B680392FBF7BAFD039A5FE6224800963E
S315080170A0434600210492FCF741FA1F480021FBF7E9
S315080170B075FF4FEA4609049A36E61B480096434689
S315080170C000210392FCF732FA17480021FBF766FF05
S315080170D0039A43E6204600964B4632460021FCF7C2
S315080170E025FA20460021FBF759FF01E60E480096CE
S315080170F05B4600210492FCF719FA0B480021FBF7BD
S315080171004DFF7400049AF3E6400B0020343205085B
S315080171107C0A0020F8E7040860F60408683F0508B9
S31508017120E8390020E80A002020C00120541C00206C
S31508017130943F050820460096534632460021FCF73F
S31508017140F5F920460021FBF729FFB7E6049B064817
S31508017150CDF8008000210392FCF7E8F902480021E6
S31508017160FBF71CFF039A7CE420C0012048B9074BB2
S3150801717093F86030012B05D90549064A00230B709F
S3150801718013707047044B01221A70F5E7A418002002
S31508017190A41D00205409002064B7012008B5F4F79E
S315080171A025FD012805D0032802D0042818BF002090
S315080171B008BD074B1B7B2BB901460648F3F774FA42
S315080171C0032008BD03480021F3F76EFA032008BD22
S315080171D0A41800206040002070B5F4F707FD0128C7
S315080171E001D0032070BD314E3578002D2ED03048A0
S315080171F0F3F756FA2F4B2E481968F3F735FE2E4842
S31508017200F3F74EFA2D48F3F74BFA2948F3F744FA00
S31508017210012834D02A480121F3F746FA29480121E1
S31508017220F3F742FA28480121F3F73EFA274B1B7870
S31508017230002B33D0022BD4D13378002BD1D0244B59
S315080172401D4801211970F3F72FFACAE704460146CA
S315080172501748F3F729FA174B15489968F3F704FE07
S315080172601B4B15481D702146F3F71EFA1348214694
S31508017270F3F71AFA0E48F3F70FFA0128CAD10C48A0
S31508017280F3F70AFA0128D1D10D48F3F709FA0D489F
S31508017290F3F706FA0C48F3F703FAC7E70C4A064868
S315080172A013700121F3F700FA032070BD2D1B00208E
S315080172B0702F0020B0070020903E0020B83800202B
S315080172C0781E002054380020E41F00202C0A0020D4
S315080172D0A41D0020012800D0704708B5054B0648B3
S315080172E0196833F0DBFBBDE8084003490322562041
S315080172F0F2F788B89C390020245101201D4B1B78D0
S315080173000B3B042B04D8DFE803F01218212D0400E7
S315080173107047194A19491368096805338B4213607E
S3150801732001DB01391160164B01221A7070471549A4
S31508017330134A01230B70137070470F4A0F491368DC
S31508017340096801338B421360EDDBEAE70A4B1A68D9
S31508017350053A002A1A60E6DA00221A60084B012269
S315080173601A707047044B1A68013A002A1A60DADA69
S31508017370F2E700BF64B70120681F0020E0B60120CC
S31508017380CC070020541C0020244B25491868DFF837
S31508017390A4C0F0B5DFF8A0E0C87004120C7145F27C
S315080173A05344DEF804200C805F248C700414000E0C
S315080173B0DCF804301B4F88711012CEF80820CA7108
S315080173C008721014120E7D688A721A12164ECB7242
S315080173D0CCF808300A731A141B0E8B732B124C71D6
S315080173E00B74746848722B144B742B0E8B7423120E
S315080173F00B7523144B75230E0C488B750D234A7395
S31508017400CB7519220A23CD73CC740B760270BD6035
S31508017410B4600748BDE8F0402AF0C2BA681F0020E8
S31508017420183A0020741A0020B81A0020FCB6012068
S3150801743058C5012024310020E0300020F8B58E4AD5
S31508017440137853B38D4B8E491B7801200B3B08707B
S31508017450202B42D8DFE813F0E800A6003C00BB0069
S31508017460D10041002801410040014100410041008D
S3150801747041004100410041004100410041004100F5
S3150801748041004100410041004100410041004100E5
S3150801749041004100410041000601784978480B78CE
S315080174A001240B3B0470212B38D8DFE803F04A513D
S315080174B05E657237373737373737373737373737BD
S315080174C03737373737373737373737373737374430
S315080174D06C4B1B78002B00F031816B4B6B4EB3F96B
S315080174E00000B6F90070042819DDF1F74BF8684B6E
S315080174F00022F1F7B1F8002F04460D4616DB38468F
S31508017500F1F740F802460B4620462946F1F716FBE5
S3150801751020B120462946F1F74FFB3080F8BD0522F8
S31508017520002F5C4D1A804FF00004E8DA0021002292
S3150801753000233180E8E7534A137883F00103137077
S31508017540F8BD55484F490123037013700B70F8BDF8
S315080175504C4B1B78002BE1D1504A92F90030002B95
S31508017560EDD0013B5BB21370EAE7464B1B78002B63
S31508017570D4D12A230B70F8BD424B1B78002BCDD1F1
S31508017580464A137801335BB2032BD8DD0323137004
S31508017590F8BD3C4B1B78002BC0D14048292203700B
S315080175A00A70F8BD374B1B78002B96D13B4B93F9E4
S315080175B00030012B00F0DC80022B8ED1334E324B8A
S315080175C03788B3F9000001373FB237808BE72D4B77
S315080175D01B78002B81D1314B93F90030012B00F038
S315080175E0E680022B7FF479AF284E274B3788B3F90B
S315080175F00000013F3FB2378075E7224B1B78002B0D
S315080176007FF46BAF254B93F90030012B00F0A7806F
S31508017610022B7FF462AF1D4E1B4B3788B3F900006E
S3150801762005373FB237805EE71C4B1B4893F900309C
S315080176300124002104701170002B65D0032B7FF4FF
S315080176404CAF1748174A104B104E116000240025FD
S31508017650C0E90045C0E90245B6F90070B3F9000072
S31508017660918040E7084B094EB3F90000B6F900705E
S315080176700021117037E700BF541C002064B70120B0
S31508017680CC0700206450012030050020300400207A
S315080176900000E03F0000044069060020EC2A0020B3
S315080176A028220020282A00204A4B1B78002B7FF429
S315080176B014AF494B93F90030012B6DD0022B7FF49F
S315080176C00CAF464E464B32881F78464B17443FB29D
S315080176D0B3F90000378006E73E4B1B78002B7FF491
S315080176E0FCAE3D4B93F90030012B4AD0022B7FF4B7
S315080176F0F4AE3A4E3A4B37881A783A4BBF1A3FB22C
S31508017700B3F900003780EEE63749384B384A394D28
S31508017710394C3A4849685B6864681160536038496E
S315080177206D68304B2D4ED460956004688288B6F931
S315080177300070B3F900000C608A80D4E6264B93F9F1
S315080177400030012B3CD0022B7FF4C7AE234E254BCC
S315080177503788B3F90000053F3FB23780C3E6214BAE
S315080177601E4E1888B6F90070053000B21880BAE6C0
S315080177701C4B1A4E1888B6F90070013000B21880F1
S31508017780B1E6184B164A18881278144E801A00B2B8
S31508017790B6F900701880A6E6124B11491A880878BE
S315080177A00E4E104400B2B6F9007018809BE60D4BD8
S315080177B00A4E1888B6F90070013800B2188092E6A8
S315080177C0084B064E1888B6F90070053800B21880BD
S315080177D089E600BF64500120EC2A0020300400200D
S315080177E0D402002030050020E0300020243100209A
S315080177F028220020741A0020B81A0020845101207A
S31508017800282A0020F8B58E4A137853B38D4B8E4932
S315080178101B7801200B3B0870202B42D8DFE813F0B8
S31508017820E800A6003C00BB00D10041002801410048
S315080178304001410041004100410041004100410031
S315080178404100410041004100410041004100410021
S315080178504100410041004100410041004100410011
S315080178600601784978480B7801240B3B0470212BD3
S3150801787038D8DFE803F04A515E657237373737374C
S315080178803737373737373737373737373737373779
S3150801789037373737373737446C4B1B78002B00F0AF
S315080178A033816B4B6B4EB3F90200B6F902700428AB
S315080178B019DDF0F767FE684B0022F0F7CDFE002FC1
S315080178C004460D4616DB3846F0F75CFE02460B46C3
S315080178D020462946F1F732F920B120462946F1F723
S315080178E06BF97080F8BD0522002F5C4D5A804FF068
S315080178F00004E8DA0021002200237180E8E7534AF0
S31508017900137883F001031370F8BD55484F490123D5
S31508017910037013700B70F8BD4C4B1B78002BE1D12B
S31508017920504A92F90030002BEDD0013B5BB213703F
S31508017930EAE7464B1B78002BD4D12A230B70F8BDF6
S31508017940424B1B78002BCDD1464A137801335BB2E3
S31508017950032BD8DD03231370F8BD3C4B1B78002B92
S31508017960C0D14048292203700A70F8BD374B1B78ED
S31508017970002B96D13B4B93F90030012B00F0DE80AA
S31508017980022B8ED1334E324B7788B3F90200013779
S315080179903FB277808BE72D4B1B78002B81D1314B7A
S315080179A093F90030012B00F0E880022B7FF479AFC0
S315080179B0284E274B7788B3F90200013F3FB27780FB
S315080179C075E7224B1B78002B7FF46BAF254B93F998
S315080179D00030012B00F0A980022B7FF462AF1D4E07
S315080179E01B4B7788B3F9020005373FB277805EE70C
S315080179F01C4B1B4893F900300124002104701170B7
S31508017A00002B65D0032B7FF44CAF1748174A104B50
S31508017A10104ED18000240025C0E90445C0E9064579
S31508017A20B6F90270B3F90200916040E7084B094EB6
S31508017A30B3F90200B6F902700021117037E700BFE9
S31508017A40541C002064B70120CC0700206450012093
S31508017A5030050020300400200000E03F000004400B
S31508017A6069060020EC2A002028220020282A002066
S31508017A704B4B1B78002B7FF414AF4A4B93F900301C
S31508017A80012B6FD0022B7FF40CAF474E474B728800
S31508017A901F78474B17443FB2B3F90200778006E7D0
S31508017AA03F4B1B78002B7FF4FCAE3E4B93F900301D
S31508017AB0012B4CD0022B7FF4F4AE3B4E3B4B77881F
S31508017AC01A783B4BBF1A3FB2B3F902007780EEE64C
S31508017AD03849394B394A3A4D3A4C3B4849685B680B
S31508017AE06D686468116153613849314B2E4E956151
S31508017AF0D461058844888288B6F90270B3F9020010
S31508017B00CD800C814A81D2E6264B93F90030012BB0
S31508017B103CD0022B7FF4C5AE234E254B7788B3F9AB
S31508017B200200053F3FB27780C1E6214B1E4E5888B9
S31508017B30B6F90270053000B25880B8E61C4B1A4EE9
S31508017B405888B6F90270013000B25880AFE6184B72
S31508017B50164A58881278144E801A00B2B6F902707D
S31508017B605880A4E6124B11495A8808780E4E1044DB
S31508017B7000B2B6F90270588099E60D4B0A4E58883C
S31508017B80B6F90270013800B2588090E6084B064EE5
S31508017B905888B6F90270053800B2588087E600BFE2
S31508017BA064500120EC2A002030040020D402002071
S31508017BB030050020E0300020243100202822002052
S31508017BC0741A0020B81A002084510120282A00209E
S31508017BD0F8B58E4A137853B38D4B8E491B7801201D
S31508017BE00B3B0870202B42D8DFE813F0E800A6000B
S31508017BF03C00BB00D1004100280141004001410081
S31508017C00410041004100410041004100410041005D
S31508017C10410041004100410041004100410041004D
S31508017C2041004100410041004100410006017849F7
S31508017C3078480B7801240B3B0470212B38D8DFE8F0
S31508017C4003F04A515E657237373737373737373773
S31508017C5037373737373737373737373737373737A5
S31508017C60373737446C4B1B78002B00F031816B4B4F
S31508017C706B4EB3F90400B6F90470042819DDF0F760
S31508017C8081FC684B0022F0F7E7FC002F04460D46FD
S31508017C9016DB3846F0F776FC02460B46204629469F
S31508017CA0F0F74CFF20B120462946F0F785FFB08052
S31508017CB0F8BD0522002F5C4D9A804FF00004E8DAE2
S31508017CC0002100220023B180E8E7534A137883F0A4
S31508017CD001031370F8BD55484F490123037013700A
S31508017CE00B70F8BD4C4B1B78002BE1D1504A92F929
S31508017CF00030002BEDD0013B5BB21370EAE7464B2F
S31508017D001B78002BD4D12A230B70F8BD424B1B7864
S31508017D10002BCDD1464A137801335BB2032BD8DD4C
S31508017D2003231370F8BD3C4B1B78002BC0D1404888
S31508017D30292203700A70F8BD374B1B78002B96D1A0
S31508017D403B4B93F90030012B00F0DC80022B8ED1DE
S31508017D50334E324BB788B3F9040001373FB2B780C7
S31508017D608BE72D4B1B78002B81D1314B93F90030D2
S31508017D70012B00F0E680022B7FF479AF284E274BC2
S31508017D80B788B3F90400013F3FB2B78075E7224BC4
S31508017D901B78002B7FF46BAF254B93F90030012B31
S31508017DA000F0A780022B7FF462AF1D4E1B4BB788EC
S31508017DB0B3F9040005373FB2B7805EE71C4B1B4891
S31508017DC093F900300124002104701170002B65D04D
S31508017DD0032B7FF44CAF1748174A104B104ED1604E
S31508017DE000240025C0E90845C0E90A45B6F904702A
S31508017DF0B3F90400118240E7084B094EB3F90400B0
S31508017E00B6F904700021117037E700BF541C002031
S31508017E1064B70120CC0700206450012030050020FA
S31508017E20300400200000E03F0000044069060020FD
S31508017E30EC2A002028220020282A00204A4B1B78F9
S31508017E40002B7FF414AF494B93F90030012B6DD009
S31508017E50022B7FF40CAF464E464BB2881F78464B31
S31508017E6017443FB2B3F90400B78006E73E4B1B78C7
S31508017E70002B7FF4FCAE3D4B93F90030012B4AD021
S31508017E80022B7FF4F4AE3A4E3A4BB7881A783A4B3E
S31508017E90BF1A3FB2B3F90400B780EEE63749384B4B
S31508017EA0384A394D394C3A4849685B686468116201
S31508017EB0536238496D68304B2D4ED4629562046819
S31508017EC08288B6F90470B3F90400CC600A82D4E654
S31508017ED0264B93F90030012B3CD0022B7FF4C7AE19
S31508017EE0234E254BB788B3F90400053F3FB2B78047
S31508017EF0C3E6214B1E4E9888B6F90470053000B2C8
S31508017F009880BAE61C4B1A4E9888B6F90470013067
S31508017F1000B29880B1E6184B164A98881278144E22
S31508017F20801A00B2B6F904709880A6E6124B114978
S31508017F309A8808780E4E104400B2B6F904709880F3
S31508017F409BE60D4B0A4E9888B6F90470013800B2C3
S31508017F50988092E6084B064E9888B6F9047005385B
S31508017F6000B2988089E600BF64500120EC2A0020FF
S31508017F7030040020D402002030050020E030002023
S31508017F802431002028220020741A0020B81A002063
S31508017F9084510120282A0020F8B58E4A137853B354
S31508017FA08D4B8E491B7801200B3B0870202B42D83C
S31508017FB0DFE813F0E800A6003C00BB00D100410051
S31508017FC028014100400141004100410041004100B2
S31508017FD0410041004100410041004100410041008A
S31508017FE0410041004100410041004100410041007A
S31508017FF0410041000601784978480B7801240B3B7A
S315080180000470212B38D8DFE803F04A515E657237D0
S3150801801037373737373737373737373737373737E1
S315080180203737373737373737373737446C4B1B7856
S31508018030002B00F033816B4B6B4EB3F90600B6F992
S315080180400670042819DDF0F79DFA684B0022F0F74F
S3150801805003FB002F04460D4616DB3846F0F792FA65
S3150801806002460B4620462946F0F768FD20B1204610
S315080180702946F0F7A1FDF080F8BD0522002F5C4DD9
S31508018080DA804FF00004E8DA002100220023F180AB
S31508018090E8E7534A137883F001031370F8BD55488E
S315080180A04F490123037013700B70F8BD4C4B1B78B5
S315080180B0002BE1D1504A92F90030002BEDD0013B5B
S315080180C05BB21370EAE7464B1B78002BD4D12A23FF
S315080180D00B70F8BD424B1B78002BCDD1464A13785D
S315080180E001335BB2032BD8DD03231370F8BD3C4B78
S315080180F01B78002BC0D14048292203700A70F8BDAD
S31508018100374B1B78002B96D13B4B93F90030012B4B
S3150801811000F0DE80022B8ED1334E324BF788B3F94D
S31508018120060001373FB2F7808BE72D4B1B78002BF2
S3150801813081D1314B93F90030012B00F0E880022BF5
S315080181407FF479AF284E274BF788B3F90600013F2C
S315080181503FB2F78075E7224B1B78002B7FF46BAF94
S31508018160254B93F90030012B00F0A980022B7FF4EF
S3150801817062AF1D4E1B4BF788B3F9060005373FB2B0
S31508018180F7805EE71C4B1B4893F900300124002158
S3150801819004701170002B65D0032B7FF44CAF174880
S315080181A0174A104B104E518200240025C0E90C4590
S315080181B0C0E90E45B6F90670B3F90600516140E704
S315080181C0084B094EB3F90600B6F90670002111707D
S315080181D037E700BF541C002064B70120CC070020F4
S315080181E06450012030050020300400200000E03FE3
S315080181F00000044069060020EC2A002028220020FD
S31508018200282A00204B4B1B78002B7FF414AF4A4BCE
S3150801821093F90030012B6FD0022B7FF40CAF474E38
S31508018220474BF2881F78474B17443FB2B3F906000C
S31508018230F78006E73F4B1B78002B7FF4FCAE3E4BDD
S3150801824093F90030012B4CD0022B7FF4F4AE3B4E50
S315080182503B4BF7881A783B4BBF1A3FB2B3F9060076
S31508018260F780EEE63849394B394A3A4D3A4C3B489C
S3150801827049685B686D686468116353633849314BB3
S315080182802E4E9563D463058844888288B6F90670AC
S31508018290B3F906004D828C82CA82D2E6264B93F93F
S315080182A00030012B3CD0022B7FF4C5AE234E254B63
S315080182B0F788B3F90600053F3FB2F780C1E6214BBF
S315080182C01E4ED888B6F90670053000B2D880B8E6D1
S315080182D01C4B1A4ED888B6F90670013000B2D88000
S315080182E0AFE6184B164AD8881278144E801A00B28F
S315080182F0B6F90670D880A4E6124B1149DA880878CF
S315080183000E4E104400B2B6F90670D88099E60D4BA8
S315080183100A4ED888B6F90670013800B2D88090E6B8
S31508018320084B064ED888B6F90670053800B2D880CB
S3150801833087E600BF64500120EC2A002030040020A3
S31508018340D402002030050020E0300020243100202E
S3150801835028220020741A0020B81A0020845101200E
S31508018360282A0020514A524B5249F0B514881C80DC
S3150801837024B224EAE47442F20F739C42A8BF1C4655
S31508018380E31D89B001224C4E4C4D03EB24235B427D
S31508018390174601A8337032F011FB49492F703A4646
S315080183A001A832F00BFB4349062202A832F006FB6C
S315080183B043492F70062202A832F000FB3D490022EC
S315080183C004A832F0FBFA3F492F70002204A832F0C4
S315080183D0F5FA3849224606A832F0F0FAC3B203285C
S315080183E02B7045D0022B54D0012B58D03278314905
S315080183F003A832F0E3FA0128287044D032499DF8DF
S3150801840004009DF8052048703A209DF80840087038
S315080184108A709DF809009DF81020CC7008719DF8A6
S3150801842011409DF812004A719DF813208C71C8718C
S315080184309DF818409DF819000A729DF81A204C7289
S3150801844088729DF81B409DF80C00CA721F4B9DF857
S315080184500D200C7348738A730D240A201122CC73DC
S3150801846008742A7093F90030012B07D009B0F0BDC2
S315080184701349224606A832F0A1FAB7E7144829F0AB
S315080184808FFA09B0F0BD32780D4903A832F096FA91
S31508018490B4E71049224606A832F090FAA6E7094938
S315080184A0224606A832F08AFAA0E700BF8C510120BD
S315080184B084510120A03F050833510120FCB6012053
S315080184C0A43F0508A83F0508902000205820002051
S315080184D09CC50120B03F0508514A524B5249F0B597
S315080184E054885C8024B224EAE47442F20F739C42F5
S315080184F0A8BF1C4604F1080389B04C4E4C4D03EB4A
S3150801850024235B42022201A83370012732F056FA6E
S3150801851048492F70022201A832F050FA4249062230
S3150801852002A832F04BFA43492F70062202A832F00C
S3150801853045FA3D49002204A832F040FA3E492F7017
S31508018540002204A832F03AFA3749224606A832F040
S3150801855035FAC3B203282B7045D0022B54D0012B10
S3150801856058D03278304903A832F028FA0128287001
S3150801857044D032499DF804009DF8052048703A20F8
S315080185809DF8084008708A709DF809009DF810202A
S31508018590CC7008719DF811409DF812004A719DF83A
S315080185A013208C71C8719DF818409DF819000A723C
S315080185B09DF81A204C7288729DF81B409DF80C0094
S315080185C0CA721F4B9DF80D200C7348738A730D24CC
S315080185D00A201122CC7308742A7093F90030012BF2
S315080185E007D009B0F0BD1349224606A832F0E6F9CC
S315080185F0B7E7144829F0D4F909B0F0BD32780D4926
S3150801860003A832F0DBF9B4E70F49224606A832F08F
S31508018610D5F9A6E70849224606A832F0CFF9A0E718
S315080186208C51012084510120A03F050833510120B6
S31508018630FCB60120A43F0508A83F050890200020A4
S31508018640582000209CC50120B03F050830B585B0EB
S3150801865020B10128034620D005B030BD224A234C5B
S3150801866053680093D36E224952692248032525701F
S3150801867032F0A4F9204B1F49C2B21A701F484FF4B1
S315080186807A7329F04BF841F2883023F071FD012104
S315080186901B48F1F799FC05B030BD1A4A1A491078FA
S315080186A01A4A124C137051F8200000230A2203A912
S315080186B0237033F0C3F8114B5A68904203D0014630
S315080186C0184623F0D1FC084B11499A68094832F03B
S315080186D075F9094B0749C2B21A7008484FF47A73FB
S315080186E029F01CF805B030BDBC030020BC350020BC
S315080186F0B83F050800B70120FCB6012058C501207E
S3150801870068B70120BD350020D45A05080236002075
S31508018710D83E05082DE9F043044689B0002851D012
S31508018720012802D009B0BDE8F083374B374ADFF894
S31508018730EC90B2F80080364C93E8070003AE0023AC
S3150801874086E80700CDE9063305273046EFF76AFDC7
S3150801875003463146484626F80380F1F7EFFF2046DF
S31508018760FAF780FB2B4D2846F3F7A8FA2046FAF7C5
S3150801877095FB0028F7D14FF47A7023F0F9FC013FF5
S31508018780E3D125492548F1F7D9FF2548254A264940
S31508018790264B0078107001220F701A70FDF73EFE05
S315080187A0234B24499A68244832F008F9234B224975
S315080187B0C2B21A7022484FF47A7328F0AFFF09B093
S315080187C0BDE8F0831F492048174DF0F765FD184AA3
S315080187D01E485368009304700324D36E1C495269DA
S315080187E02C70154832F0EAF8144B1349C2B21A70C4
S315080187F013484FF47A7328F091FF01210748F1F7DE
S31508018800E3FB09B0BDE8F08348E50408C03505086F
S3150801881020C00120FC410020C83F0508F41E0020A5
S3150801882020510120BD350020BC350020023600202C
S31508018830BC030020D83E050800B70120FCB601207C
S3150801884058C50120C03F0508CC3000200436002059
S31508018850B83F05082DE9F04F85B0F3F7C7F90128A8
S315080188602CD0C31EDBB2012B044665D920B10024E6
S31508018870204605B0BDE8F08F354B1B782B2BF7D179
S31508018880344E354933783548354D022B0CBF042310
S3150801889000233370F1F752FF324A3349536833489C
S315080188A0926E2C7032F08AF8314B3049C2B21A7086
S315080188B030484FF47A7328F031FFD9E72E4BDFF8A9
S315080188C0A090244E2B4F99F80080DFF898B0DFF876
S315080188D0B0A00FCB6C46002584E80F0035703846EA
S315080188E0B8F1000F22D154F8041B23F0BDFBDBF8C5
S315080188F008201E48514632F061F81D4B1B49C2B289
S315080189001A7038464FF47A7328F008FFC82023F006
S315080189102FFC32786B1CDBB29AB9042B06D099F876
S3150801892000801D463846B8F1000FDCD000230B48FD
S3150801893033700121F1F7B8FE0324204605B0BDE8DE
S31508018940F08F0E4B05481D704146F1F7ADFEF3E772
S3150801895064B70120BC350020D43F0508F41E002069
S3150801896002360020BC030020544A050800B701203E
S31508018970FCB6012058C501205CE50408BD35002078
S31508018980D83E0508000000002DE9F047844D2C6803
S315080189902DED028B002C32D1824B834E1B68326837
S315080189A0013B934209D001DD013232607F4B01223E
S315080189B01A70BDEC028BBDE8F0877D4C7D4F23789C
S315080189C0002B00F0988023F0CDFB7B4B3A68821A86
S315080189D0B3F9000008EE102AEFF7D4FD774B002211
